:020000040800F2
:108000000000012049EE00082DE2000831E20008DE
:1080100035E2000839E200083DE2000800000000F7
:1080200000000000000000000000000041E2000825
:1080300045E200080000000049E200084DE20008A7
:1080400091EE000891EE000891EE000891EE000814
:1080500091EE000891EE000891EE000891EE000804
:1080600091EE000891EE000891EE000851E2000840
:1080700081E200088DE2000891EE000891EE000810
:1080800099E20008A5E20008B1E2000891EE0008BC
:10809000E1E2000891EE000891EE000891EE000880
:1080A00091EE000891EE000891EE000891EE0008B4
:1080B00091EE000811E3000891EE000891EE00082F
:1080C00091EE000891EE000891EE000891EE000894
:1080D00091EE000841E300084DE3000879E3000851
:1080E00091EE000891EE000891EE000800000000FB
:1080F0000000000000000000000000000000000080
:10810000000000000000000091EE000891EE000861
:1081100091EE0008A5E3000891EE000891EE00083A
:1081200091EE000891EE000891EE000891EE000833
:1081300091EE000891EE000891EE0008D1E30008EE
:1081400091EE000801E4000891EE000891EE0008AD
:10815000000000000000000000000000000000001F
:10816000000000000000000000000000000000000F
:1081700000000000000000000000000000000000FF
:1081800000000000000000000000000000000000EF
:1081900000000000000000000000000000000000DF
:1081A00000000000000000000000000000000000CF
:1081B00000000000000000000000000000000000BF
:1081C00000000000000000000000000000000000AF
:1081D000000000000000000000000000000000009F
:0881E0005FF8E0F166666666D7
:1081E80010B5054C237833B9044B13B10448AFF3E9
:1081F80000800123237010BD5802002000000000F9
:10820800F07A010808B5034B1BB103490348AFF3E3
:10821800008008BD000000005C020020F07A010820
:10822800034613F8012B002AFBD1181A01387047AE
:1082380081F0004102E000BF83F0004330B54FEA0F
:1082480041044FEA430594EA050F08BF90EA020F7C
:108258001FBF54EA000C55EA020C7FEA645C7FEA0F
:10826800655C00F0E2804FEA5454D4EB5555B8BF32
:108278006D420CDD2C4480EA020281EA030382EAA3
:10828800000083EA010180EA020281EA0303362D35
:1082980088BF30BD11F0004F4FEA01314FF4801C08
:1082A8004CEA113102D0404261EB410113F0004F1A
:1082B8004FEA03334CEA133302D0524263EB4303D1
:1082C80094EA050F00F0A780A4F10104D5F1200E6F
:1082D8000DDB02FA0EFC22FA05F2801841F10001CA
:1082E80003FA0EF2801843FA05F359410EE0A5F19E
:1082F80020050EF1200E012A03FA0EFC28BF4CF0CF
:10830800020C43FA05F3C01851EBE37101F0004584
:1083180007D54FF0000EDCF1000C7EEB00006EEB91
:108328000101B1F5801F1BD3B1F5001F0CD349081B
:108338005FEA30004FEA3C0C04F101044FEA445272
:1083480012F5800F80F09A80BCF1004F08BF5FEAF9
:10835800500C50F1000041EB045141EA050130BDD9
:108368005FEA4C0C404141EB0101013C28BFB1F5EB
:10837800801FE9D291F0000F04BF01460020B1FA36
:1083880081F308BF2033A3F10B03B3F120020CDA09
:108398000C3208DD02F1140CC2F10C0201FA0CF0E7
:1083A80021FA02F10CE002F11402D8BFC2F1200C4C
:1083B80001FA02F120FA0CFCDCBF41EA0C01904002
:1083C800E41AA2BF01EB0451294330BD6FEA04044B
:1083D8001F3C1CDA0C340EDC04F11404C4F1200236
:1083E80020FA04F001FA02F340EA030021FA04F348
:1083F80045EA030130BDC4F10C04C4F1200220FA9F
:1084080002F001FA04F340EA0300294630BD21FADC
:1084180004F0294630BD94F0000F83F4801306BFA2
:1084280081F480110134013D4EE77FEA645C18BF96
:108438007FEA655C29D094EA050F08BF90EA020F2D
:1084480005D054EA000C04BF1946104630BD91EA25
:10845800030F1EBF0021002030BD5FEA545C05D128
:108468004000494128BF41F0004130BD14F5800467
:108478003CBF01F5801130BD01F0004545F0FE41DB
:1084880041F470014FF0000030BD7FEA645C1ABF10
:10849800194610467FEA655C1CBF0B46024650EA47
:1084A800013406BF52EA033591EA030F41F4002173
:1084B80030BD00BF90F0000F04BF0021704730B5F9
:1084C8004FF4806404F132044FF000054FF00001CE
:1084D80050E700BF90F0000F04BF0021704730B58F
:1084E8004FF4806404F1320410F0004548BF404264
:1084F8004FF000013EE700BF42004FEAE2014FEAB9
:1085080031014FEA02701FBF12F07F4393F07F4F93
:1085180081F06051704732F07F4208BF704793F096
:108528007F4F04BF41F40021704730B54FF46074A9
:1085380001F0004521F000411CE700BF50EA0102AC
:1085480008BF704730B54FF000050AE050EA010255
:1085580008BF704730B511F0004502D5404261EBC5
:1085680041014FF4806404F132045FEA915C3FF406
:10857800D8AE4FF003025FEADC0C18BF03325FEAA3
:10858800DC0C18BF033202EBDC02C2F1200300FA54
:1085980003FC20FA02F001FA03FE40EA0E0021FA79
:1085A80002F11444BDE600BF70B54FF0FF0C4CF467
:1085B800E06C1CEA11541DBF1CEA135594EA0C0F19
:1085C80095EA0C0F00F0DEF82C4481EA030621EA54
:1085D8004C5123EA4C5350EA013518BF52EA03358F
:1085E80041F4801143F4801338D0A0FB02CE4FF041
:1085F8000005E1FB02E506F00042E0FB03E54FF071
:108608000006E1FB03569CF0000F18BF4EF0010E68
:10861800A4F1FF04B6F5007F64F5407404D25FEA64
:108628004E0E6D4146EB060642EAC62141EA555117
:108638004FEAC52040EA5E504FEACE2EB4F1FD0C59
:1086480088BFBCF5E06F1ED8BEF1004F08BF5FEAD7
:10865800500E50F1000041EB045170BD06F0004689
:1086680046EA010140EA020081EA0301B4EB5C0436
:10867800C2BFD4EB0C0541EA045170BD41F480112E
:108688004FF0000E013C00F3AB8014F1360FDEBF53
:10869800002001F0004170BDC4F10004203C35DA2F
:1086A8000C341BDC04F11404C4F1200500FA05F3B2
:1086B80020FA04F001FA05F240EA020001F0004253
:1086C80021F0004110EBD37021FA04F642EB0601C9
:1086D8005EEA430E08BF20EAD37070BDC4F10C04F3
:1086E800C4F1200500FA04F320FA05F001FA04F2B7
:1086F80040EA020001F0004110EBD37041F10001A3
:108708005EEA430E08BF20EAD37070BDC4F12005AD
:1087180000FA05F24EEA020E20FA04F301FA05F215
:1087280043EA020321FA04F001F0004121FA04F2BD
:1087380020EA020000EBD3705EEA430E08BF20EA8D
:10874800D37070BD94F0000F0FD101F000464000C7
:1087580041EB010111F4801F08BF013CF7D041EA49
:10876800060195F0000F18BF704703F0004652004D
:1087780043EB030313F4801F08BF013DF7D043EA1E
:108788000603704794EA0C0F0CEA135518BF95EAD4
:108798000C0F0CD050EA410618BF52EA4306D1D15B
:1087A80081EA030101F000414FF0000070BD50EA7A
:1087B800410606BF1046194652EA430619D094EA04
:1087C8000C0F02D150EA013613D195EA0C0F05D1EE
:1087D80052EA03361CBF104619460AD181EA030142
:1087E80001F0004141F0FE4141F470014FF00000FA
:1087F80070BD41F0FE4141F4780170BD70B54FF095
:10880800FF0C4CF4E06C1CEA11541DBF1CEA135514
:1088180094EA0C0F95EA0C0F00F0A7F8A4EB0504F6
:1088280081EA030E52EA03354FEA013100F08880ED
:108838004FEA03334FF0805545EA131343EA1263B6
:108848004FEA022245EA111545EA10654FEA00266B
:108858000EF000419D4208BF964244F1FD0404F524
:10886800407402D25B084FEA3202B61A65EB030580
:108878005B084FEA32024FF480104FF4002CB6EB3D
:10888800020E75EB030E22BFB61A754640EA0C00BD
:108898005B084FEA3202B6EB020E75EB030E22BFFD
:1088A800B61A754640EA5C005B084FEA3202B6EB3E
:1088B800020E75EB030E22BFB61A754640EA9C00FD
:1088C8005B084FEA3202B6EB020E75EB030E22BFCD
:1088D800B61A754640EADC0055EA060E18D04FEA8B
:1088E800051545EA16754FEA06164FEAC30343EA2B
:1088F80052734FEAC2025FEA1C1CC0D111F4801FF8
:108908000BD141EA00014FF000004FF0004CB6E7F0
:1089180011F4801F04BF01430020B4F1FD0C88BF8F
:10892800BCF5E06F3FF6AFAEB5EB030C04BFB6EB9A
:10893800020C5FEA500C50F1000041EB045170BD8D
:108948000EF0004E4EEA113114EB5C04C2BFD4EBBA
:108958000C0541EA045170BD41F480114FF0000E3E
:10896800013C90E645EA060E8DE60CEA135594EABA
:108978000C0F08BF95EA0C0F3FF43BAF94EA0C0FBD
:108988000AD150EA01347FF434AF95EA0C0F7FF432
:1089980025AF104619462CE795EA0C0F06D152EA86
:1089A80003353FF4FDAE1046194622E750EA41066A
:1089B80018BF52EA43067FF4C5AE50EA41047FF47B
:1089C8000DAF52EA43057FF4EBAE12E74FF0FF3CE0
:1089D80006E000BF4FF0010C02E000BF4FF0010CB1
:1089E8004DF804CD4FEA410C7FEA6C5C4FEA430C2A
:1089F80018BF7FEA6C5C1BD001B050EA410C0CBF79
:108A080052EA430C91EA030F02BF90EA020F0020DA
:108A1800704710F1000F91EA030F58BF994208BF41
:108A280090422CBFD8176FEAE37040F001007047FE
:108A38004FEA410C7FEA6C5C02D150EA013C07D155
:108A48004FEA430C7FEA6C5CD6D152EA033CD3D0A0
:108A58005DF8040B704700BF8446104662468C469A
:108A68001946634600E000BF01B5FFF7B7FF0028CD
:108A780048BF10F1000F01BD4DF808EDFFF7F4FFF6
:108A88000CBF012000205DF808FB00BF4DF808ED81
:108A9800FFF7EAFF34BF012000205DF808FB00BFA4
:108AA8004DF808EDFFF7E0FF94BF012000205DF8C6
:108AB80008FB00BF4DF808EDFFF7CEFF94BF01207B
:108AC80000205DF808FB00BF4DF808EDFFF7C4FF74
:108AD80034BF012000205DF808FB00BF4FEA410CBD
:108AE8007FEA6C5C02D150EA013C0AD14FEA430CA0
:108AF8007FEA6C5C02D152EA033C02D14FF00000DD
:108B080070474FF0010070474FEA410212F500121A
:108B180015D211D56FF47873B3EB625212D94FEABC
:108B2800C12343F0004343EA505311F0004F23FAA6
:108B380002F018BF404270474FF00000704750EAFB
:108B4800013005D111F0004008BF6FF000407047B8
:108B58004FF00000704700BF4FEA4102B2F1E04316
:108B680024BFB3F5001CDCF1FE5C0DD901F0004C0C
:108B78004FEAC0024CEA5070B2F1004F40EB83005C
:108B880008BF20F00100704711F0804F21D113F188
:108B98003872BCBF01F00040704741F480114FEAC1
:108BA8005252C2F11802C2F1200C10FA0CF320FA4A
:108BB80002F018BF40F001004FEAC1234FEAD32367
:108BC80003FA0CFC40EA0C0023FA02F34FEA4303D1
:108BD800CCE77FEA625307D150EA01331EBF4FF05A
:108BE800FE4040F44000704701F0004040F0FE4075
:108BF80040F40000704700BF80F0004002E000BF72
:108C080081F0004142001FBF5FEA410392EA030F6F
:108C18007FEA226C7FEA236C6AD04FEA1262D2EBB9
:108C28001363C1BFD218414048404140B8BF5B42BE
:108C3800192B88BF704710F0004F40F4000020F057
:108C48007F4018BF404211F0004F41F4000121F06D
:108C58007F4118BF494292EA030F3FD0A2F10102B7
:108C680041FA03FC10EB0C00C3F1200301FA03F1F5
:108C780000F0004302D5494260EB4000B0F5000F18
:108C880013D3B0F1807F06D340084FEA310102F1D7
:108C98000102FE2A51D2B1F1004F40EBC25008BF89
:108CA80020F0010040EA03007047490040EB000053
:108CB800013A28BFB0F5000FEDD2B0FA80FCACF154
:108CC800080CB2EB0C0200FA0CF0AABF00EBC25081
:108CD80052421843BCBFD0401843704792F0000F6F
:108CE80081F4000106BF80F400000132013BB5E7C2
:108CF8004FEA41037FEA226C18BF7FEA236C21D038
:108D080092EA030F04D092F0000F08BF084670479C
:108D180090EA010F1CBF0020704712F07F4F04D16A
:108D2800400028BF40F00040704712F100723CBF7D
:108D380000F50000704700F0004343F0FE4040F4A7
:108D4800000070477FEA226216BF08467FEA236365
:108D58000146420206BF5FEA412390EA010F40F450
:108D6800800070474FF0000304E000BF10F000439C
:108D780048BF40425FEA000C08BF704743F0964383
:108D880001464FF000001CE050EA010208BF70479E
:108D98004FF000030AE000BF50EA010208BF704725
:108DA80011F0004302D5404261EB41015FEA010C3A
:108DB80002BF84460146002043F0B64308BFA3F132
:108DC8008053A3F50003BCFA8CF2083AA3EBC25314
:108DD80010DB01FA02FC634400FA02FCC2F1200233
:108DE800BCF1004F20FA02F243EB020008BF20F06A
:108DF8000100704702F1200201FA02FCC2F12002D0
:108E080050EA4C0021FA02F243EB020008BF20EAC4
:108E1800DC7070474FF0FF0C1CEAD0521EBF1CEAF2
:108E2800D15392EA0C0F93EA0C0F6FD01A4480EAE0
:108E3800010C400218BF5FEA41211ED04FF00063C9
:108E480043EA501043EA5111A0FB01310CF00040F5
:108E5800B1F5000F3EBF490041EAD3715B0040EA1B
:108E6800010062F17F02FD2A1DD8B3F1004F40EBEB
:108E7800C25008BF20F00100704790F0000F0CF0BE
:108E8800004C08BF49024CEA502040EA51207F3A82
:108E9800C2BFD2F1FF0340EAC250704740F400005D
:108EA8004FF00003013A5DDC12F1190FDCBF00F04E
:108EB80000407047C2F10002410021FA02F1C2F1FC
:108EC800200200FA02FC5FEA310040F1000053EA98
:108ED8004C0308BF20EADC70704792F0000F00F0E6
:108EE800004C02BF400010F4000F013AF9D040EAEC
:108EF8000C0093F0000F01F0004C02BF490011F480
:108F0800000F013BF9D041EA0C018FE70CEAD1537D
:108F180092EA0C0F18BF93EA0C0F0AD030F0004CFD
:108F280018BF31F0004CD8D180EA010000F00040B1
:108F3800704790F0000F17BF90F0004F084691F06F
:108F4800000F91F0004F14D092EA0C0F01D14202A9
:108F58000FD193EA0C0F03D14B0218BF084608D172
:108F680080EA010000F0004040F0FE4040F40000BC
:108F7800704740F0FE4040F4400070474FF0FF0C4F
:108F88001CEAD0521EBF1CEAD15392EA0C0F93EA96
:108F98000C0F69D0A2EB030280EA010C49024FEAE8
:108FA800402037D04FF0805343EA111143EA1013A1
:108FB8000CF000408B4238BF5B0042F17D024FF459
:108FC800000C8B4224BF5B1A40EA0C00B3EB510F34
:108FD80024BFA3EB510340EA5C00B3EB910F24BF1D
:108FE800A3EB910340EA9C00B3EBD10F24BFA3EBA2
:108FF800D10340EADC001B0118BF5FEA1C1CE0D16A
:10900800FD2A3FF650AF8B4240EBC25008BF20F01C
:10901800010070470CF0004C4CEA50207F32C2BF70
:10902800D2F1FF0340EAC250704740F400004FF00D
:109038000003013A37E792F0000F00F0004C02BF3E
:10904800400010F4000F013AF9D040EA0C0093F008
:10905800000F01F0004C02BF490011F4000F013B62
:10906800F9D041EA0C0195E70CEAD15392EA0C0FCA
:1090780008D142027FF47DAF93EA0C0F7FF470AF02
:10908800084676E793EA0C0F04D14B023FF44CAF45
:1090980008466EE730F0004C18BF31F0004CCAD1DA
:1090A80030F000427FF45CAF31F000437FF43CAF16
:1090B8005FE700BF4FF0FF3C06E000BF4FF0010C38
:1090C80002E000BF4FF0010C4DF804CD4FEA40021A
:1090D8004FEA41037FEA226C18BF7FEA236C11D064
:1090E80001B052EA530C18BF90EA010F58BFB2EB17
:1090F800030088BFC81738BF6FEAE17018BF40F097
:10910800010070477FEA226C02D15FEA402C05D14A
:109118007FEA236CE4D15FEA412CE1D05DF8040BCF
:10912800704700BF844608466146FFE70FB5FFF762
:10913800C9FF002848BF10F1000F0FBD4DF808ED1A
:10914800FFF7F4FF0CBF012000205DF808FB00BF0B
:109158004DF808EDFFF7EAFF34BF012000205DF865
:1091680008FB00BF4DF808EDFFF7E0FF94BF0120B2
:1091780000205DF808FB00BF4DF808EDFFF7D2FFAF
:1091880094BF012000205DF808FB00BF4DF808EDF2
:10919800FFF7C8FF34BF012000205DF808FB00BFBF
:1091A8004FEA4002B2F1FE4F0FD34FF09E03B3EBEC
:1091B80012620DD94FEA002343F0004310F0004F2C
:1091C80023FA02F018BF404270474FF00000704782
:1091D80012F1610F01D1420205D110F0004008BF21
:1091E8006FF0004070474FF00000704753B94AB91C
:1091F800002908BF00281CBF4FF0FF314FF0FF3097
:1092080000F08CB9ADF1080C6DE904CE00F006F859
:10921800DDF804E0DDE9022304B070472DE9F047EA
:10922800089D8E4604468846002B4AD18A42174636
:1092380062D9B2FA82F64EB1C6F1200301FA06F8F5
:1092480020FA03F3B74043EA0808B4404FEA174E40
:10925800B8FBFEF11FFA87FC0EFB118801FB0CF22C
:10926800230C43EA08439A4209D9FB1801F1FF305D
:1092780080F0EB809A4240F2E88002393B449A1A27
:10928800B2FBFEF00EFB102200FB0CFCA3B243EA7B
:1092980002439C4509D9FB1800F1FF3280F0D780C2
:1092A8009C4540F2D4803B44023840EA014000210A
:1092B800A3EB0C031DB10022F340C5E90032BDE861
:1092C800F0878B4205D90DB1C5E900010021084698
:1092D800F5E7B3FA83F1002946D1734502D38242F8
:1092E80000F20881841A6EEB030201209046002DDB
:1092F800E5D0C5E90048E2E7002A00F09180B2FA1B
:1093080082F6002E40F0A5808A1A0121030C4FEA4C
:10931800174E80B2BCB2B2FBFEFC0EFB1C2243EA25
:10932800024304FB0CF29A4207D9FB180CF1FF38F0
:1093380002D29A4200F2E380C4469B1AB3FBFEF2C3
:109348000EFB123302FB04F440EA03439C4207D9A4
:10935800FB1802F1FF3002D29C4200F2CD80024697
:109368001B1B42EA0C40A5E7C1F120068B4022FAFC
:1093780006F71F432EFA06FA4FEA1749BAFBF9F81F
:109388000EFA01FE20FA06F309FB18AA1FFA87FC59
:1093980043EA0E0300FA01FE08FB0CF01C0C44EA39
:1093A8000A44A04202FA01F20AD93C1908F1FF3A2C
:1093B80080F09E80A04240F29B80A8F102083C44C5
:1093C800241A98B2B4FBF9F309FB134403FB0CFC11
:1093D80040EA0444A44509D93C1903F1FF3080F060
:1093E8008580A44540F28280023B3C4443EA084021
:1093F800A4EB0C04A0FB028C64454346E14664D30D
:1094080061D05DB1BEEB030264EB090404FA06F611
:1094180022FA01F31E43CC40C5E9006400214EE75F
:10942800B1FBF2FC010C41EA0E4180B240EA014274
:109438003B46B1FBF7F138463C46B846BE462026C7
:10944800A2EB080241EA0C4165E7014617E710461E
:109458002BE7C6F120012EFA01FCB7400EFA06FEF2
:1094680020FA01F141EA0E014FEA174EBCFBFEF863
:10947800BCB20EFB18CC08FB04F90A0C42EA0C42F9
:10948800B04091454FEA104380B23ED9BA1808F16E
:10949800FF3C01D291451FD8A2EB0902B2FBFEF9AD
:1094A80009FB04F80EFB192A8AB242EA0A4242452D
:1094B80029D2BA1809F1FF31C2D24245C0D2A9F166
:1094C80002013A44BCE7C6459BD2B8EB02036CEBF9
:1094D800070C0138E14694E7A7EB09094A44B2FBB7
:1094E800FEF9A8F1020C09FB04F8DBE703467DE767
:1094F800D04665E70846FAE63B44023A30E7ACF165
:10950800020C3B4419E749469AE7A2EB0902B2FB71
:10951800FEF9C44609FB04F8C4E700BF704700BF62
:1095280080B500AF06220549054805F00DFE034643
:10953800002B01D001F0CAFB00BF80BD74020020DF
:10954800900200200E4B02689A4218D14FF0010C8D
:109558000C4A0D4B11880D4889B21980518889B27F
:109568005980918889B29980D18889B2D980118926
:1095780089B21981528992B25A8180F800C0704725
:109588000024014074020020800200208C02002088
:1095980080B584B000AF3B1D00221A605A609A6003
:1095A8003C4B3D4A1A603B4B4FF480729A60394BF2
:1095B80000221A73374B00221A75364B4FF40022DB
:1095C800DA61344B00225A60324B06221A61314864
:1095D80005F0E2FC0346002B01D001F077FB0323E2
:1095E8007B600123BB600423FB603B1D19462948AF
:1095F80005F062FF0346002B01D001F067FB04234E
:109608007B600223BB603B1D1946224805F054FFCE
:109618000346002B01D001F059FB08237B6003238C
:10962800BB603B1D19461B4805F046FF0346002B4F
:1096380001D001F04BFB09237B600423BB603B1D79
:109648001946144805F038FF0346002B01D001F0F5
:109658003DFB10237B600523BB603B1D19460D486D
:1096680005F02AFF0346002B01D001F02FFB112340
:109678007B600623BB603B1D1946064805F01CFFAE
:109688000346002B01D001F021FB00BF1037BD4677
:1096980080BD00BF900200200024014080B58AB040
:1096A80000AF786007F1180300221A605A609A60C8
:1096B800DA607B681B68384A934268D1374B9B69EC
:1096C800364A43F400739361344B9B6903F4007387
:1096D8007B617B69314B9B69304A43F0040393619A
:1096E8002E4B9B6903F004033B613B692B4B9B6941
:1096F8002A4A43F008039361284B9B6903F0080347
:10970800FB60FB681823BB610323FB6107F11803A7
:109718001946234807F00EFE0323BB610323FB61B0
:1097280007F1180319461F4807F004FE1E4B1F4A8D
:109738001A601D4B00225A601B4B00229A601A4B7C
:109748008022DA60184B4FF480721A61164B4FF47E
:1097580080625A61144B20229A61134B4FF4805255
:10976800DA61114807F058F90346002B01D001F0DF
:10977800ADFA7B680C4A1A620B4A7B685362002276
:109788000721122007F0F5F8122007F00EF900BFA4
:109798002837BD4680BD00BF0024014000100240AC
:1097A80000080140000C0140C002002008000240EF
:1097B80080B582B000AF03460A46FB711346BB7101
:1097C800FB79072B50D801A252F823F0F59700082F
:1097D800059800081598000825980008359800088D
:1097E800459800085398000863980008BB791A4602
:1097F8004FF48071214807F038FF36E0BB791A46EC
:109808004FF400711D4807F030FF2EE0BB791A466F
:109818004FF48061194807F028FF26E0BB791A4603
:109828004FF40061154807F020FF1EE0BB791A4687
:109838004FF48051114807F018FF16E0BB791A461B
:1098480008210F4807F011FF0FE0BB791A464FF4C3
:1098580000410C4807F009FF07E0BB791A460821C8
:10986800094807F002FF00E000BFFB790749BA7911
:10987800CA5400BF0837BD4680BD00BF001801406C
:1098880000100140000801400014014004030020BA
:1098980080B483B000AF0346FB71FB79034AD35C05
:1098A80018460C37BD4680BC704700BF0403002033
:1098B80080B582B000AF0346FB71FB79062B3BD81D
:1098C80001A252F823F000BFED980008F9980008AB
:1098D80005990008119900081D99000829990008A0
:1098E800359900080221174807F0A8FE034624E02E
:1098F8000421144807F0A2FE03461EE08021124806
:1099080007F09CFE034618E08021104807F096FEF9
:10991800034612E010210E4807F090FE03460CE0C3
:1099280008210B4807F08AFE034606E00221064894
:1099380007F084FE034600E0002318460837BD46BA
:1099480080BD00BF0008014000180140001401401C
:10995800000C014080B483B000AF02237B600F4B42
:109968009B690E4A43F0100393610C4B9B6903F00B
:1099780010033B603B680A4B5B6823F470227B68EA
:109988001B04074913434B60054B4FF080521A6183
:1099980000BF0C37BD4680BC704700BF00100240B6
:1099A8000010014080B500AFFFF7D4FF00224FF44C
:1099B8008051184807F059FE174805F077FFFFF760
:1099C800AFFD00210020FFF7F3FE00210120FFF783
:1099D800EFFE00210220FFF7EBFE00210320FFF736
:1099E800E7FE00210420FFF7E3FE00210520FFF732
:1099F800DFFE00210620FFF7DBFE00210720FFF72E
:109A0800D7FE064804F050FB054804F04DFB00BFA4
:109A180080BD00BF00100140900200200C03002010
:109A28003403002090B587B000AF78600C4B7B61A1
:109A38000C4B3B6179697868FFF7E2F803461C46EE
:109A480039697869FFF7E6F9034619462046FFF7B2
:109A580095FA0346FB60FB6818461C37BD4690BD67
:109A680000007A443211803BB0B586B000AFF86090
:109A7800B9607A603B60F868FEF72CFD1CA3D3E957
:109A88000023FEF7BBFE02460B4614461D46B86887
:109A9800FEF732FD02460B4620462946FEF784FDB6
:109AA80002460B4610461946FFF756F803467B61F7
:109AB80079687869FFF760FB0346002B01D00E4BED
:109AC80010E079697868FFF79BF8034619467869CA
:109AD800FFF754FA034619463868FFF79BF903461F
:109AE8003B613B6918461837BD46B0BDAFF30080EF
:109AF8000000000000FEAF40000080BF80B588B0C5
:109B080000AF0346FB710023FB61FB79002B03D0F8
:109B18001C4BDB889BB202E01A4B9B889BB2FB6113
:109B2800FB79002B01D0012200E0002213469B00A4
:109B38001344DB00144A1344FA691146184604F02A
:109B4800D8FAB861BB69B3F57A6F01D9142315E067
:109B58000E4B7B610E4B3B610E4BFB60FB683A6919
:109B68007969B869FFF780FF03461846FFF75AFF7F
:109B7800B860B868FFF714FB03461BB218462037D5
:109B8800BD4680BD800200200C03002033335340C3
:109B98000000A04000007A4480B500AF174B184A77
:109BA8001A60164B08225A60144B00229A60134B15
:109BB8000022DA60114B4FF460221A610F4B4FF408
:109BC80080125A610D4B00221A760C4B01225A76EC
:109BD8000A4B01229A76094B0122DA76074B0022BA
:109BE8001A77064B01225A77044805F016FF0346F8
:109BF800002B01D001F06AF800BF80BD5C03002093
:109C08000064004080B500AF174B184A1A60164B25
:109C180010225A60144B00229A60134B0022DA601B
:109C2800114B4FF460221A610F4B4FF480125A61A6
:109C38000D4B00221A760C4B01225A760A4B012250
:109C48009A76094B0122DA76074B00221A77064BDF
:109C580001225A77044805F0E0FE0346002B01D0A4
:109C680001F034F800BF80BD840300200068004084
:109C780080B58EB000AF786007F1200300221A602B
:109C88005A609A60DA607B681B68614A934253D1D4
:109C9800604B1B6801335F4A13605E4B1B68012BE6
:109CA8000BD15D4BDB695C4A43F00073D3615A4BBF
:109CB800DB6903F00073FB61FB69574B9B69564AEC
:109CC80043F020039361544B9B6903F02003BB616D
:109CD800BB6901233B6200237B620023BB6207F15F
:109CE800200319464D4807F025FB02233B62022357
:109CF8007B620323FB6207F120031946474807F0FC
:109D080019FB474B5B683B633B6B23F4C0433B63E6
:109D18003B6B43F0E0633B633B6B43F4C0433B6303
:109D28003F4A3B6B536000220321142006F021FEBA
:109D3800142006F03AFE67E07B681B68394A9342B4
:109D480062D1354BDB69344A43F08063D361324BCF
:109D5800DB6903F080637B617B692E4B1B680133F1
:109D68002C4A13602B4B1B68012B0BD12A4BDB6948
:109D7800294A43F00073D361274BDB6903F0007372
:109D88003B613B69244B9B69234A43F00803936179
:109D9800214B9B6903F00803FB60FB6820233B62AF
:109DA80000237B620023BB6207F1200319461E488B
:109DB80007F0C0FA40233B6202237B620323FB6265
:109DC80007F120031946184807F0B4FA144B5B68EA
:109DD8007B637B6B43F0E0637B637B6B43F48003C3
:109DE8007B630F4A7B6B5360002200213F2006F003
:109DF800C0FD3F2006F0D9FD00220321412006F0D6
:109E0800B8FD412006F0D1FD00BF3837BD4680BD02
:109E180000640040AC030020001002400014014020
:109E28000000014000680040000C014080B400AF11
:109E3800084B00221A70074B00225A70054B00226B
:109E480062F06902DA7300221A7400BFBD4680BC52
:109E5800704700BFB003002080B500AF1F4B5A7891
:109E68001F4B1B789A4206D01C4B5A781C4B1A7011
:109E78001A4B00221A7000F0E7FB0346002B03D0B0
:109E8800164B0B225A7716E0164B1B7B002B03D080
:109E9800124B07225A770EE0124B5B7B002B03D044
:109EA8000E4B0A225A7706E00C4B9B7F002B02D1FF
:109EB8000A4B00225A77094B5B7F0021184600F0B5
:109EC80047FD0346002B06D0044B5B7F1A46064924
:109ED800052000F045FB00BF80BD00BFB003002097
:109EE800D00300201C090020087B010880B582B03F
:109EF80000AF0346FB71414B1B78FA799A4203D1B4
:109F08003F4AFB79537075E03C4AFB7913703B4B31
:109F18001B78002B03D13B49072000F021FB374B6E
:109F28001B78012B03D13849072000F019FB334B6C
:109F38001B78022B03D13549072000F011FB2F4B6A
:109F48001B78032B03D13249072000F009FB2B4B68
:109F58001B78042B03D12F49072000F001FB274B66
:109F68001B78052B03D12C49072000F0F9FA234B65
:109F78001B78062B03D12949072000F0F1FA1F4B63
:109F88001B78072B03D12649072000F0E9FA1B4B61
:109F98001B78082B03D12349072000F0E1FA174B5F
:109FA8001B78092B03D12049072000F0D9FA134B5D
:109FB8001B780A2B03D11D49072000F0D1FA0F4B5B
:109FC8001B780B2B03D11A49072000F0C9FA0B4B59
:109FD8001B780C2B03D11749072000F0C1FA074B57
:109FE8001B780D2B03D11449072000F0B9FA044A55
:109FF800FB7953700837BD4680BD00BFCF030020F2
:10A00800B00300201C7B0108307B0108487B010855
:10A01800607B0108787B0108947B0108B47B010808
:10A02800D47B0108F47B01080C7C0108247C01081E
:10A038003C7C0108587C0108707C010880B487B01A
:10A0480000AF134B5B889BB27B61114B5B899BB262
:10A058003B6140F2BA43FB60FB687A6903FB02F29A
:10A068003B69B2FBF3F3BB60BB68A3F2BB6341F689
:10A07800186202FB03F3074A82FB03129211DB17F3
:10A08800D31A7B607B6818461C37BD4680BC704776
:10A0980080020020D34D621080B500AF0E4B1B68C4
:10A0A8009F229A620C4B1B6840F2C112DA620A4B7B
:10A0B8001B684FF4E1729A63074B1B6840F2C712A2
:10A0C8005A630421044808F007FE0021024808F0FA
:10A0D80001FD00BF80BD00BFF811002080B485B02D
:10A0E80000AF0346FB71FB794FF4E17202FB03F307
:10A0F8000B4A82FB03125211DB17D31AFB60094A81
:10A10800FB791370084B1B68FA689A63064B1B6847
:10A1180001225A6300BF1437BD4680BC704700BF98
:10A128001F85EB51D8030020F811002080B400AF40
:10A13800024B1B781846BD4680BC7047D8030020E8
:10A1480080B500AFFFF77AFF0346034A1360024B5E
:10A158001B68184680BD00BFD403002080B582B0BC
:10A1680000AFFFF7EDFF7860214B1B78062B02D07C
:10A178001F4B1B7838E07B6842F6F722934201DDDB
:10A18800002331E07B68B3F5FA5F06DB7B6842F2B7
:10A198001072934201DC012326E07B6841F287328A
:10A1A800934206DD7B6841F65832934201DC022374
:10A1B8001AE07B68B3F5FA6F05DB7B68B3F57A6F55
:10A1C80001DC032310E07B6813F57A7F05DB7B68ED
:10A1D800B3F5FA6F01DC042306E07B68054A934275
:10A1E80001DA052300E0062318460837BD4680BD7E
:10A1F8000400002009D5FFFF80B400AF024B1B7894
:10A208001846BD4680BC70470500002080B582B066
:10A2180000AFFFF7A3FF0346FB71FB79062B06D1BE
:10A22800134B06221A70134B00221A701DE0104BB4
:10A238001B78FA799A4206D00D4AFB7913700D4BB8
:10A2480001221A7011E00B4B1B78632B05D8094BC0
:10A258001B780133DAB2074B1A70064B1B78632B55
:10A2680003D9034B1A78044B1A700837BD4680BDD2
:10A2780006000020D90300200500002080B582B028
:10A2880000AF04F05BFE0246224B1B68D31A002B7A
:10A298003CDD04F053FE03461E4A1360FFF7B6FF89
:10A2A800FFF7AAFF0346FB711B4B1B78BB711B4BC7
:10A2B8001B78002B09D11A4AFB791370194ABB790C
:10A2C8001370164B01221A7021E0154B1B78FA798E
:10A2D8009A420AD0124B1B781A46FB79124907207A
:10A2E80000F03EF90E4AFB7913700E4B1B78BA79D1
:10A2F8009A420CD00B4B1B781A46BB790B490720A6
:10A3080000F02EF9074ABB79137000E000BF083748
:10A31800BD4680BDDC030020D8030020E0030020F8
:10A3280007000020E1030020887C0108A47C0108C4
:10A3380080B500AF064B074A1A60054806F04FFB88
:10A348000346002B01D000F0C1FC00BF80BD00BF58
:10A35800E40300200030024080B485B000AF78608C
:10A368007B681B68094A93420BD1094B5B69084A11
:10A3780043F040035361064B5B6903F04003FB6005
:10A38800FB6800BF1437BD4680BC704700300240F0
:10A398000010024080B584B000AFF860B9607A6000
:10A3A8007B689BB21946B86800F006F87B681846C7
:10A3B8001037BD4680BD000080B485B000AF78601E
:10A3C8000B467B8072B600BF0023FB8145E0284B1B
:10A3D800B3F804349BB2B3F5806F18D3244BB3F8A9
:10A3E80002349BB201335A42C3F30903C2F3090290
:10A3F80058BF53429AB21E4BA3F802241C4BB3F821
:10A4080004349BB2013B9AB2194BA3F80424FB898C
:10A418007A681344164AB2F8002492B21978144B99
:10A428009954134BB3F800349BB201335A42C3F327
:10A438000903C2F3090258BF53429AB20C4BA3F85E
:10A4480000240B4BB3F804349BB201339AB2084B87
:10A45800A3F80424FB890133FB81FA897B889A429B
:10A46800B5D362B600BF00BF1437BD4680BC704785
:10A47800EC03002080B483B000AF72B600BF064B77
:10A48800B3F80434FB8062B600BFFB8818460C376B
:10A49800BD4680BC704700BFEC03002080B582B089
:10A4A80000AF72B600BF2D4BB3F804349BB2002B3B
:10A4B80002D162B600BF4EE0284BB3F80434FB80EB
:10A4C800FB88802B01D98023FB80244BB3F802340E
:10A4D8009BB2C3F58063BB80FA88BB889A4201D9D6
:10A4E800BB88FB801D4BB3F804349BB2FA889A42B0
:10A4F8000CD11A4BB3F802349BB21A46174B1344CB
:10A50800F9885022184603F031FA0BE0134BB3F8E0
:10A5180002349BB21A46114B1344F988512218464B
:10A5280003F024FA0D4BB3F802349AB2FB881344B3
:10A538009BB2C3F309039AB2084BA3F80224074B52
:10A54800B3F804349AB2FB88D31A9AB2034BA3F82F
:10A55800042462B600BF0837BD4680BDEC03002066
:10A568000EB480B585B000AF0346FB71154AFB7980
:10A57800137007F12003BB60BB68FA697E2112489B
:10A588000BF0CCF9F860FB68002B01DAFB6812E0ED
:10A59800FB687D2B01DD7E23FB60FB680133094AE4
:10A5A8000021D154FB689BB202339BB2194605487F
:10A5B800FFF702FFFB6818461437BD46BDE8804028
:10A5C80003B07047F4070020F507002080B582B07B
:10A5D80000AF1C4B5B691B4A43F001035361194BE5
:10A5E8005B6903F001037B607B68002201210B207B
:10A5F80006F0BFF90B2006F0D8F9002204210C2040
:10A6080006F0B7F90C2006F0D0F9002201210D2040
:10A6180006F0AFF90D2006F0C8F90022012110203C
:10A6280006F0A7F9102006F0C0F900220421112035
:10A6380006F09FF9112006F0B8F900BF0837BD46AB
:10A6480080BD00BF0010024080B400AF024B1B78F1
:10A658001846BD4680BC70477408002080B500AF1E
:10A66800064B1B78002B07D1044B01221A700449B2
:10A678000420FFF775FF00E000BF80BD74080020CC
:10A68800C07C010880B58AB000AF07F1140300222E
:10A698001A605A609A60DA60944B9B69934A43F057
:10A6A80010039361914B9B6903F010033B613B6975
:10A6B8008E4B9B698D4A43F0040393618B4B9B69D6
:10A6C80003F00403FB60FB68884B9B69874A43F0EF
:10A6D80008039361854B9B6903F00803BB60BB6863
:10A6E800824B9B69814A43F0400393617F4B9B698E
:10A6F80003F040037B607B687C4B9B697B4A43F09B
:10A7080020039361794B9B6903F020033B603B680E
:10A7180000224FF40F71764806F0A7FF002248F296
:10A728006001744806F0A1FF00224FF4F851724806
:10A7380006F09BFF00224FF44861704806F095FF31
:10A74800002218216E4806F090FF4FF401737B61D8
:10A758000123BB610023FB6103233B6207F1140360
:10A768001946634806F0E6FD38237B610123BB6187
:10A778000023FB6102233B6207F1140319465C487E
:10A7880006F0D8FD02237B610023BB610023FB6137
:10A7980007F114031946574806F0CCFD04237B61E2
:10A7A8000023BB610223FB6107F1140319465148DA
:10A7B80006F0C0FD60237B610123BB610023FB61C0
:10A7C80003233B6207F1140319464A4806F0B2FD19
:10A7D80044F282037B610023BB610023FB6107F124
:10A7E80014031946444806F0A5FD4FF4F8537B615D
:10A7F8000123BB610023FB6102233B6207F11403C1
:10A8080019463D4806F096FD4FF440637B610123ED
:10A81800BB610023FB6103233B6207F11403194664
:10A82800364806F087FD4FF400437B610123BB6186
:10A838000023FB6102233B6207F1140319462D48EC
:10A8480006F078FD18237B610123BB610023FB61BF
:10A8580002233B6207F114031946294806F06AFDF2
:10A8680080237B610023BB610023FB6107F1140394
:10A878001946234806F05EFD18237B610023BB615F
:10A888000023FB6107F1140319461C4806F052FD2A
:10A8980080237B610123BB610023FB6102233B62B0
:10A8A80007F114031946154806F044FD4FF44073A8
:10A8B8007B611223BB6103233B6207F11403194632
:10A8C8000E4806F037FD0F4B5B687B627B6A43F0EE
:10A8D800E0637B627B6A43F002037B62094A7B6A1E
:10A8E800536000BF2837BD4680BD00BF001002403E
:10A8F800001001400008014000180140000C014010
:10A90800001401400000014080B400AFBFF34F8F36
:10A9180000BF064BDB6803F4E0620449044B1343B1
:10A92800CB60BFF34F8F00BF00BFFDE700ED00E035
:10A938000400FA0580B400AF034B044A9A6000BFD4
:10A94800BD4680BC704700BF00ED00E000800008F5
:10A9580080B485B000AF03460A46FB711346BB714D
:10A96800BB791F2B01D900230EE00023FB73BB79B1
:10A97800084AD35CFA799A4201D00123FB73BB7968
:10A988000449FA79CA54FB7B18461437BD4680BC83
:10A99800704700BF7808002080B584B000AF7860A9
:10A9A80004F0CCFAB8607B68FB60FB68B3F1FF3F4A
:10A9B80010D00F4B1B781A46FB681344FB6009E064
:10A9C80002F03CF800F016F8FFF758FC01F0F8FD2B
:10A9D80002F072FE04F0B2FA0246BB68D31AFA68B3
:10A9E8009A42EDD800BF00BF1037BD4680BD00BFFA
:10A9F8008C00002080B582B000AF04F09FFA786028
:10AA08002A4B1B687A68D31A092B49D9274A7B68CD
:10AA180013600320FEF74CFF0346002B0CBF0123F5
:10AA28000023DBB2FB70FB78002B02D1204B002205
:10AA38001A701F4B1B78002B34D1FB78002B2BD0BE
:10AA48001C4B1B68002B02D11B4B01221A70194B9F
:10AA58001B680A33174A1360164B1B6841F2883289
:10AA6800934202D1144B03221A70124B1B6849F609
:10AA78004042934217D912220021002002F076FFAB
:10AA880000BF0E4B93F84130DBB2212BF9D00A20DE
:10AA980004F05EFAFFF738FF064B00221A6002E066
:10AAA80000BF00E000BF0837BD4680BD9808002001
:10AAB800080000209C080020B00300201813002084
:10AAC80080B500AF0B4805F0C7F9FFF765F80948EE
:10AAD80005F07EF90346002B01D000F0F7F80221BB
:10AAE800044805F026FC0346002B01D000F0EEF8E0
:10AAF80000BF80BD5C03002080B582B002AFFFF7C5
:10AB080019FF04F0C3F906F0D5FD00F06FF8FFF760
:10AB1800B9FDFFF75BFDFEF73BFDFFF73DF8FFF7DB
:10AB280071F801F0F1FD03F0B9FD03F037FFFFF70D
:10AB3800FFFB03F0DFFE03F007FF03F059FF03F00C
:10AB48001FFDFEF72FFF01F017FD4FF4967004F07C
:10AB5800FFF902F00BFA02F085FD1F490720FFF705
:10AB6800FFFC02F05BFD1D4B1B889BB21A461C497B
:10AB78000720FFF7F5FC194B9B781A46194907205F
:10AB8800FFF7EEFC154B9B889BB21A46134BDB88EC
:10AB98009BB21946114B1B899BB200930B46124975
:10ABA8000720FFF7DDFCFFF78BFF00F091FCFFF7B4
:10ABB8003DF900F0A1FD00F06BFE0A20FFF7ECFE66
:10ABC80000F08AF8FFF748F901F096F90A20FFF734
:10ABD800E3FE00BFEDE700BF3C7D0108E011002067
:10ABE800507D0108647D0108787D010880B59CB01E
:10ABF80000AF07F138033822002118460AF09CFEFE
:10AC080007F1240300221A605A609A60DA601A6118
:10AC18003B1D2022002118460AF08EFE0523BB6347
:10AC28004FF480333B6404237B640123BB6401231A
:10AC3800FB644FF48033FB630223BB654FF480331E
:10AC4800FB654FF4E0133B6602237B664FF4C06359
:10AC5800BB664023FB6607F13803184606F0FAFD89
:10AC68000346002B01D000F031F80F237B6202234A
:10AC7800BB620023FB624FF480633B6300237B636A
:10AC880007F124030221184607F0FAF80346002BBF
:10AC980001D000F01BF803237B604FF48073BB6086
:10ACA8004FF40043FB603B1D184607F0DFFA0346EC
:10ACB800002B01D000F00AF8034B01221A6000BFF4
:10ACC8007037BD4680BD00BF7000424280B400AFFF
:10ACD80072B600BF00BFFDE72DE9B04384B000AFF6
:10ACE8002C4B00221A702C4B5B78082B03D1294B74
:10ACF80001221A7602E0274B00221A7604F01EF988
:10AD0800F860244B5B68FA68D31ABB60214AFB6879
:10AD18005360214BD3F80330BA6802FB03F31F4A90
:10AD2800A2FB03239B097B601A4BD3E902237968B2
:10AD380000200C46054612EB040843EB0509154BA9
:10AD4800C3E90289134BD3E90223154BA3FB022362
:10AD5800DB0A104A13610F4B1B7E002B08D00D4BEA
:10AD68001A690C4B5B69D31A0B4AC2F807300CE01E
:10AD7800094B0022DA7100221A7200225A7200224C
:10AD88009A72044B1B69034A536100BF1037BD46D2
:10AD9800BDE8B083A0080020B0030020D34D6210A6
:10ADA800C5B3A29180B483B000AF0346FB71FB79B1
:10ADB800002B0BD0FB79012B08D0FB790A2B05D08F
:10ADC800FB790C2B02D0FB790B2B01D1012300E07E
:10ADD8000023DBB218460C37BD4680BC7047000024
:10ADE80080B400AF114B96221A80104B00225A8073
:10ADF8000F4A0E4B1B6813600E4A0C4B1B681360FE
:10AE08000D4B00221A700D4B00221A700C4B0022B9
:10AE18001A700C4B00221A700B4B00221A600B4B55
:10AE280000221A6000BFBD4680BC7047C0080020E1
:10AE3800C4080020C8080020CC080020CD08002045
:10AE4800CE080020CF080020D0080020D408002019
:10AE580080B483B000AF03460A46FB801346BB802C
:10AE6800064AFB881380054ABB885380044B01229D
:10AE78001A7000BF0C37BD4680BC7047C40800205C
:10AE8800CC08002080B582B000AF04F057F8786095
:10AE9800254BDB7D002B0BD0234B9B7F002B07D052
:10AEA800224B1B781846FFF77DFF0346002B0CD07A
:10AEB8001F4B00221A701F4B00221A701E4B0022D3
:10AEC8001A601E4B00221A602BE0174BB3F81B3098
:10AED8009BB2142B02D9164B01221A70134B1B7804
:10AEE800082B02D1124B01221A700F4BB3F8153000
:10AEF8009BB21D2B12D9114B1B68002B03D10F4A93
:10AF08007B6813600DE00D4B1B687A68D31AB3F5A4
:10AF1800FA7F06D3064B01221A7002E0074B002283
:10AF28001A600837BD4680BDB0030020400D0020E0
:10AF3800CE080020CF080020D0080020D408002028
:10AF480080B400AF024B1B781846BD4680BC7047E2
:10AF5800CC08002080B400AF084B1B78002B01D12F
:10AF6800002307E0064BDB79063B042B01D80123BD
:10AF780000E000231846BD4680BC7047CD0800207D
:10AF88001C090020B0B588B000AF78601C4BDB7A94
:10AF98003B731B4B9B7A7B731A4BB3F813309BB2F2
:10AFA800FB81184BB3F815309BB23B82164B1B78CC
:10AFB800BB74144BDB7DFB74114BDB79052B01D182
:10AFC800012300E000233B750D4B1B7B7B750C4B6D
:10AFD8005B7BBB750D4B1B78FB750D4B1B68BB6111
:10AFE80003F0ACFF0346FB617B681D4607F10C04C8
:10AFF8000FCC0FC523682B6078682037BD46B0BDDD
:10B008001C090020B0030020CE080020CF08002033
:10B01800D0080020B0B58EB002AF2B4B1B78002BA8
:10B0280003D02A4B1B78002B01D0002348E03B4675
:10B038001846FFF7A7FF07F118043D460FCD0FC4C8
:10B048002B68236007F118031A462149214800F0AC
:10B05800ADF8034687F82F3097F82F30012B19D118
:10B068001D4A1B4B1B681360184B01221A70164BA4
:10B0780000221A70174B1B881A46174B1B88194653
:10B08800154B5B8800930B4614490720FFF768FAB5
:10B09800022315E0124B5B7A002B01D100230FE04D
:10B0A8000B4B1B880A4A52881946002000F074FA94
:10B0B800084A074B1B681360034B00221A700123D0
:10B0C80018463037BD46B0BDCC080020CD0800205A
:10B0D800C4080020C0080020C8080020D87C010847
:10B0E8001C09002080B483B000AF78607B68002B17
:10B0F80003D07B68034A1068186000BF0C37BD4650
:10B1080080BC7047C808002080B500AF0E4A0F4BBE
:10B118001B6813600E4B00221A700E4B1B7801330C
:10B12800DAB20C4B1A7003F009FF03460A4A13609F
:10B138000A4BB3F813309BB21A4609490720FFF7A8
:10B148000FFA00BF80BD00BFC0080020C80800205B
:10B15800CD080020CF080020D0080020B003002030
:10B16800FC7C010880B500AF0A4B00221A700A4A1D
:10B178000A4B1B6813600A4B01221A70094BB3F87B
:10B1880013309BB21A4608490520FFF7E9F900BFBA
:10B1980080BD00BFCD080020C4080020C8080020DA
:10B1A800CC080020B00300201C7D010880B487B0C3
:10B1B80000AFF860B9607A60FB68002B05D0BB6807
:10B1C800002B02D07B68002B01D1002369E0BB680B
:10B1D8001A88FB681B889A4201D3002361E0FB6848
:10B1E8001A88BB681B88D31AFB82FB8A312B01D8CB
:10B1F800002356E0FB685B88142B03D8BB685B8888
:10B20800142B01D900234CE07B689B881D2B01D9A6
:10B21800002346E07B685A88BB681B880F339BB2C3
:10B228009A4201D800233CE07B689B79002B01D02F
:10B23800002336E07B68DB79002B01D1002330E066
:10B248007B681B7A002B01D100232AE07B681B78DE
:10B25800002B01D1002324E07B685B78002B01D10F
:10B2680000231EE07B685B7A002B03D17B689B7A06
:10B27800002B01D0002314E07B68DB7A032B01D973
:10B2880000230EE07B68DB68002B09D07B681A6915
:10B298007B68DB68D31AB3F5FA6F01D2002300E0AC
:10B2A800012318461C37BD4680BC704780B582B064
:10B2B80000AF0346FB71064AFB79D37103F03EFEEB
:10B2C8000346034A136100BF0837BD4680BD00BF6F
:10B2D8001C09002080B500AF03F030FE0246024B87
:10B2E8001B69D31A184680BD1C09002080B582B09E
:10B2F80000AF3B1D1846FFF7F5FEBB88FA881946D4
:10B30800002000F049F90121002000F015F900BFE4
:10B318000837BD4680BD00BF80B500AFFFF722FFEC
:10B32800054B9B7A002B01D1FFF7E0FF0520FFF7C3
:10B33800BDFF00BF80BD00BF1C09002038B5424CCE
:10B34800424D23462A46012104F0D2FE10B96D6809
:10B35800EBB203B138BD03F0F1FDC5F305453C4B35
:10B36800022D186013D0042D17D194E80300394B2F
:10B37800394A83E80300187A1C79D9799B791462D1
:10B3880082F8240082F8251082F8263038BD334B25
:10B3980094E8030083E8030038BD062D11D194E832
:10B3A80003002F4B83E80300188859889A8840BA0D
:10B3B80049BA52BA80B289B292B2C3E902011A619B
:10B3C80038BD082D3AD0092DC4D194E80300214B8B
:10B3D800244D214C93F804C0234A85E8030000BAA1
:10B3E80084F806C0A2FB00C209BAC5E90201C2F38B
:10B3F8008F1013284FF0010E94BF002501251B4B19
:10B4080084F808E0A3FB01C3E1795B09714560801A
:10B41800A3804FEA9212A5729CD999B292B201FB0D
:10B4280002F2134C1349A4FB0242A1F815300D7621
:10B43800D308A1F81300C1F8033038BD0E4B94E8C7
:10B44800030083E8030038BD640900204809002090
:10B4580044090020E40800201C090020D808002026
:10B46800F00800200C090020D34D62101F85EB5115
:10B47800CDCCCCCCB00300200409002080B58AB024
:10B4880000AF0E237B610023BB610123FB61002316
:10B498003B6000237B600023BB600023FB6000232C
:10B4A8003B6101233B6201233B610E237B623B46E8
:10B4B8001946064804F0ACFB0346002B01D0FFF701
:10B4C80005FC00BF2837BD4680BD00BF84030020AF
:10B4D80080B500AF164804F0BFFCFEF793FBFFF7FA
:10B4E800CDFF134804F074FC1021114804F021FF2B
:10B4F800282200210F480AF01FFA0E4B0022DA71A9
:10B5080003F01CFD03460B4A13610A4B49F64042FF
:10B518005A61084B00221A76064B0022DA61002194
:10B52800002000F009F8FFF75BFC00BF80BD00BFFA
:10B53800840300201C09002080B584B000AF0346B6
:10B548000A46FB711346BB7107F108030822002164
:10B5580018460AF0F1F9FB79002B15D10D4B1B7A2F
:10B56800002B13D0BB79002B0CBF01230023DBB2C7
:10B578003B7207F10803F9791A22F02000F066F807
:10B588001420FFF709FA02E000BF00E000BF1037FF
:10B59800BD4680BD1C09002080B586B000AF0346BB
:10B5A800FB710B46BB8013467B8007F1080308221A
:10B5B800002118460AF0C0F9FB79002B40D1BB885E
:10B5C800952B01D89623BB801F4B1B7E002B06D1E1
:10B5D800BB88B3F5FA7F02D340F2F313BB807B88B4
:10B5E800642202FB03F37B61BB884FF47A7202FB8F
:10B5F80003F33B617B691B0EDBB23B737B691B0C5E
:10B60800DBB27B737B691B0ADBB2BB737B69DBB282
:10B61800FB733B691B0EDBB23B723B691B0CDBB255
:10B628007B723B691B0ADBB2BB723B69DBB2FB7204
:10B6380007F10803F9791C22F02000F007F800E070
:10B6480000BF1837BD4680BD1C09002080B58CB0EE
:10B6580000AF3B600346FB710B46BB7113467B7121
:10B66800FB7987F82830BB7987F829307B7903F094
:10B678003F03DAB297F82A3062F3050387F82A30D5
:10B688007B8D0A2262F389137B850A2387F82F3082
:10B69800BB6A7B610023FB610423BB6108233B6217
:10B6A8001EE0144804F0F0FC0346002B0ED007F10E
:10B6B8000C0307F110013A680E4804F016FC034623
:10B6C80087F82E3097F82E30002B0ED00120FFF788
:10B6D80063F997F92F30DBB2013BDBB287F82F30E3
:10B6E80097F92F30002BDCDC00E000BF3037BD4677
:10B6F80080BD00BF8403002080B584B000AF3B1D2F
:10B7080000221A605A603B1D04220021F020FFF736
:10B718009DFF1420FFF740F93B1D06220021F02071
:10B72800FFF794FF1420FFF737F93B1D092200218A
:10B73800F020FFF78BFF1420FFF72EF9504BB3F8DA
:10B748001B309BB24F4AA2FB0323DB089BB21A466D
:10B758004B4BB3F813309BB202FB03F31A464A4B28
:10B768005B699A4211D9484B5A6913469B001344A6
:10B778005B001A46424BB3F813309BB2B2FBF3F3AB
:10B788009AB23F4BA3F8112006E03D4BB3F81B30AB
:10B798009AB23B4BA3F81120394BB3F811309BB246
:10B7A80040F23252934208D9354B002242F032021D
:10B7B8005A74002242F005029A74314BB3F81130E2
:10B7C8009BB21A462E4BB3F80F309BB202FB03F321
:10B7D8002E4A82FB03129210DB17D31A1A46284B03
:10B7E800C3F80B20FFF7ACFB0346002B04D1FFF78F
:10B7F800B1FB0346002B01D0012300E00023FB73BB
:10B80800214B5B7A002B11D0FB7B002B0ED11C4BFC
:10B81800B3F80F309BB21A4AB2F8112092B2194607
:10B828000020FFF7B9FE1420FFF7B6F8164B5B7A35
:10B83800002B21D0124BB3F813309BB2B3F5F57F30
:10B8480017D9114BDB69002B05D103F077FB0346B1
:10B858000D4AD36110E003F071FB02460A4BDB6925
:10B86800D31A42F20F72934206D9074B01221A7675
:10B8780002E0054B0022DA6100BF1037BD4680BDEB
:10B88800B0030020CDCCCCCC1C09002067666666CE
:10B8980090B585B000AFFFF7F5FAFFF751FB034607
:10B8A800002B09D0FFF7B6FB0346FB73FB7B022B8B
:10B8B80002D10620FFF7FAFC03F040FB0246AD4B2D
:10B8C8001B68D31AB3F5FA7F20D9AB4B00221A7242
:10B8D800A94B00229A72A94B00221A71A74B002289
:10B8E8001A72A64B0022DA71A44B00229A71A44B5B
:10B8F80000229A60A24B0022DA60A14B00221A6152
:10B90800A04B0022DA609F4B00229A609A4B1B7A68
:10B91800002B03D0984B1B78002B0CD19A4B00229C
:10B92800DA7400221A75984B00225A7500229A750B
:10B93800954B00221A76944B9B7F002B0CD001214B
:10B948000420FDF735FF03F0F9FA03468F4A136028
:10B95800894B01221A7010E003F0F0FA02468B4B73
:10B968001B68D31A4EF66022934206D900210420A0
:10B97800FDF71EFF804B00221A700520FDF798FF87
:10B9880003461A467C4BDA727B4B1B7A002B07D096
:10B99800794B1B7B002B03D1774B1B78002B02D1F3
:10B9A800754B00225A72744BDB790E2B00F27F82A2
:10B9B80001A252F823F000BFFDB9000831BA00080F
:10B9C8004DBA00088BBA0008CFBA000811BB0008AE
:10B9D800A5BB0008E9BB000873BC0008C3BC00088D
:10B9E80011BD0008CBBD000869BE0008F7BD0008FE
:10B9F800A3BE0008604B00225A7000210320FDF707
:10BA0800D7FE5D4B1B7A002B00F055825A4B1B78F2
:10BA1800002B00F05082584B1B7B002B40F04B82D0
:10BA28000120FFF743FC46E2FFF754FC0346B3F559
:10BA38007A6F40F24282504B01225A720220FFF77D
:10BA480035FC3AE24C4B00221A764B4B0022DA6165
:10BA580000210320FDF7ACFE474B5B7A002B03D196
:10BA68000020FFF723FC3DE2474BDB7D002B00F075
:10BA7800268201210020FFF75FFD0320FFF716FC57
:10BA88001DE23D4B9B7A002B07D03B4B5B7A002B8A
:10BA980003D00420FFF70AFC13E2FFF71BFC034660
:10BAA80042F21072934240F20C82334B01225A73D5
:10BAB800354B0A225A770020FFF7F8FB3449042057
:10BAC800FEF74EFDFDE101210320FDF771FE2A4B33
:10BAD800DB7A002B03D00520FFF7E8FBF3E1FFF743
:10BAE800F9FB0346B3F57A7F40F2ED81224B012240
:10BAF8001A73254B07225A770B20FFF7D7FB2549E6
:10BB08000420FEF72DFDDEE11F4BDB7D002B03D06B
:10BB1800194B5B7A002B03D10B20FFF7C7FBE1E140
:10BB28000520FDF7C5FE03461C460320FDF7B0FEC1
:10BB380003469C4217D003F001FA0246164B1B68D5
:10BB4800D31AB3F57A7F40F2C0810F4B07225A7798
:10BB5800094B01221A730B20FFF7A8FB0D4904209B
:10BB6800FEF7FEFCB1E103F0E9F903460A4A136067
:10BB7800ABE100BF440900201C090020E4080020B4
:10BB8800F00800200C090020B00300206C090020F8
:10BB9800907D0108A07D010870090020A84BDB7D7D
:10BBA800002B0BD0A74B5B7A002B07D0A54B1B7B38
:10BBB800002B03D1A34B5B7B002B09D0A2490520A6
:10BBC800FEF7CEFCFFF7CEFA0B20FFF76FFB89E1FB
:10BBD80000210020FFF7B0FC0720FFF767FB81E199
:10BBE800974BDB7D002B0BD0964B5B7A002B07D055
:10BBF800944B1B7B002B03D1924B5B7B002B09D012
:10BC080091490520FEF7ACFCFFF7ACFA0B20FFF7D3
:10BC18004DFB67E18B4B9B7A002B12D107F1080390
:10BC28001846FFF75FFA864BB3F813309BB21A46F3
:10BC38003B8986490720FEF793FC0820FFF736FB6F
:10BC480045E1FFF747FB034642F21072934240F288
:10BC58003E817B4BB3F813309BB21A467C490520D2
:10BC6800FEF77EFCFFF758FB31E1754BDB7D002BBF
:10BC78000BD0744B5B7A002B07D0724B1B7B002BCD
:10BC880003D1704B5B7B002B09D06F490520FEF771
:10BC980067FCFFF767FA0B20FFF708FB22E13B1D63
:10BCA8001846FFF71FFABB88FA8819460020FFF7E5
:10BCB80073FC0920FFF7FAFA14E1614BDB7D002BD6
:10BCC8000BD0604B5B7A002B07D05E4B1B7B002BA5
:10BCD80003D15C4B5B7B002B09D05B490520FEF749
:10BCE8003FFCFFF73FFA0B20FFF7E0FAFAE00121EB
:10BCF8000020FFF721FC03F021F90346554A1360A1
:10BD08000A20FFF7D3FAEDE04D4BDB7D002B0BD07B
:10BD18004C4B5B7A002B07D04A4B1B7B002B03D183
:10BD2800484B5B7B002B09D047490520FEF718FCE0
:10BD3800FFF718FA0B20FFF7B9FAD3E03B4618468D
:10BD4800FFF7D0F93B88282B03D93B88283B9BB2C7
:10BD580000E00023BB813B4B9B7A002B0CD0384B77
:10BD6800B3F813309BB2BA899A4205D8FFF7CCF9D9
:10BD78000520FFF79BFAACE003F0E0F80246354BEC
:10BD88001B68D31AB3F5FA7F06D3FFF7AFFA03F0AF
:10BD9800D5F803462F4A1360FFF79CFA034642F290
:10BDA8001072934240F29580254BB3F813309BB242
:10BDB8001A463B8828490520FEF7D2FBFFF7ACFA64
:10BDC80087E01F4B00225A7400229A741C4BB3F868
:10BDD80015309BB21D2B06D9FFF77CFA034641F2BA
:10BDE8008832934277D90D20FFF760FA73E000217B
:10BDF8000320FDF7DDFC134BDB7A002B07D1002174
:10BE08000020FFF799FB0C20FFF750FA65E0FFF7D9
:10BE180061FA0346B3F57A7F5FD90A4B01221A7398
:10BE2800074B07225A7700210020FFF785FB0C20DB
:10BE3800FFF73CFA09490420FEF792FB4DE000BFEA
:10BE4800B00300201C090020C07D0108E07D010826
:10BE5800087E0108740900202C7E0108A07D0108D5
:10BE6800224B9B7A002B03D10E20FFF71FFA36E0F6
:10BE7800FFF730FA034642F2107293422FD91B4B58
:10BE880001225A731A4B0A225A770020FFF70EFA3A
:10BE980018490420FEF764FB21E0FFF71BFA03466C
:10BEA800B3F57A6F1DD90220FFF700FA19E00020D8
:10BEB800FFF7FCF916E000BF14E000BF12E000BF76
:10BEC80010E000BF0EE000BF0CE000BF0AE000BFBA
:10BED80008E000BF06E000BF04E000BF02E000BFCA
:10BEE80000E000BF00BF1437BD4690BD1C0900200C
:10BEF800B00300205C7E010880B500AF3C4B5B7F3F
:10BF0800002B03D03B4800F025FB6FE0384B1B7833
:10BF1800032B03D1384800F01DFB67E0344B1B7836
:10BF2800012B03D1354800F015FB5FE0304B5B78FF
:10BF38000D2B57D801A252F823F000BF7DBF00088F
:10BF480085BF00088DBF000895BF00089DBF000889
:10BF5800A5BF0008ADBF0008B5BF0008BDBF0008F9
:10BF6800C5BF0008CDBF0008D5BF0008DDBF000869
:10BF7800E5BF0008224800F0EDFA37E0214800F05C
:10BF8800E9FA33E01B4800F0E5FA2FE01E4800F01C
:10BF9800E1FA2BE01C4800F0DDFA27E01B4800F02E
:10BFA800D9FA23E0194800F0D5FA1FE0174800F045
:10BFB800D1FA1BE0154800F0CDFA17E0144800F05C
:10BFC800C9FA13E0124800F0C5FA0FE0104800F073
:10BFD800C1FA0BE00E4800F0BDFA07E00A4800F08D
:10BFE800B9FA03E0064800F0B5FA00BF80BD00BF0B
:10BFF800B003002060000020180000200C00002082
:10C0080024000020300000203C00002048000020D0
:10C018005400002080B487B000AFF860B9601146C2
:10C028001A460B46FB801346BB80FA88BB889A42A7
:10C0380001D9BB88FB80BB88002B01D10123BB80C1
:10C04800FA8813461B029A1ABB8892FBF3F3FB8209
:10C05800FB681B781A46FB8AC3F1FF0303FB02F255
:10C06800BB681B781946FB8A01FB03F31344204A7B
:10C0780082FB03121A44D211DB17D31ADAB23B6AD5
:10C088001A70FB685B781A46FB8AC3F1FF0303FB4F
:10C0980002F2BB685B781946FB8A01FB03F3134481
:10C0A800134A82FB03121A44D211DB17D31ADAB2ED
:10C0B8003B6A5A70FB689B781A46FB8AC3F1FF03F8
:10C0C80003FB02F2BB689B781946FB8A01FB03F36A
:10C0D8001344074A82FB03121A44D211DB17D31AFE
:10C0E800DAB23B6A9A7000BF1C37BD4680BC704705
:10C0F8008180808042EA002242EA014230B44FF057
:10C10800180C4FF40075D343564C52E000BF00BFE3
:10C1180000BF00BF00BF00BF00BF00BF00BF00BF1F
:10C1280000BF00BF00BF00BF00BF00BF00BF00BF0F
:10C1380000BF00BF00BF00BF00BF00BF00BF6561F8
:10C1480000BF00BF00BF00BF00BF00BF00BF00BFEF
:10C1580000BF00BF00BF00BF00BF00BF00BF00BFDF
:10C1680000BF00BF00BF00BF00BF00BF00BF00BFCF
:10C1780000BF00BF00BF00BF00BF00BF00BF00BFBF
:10C1880000BF00BF00BF00BF00BF00BF00BF00BFAF
:10C1980000BF00BF00BF00BF00BF00BF00BF00BF9F
:10C1A80000BF00BF00BF00BFBCF1010C4FEA430352
:10C1B80055D01A022561A9D400BF00BF00BF00BF37
:10C1C80000BF00BF00BF00BF00BF00BF00BF00BF6F
:10C1D80000BF00BF00BF00BF00BF00BF00BF00BF5F
:10C1E80000BF00BF00BF00BF00BF00BF00BF00BF4F
:10C1F80000BF00BF00BF00BF00BF00BF00BF00BF3F
:10C2080000BF00BF00BF00BF00BF00BF00BF00BF2E
:10C2180000BF00BF00BF00BF00BF00BF00BF00BF1E
:10C22800656100BF00BF00BF00BF00BF00BF00BF07
:10C2380000BF00BF00BF00BF00BF00BF00BF00BFFE
:10C2480000BF00BF00BF00BF00BF00BF00BF00BFEE
:10C2580000BF00BFBCF1010C4FEA4303A9D130BCB9
:10C26800704700BF0010014038B50C46EFF3108549
:10C2780072B6827841780078FFF73CFFA27861783F
:10C288002078FFF737FF85F3108838BD80B485B074
:10C2980000AF78607B681B781A4613461B019B1A0F
:10C2A8009B00214A82FB03121A44D211DB17D31ACE
:10C2B800DBB23B727B685B781A4613461B019B1AFC
:10C2C8009B00194A82FB03121A44D211DB17D31AB6
:10C2D800DBB27B727B689B781A4613461B019B1A5C
:10C2E8009B00114A82FB03121A44D211DB17D31A9E
:10C2F800DBB2BB7207F10C0307F1080212681146A2
:10C3080019800233120C1A7000233A7B62F3070378
:10C318007A7B62F30F23BA7B62F31743184614370C
:10C32800BD4680BC704700BF8180808080B582B0E8
:10C3380000AF4C4B5B7FBB7102F000FE3860BB79ED
:10C34800002B18D1484B00221A70484B00221A7053
:10C35800474B00221A70474B00221A60464B0022B6
:10C368001A70464B00221A70444B00225A70434BF5
:10C3780000229A7072E0404B1B78BA799A420ED02C
:10C38800394B00221A70394B00221A70384B0022A0
:10C398001A70384B00221A60374ABB791370354B34
:10C3A8001B683A689A4209D2344BFF221A70334B01
:10C3B80000225A70314B00229A704FE02F4B002216
:10C3C8001A702E4B00225A702C4B00229A702C4B5C
:10C3D8001B683A68D31A632B3FD9294A3B68136014
:10C3E8000023FB71224B1B78002B06D0204B1B78B7
:10C3F800013BDAB21E4B1A701EE01B4B1B78BA7950
:10C408009A4213D9194B1B78002B03D1174B0122E1
:10C418001A7011E00123FB71144B00221A70124BA1
:10C428001B780133DAB2104B1A7005E00E4B00226C
:10C438001A700F4B1E221A70FB79002B0ED03B6826
:10C4480064330C4A13600D4BFF221A700B4B002209
:10C458005A700A4B00229A7000E000BF0837BD46A8
:10C4680080BD00BFB00300208E0900208F09002086
:10C4780090090020940900209809002078090020DC
:10C488009C09002080B483B000AF78607B681B787B
:10C498001A46642302FB03F3174A82FB03121A4469
:10C4A800D211DB17D21A154B1B689A637B685B782D
:10C4B8001A46642302FB03F30F4A82FB03121A4451
:10C4C800D211DB17D21A0D4B1B68DA637B689B7895
:10C4D8001A46642302FB03F3074A82FB03121A4439
:10C4E800D211DB17D21A054B1B681A6400BF0C3730
:10C4F800BD4680BC704700BF81808080401200200C
:10C5080080B584B000AF78607868FFF7BFFE034657
:10C518001A463A73C3F307227A73C3F30743BB730C
:10C528000B48FFF7B3FE03461A463A72C3F30722D5
:10C538007A72C3F30743BB7207F1080207F10C03D1
:10C5480011461846FFF790FE00BF1037BD4680BD64
:10C558007809002080B483B000AF7860054B7A6812
:10C568001068516803C312891A8000BF0C37BD4692
:10C5780080BC70478409002080B582B000AF0023DA
:10C588003B7100237B710023BB7104210B4806F02B
:10C59800A3FB0821094806F09FFB0C21074806F079
:10C5A8009BFB3B1D1846FFF76DFF3B1D1846FFF729
:10C5B800A7FF00BF0837BD4680BD00BF401200205E
:10C5C80080B582B002AF02F0B9FC0246494B1B6845
:10C5D800D31A142B40F28A8002F0B0FC0346454A75
:10C5E8001360454B5B8801339AB2434B5A80424BE8
:10C5F8001B78032B67D801A252F823F015C6000850
:10C6080047C6000873C60008A5C600083A4B5A88F2
:10C618003A4BDB7819463A4B00930B463749394871
:10C62800FFF7F8FC344B5B88344AD27893424ED9F2
:10C63800314B01221A70304B00225A8047E02E4BB2
:10C648002E4A04331268114619800233120C1A70EC
:10C65800294B5B88294A127993423AD9264B022200
:10C668001A70254B00225A8033E0234B5A88234BFB
:10C678005B791946224B00930B4622491F48FFF766
:10C68800C9FC1D4B5B881D4A5279934223D91A4B2A
:10C6980003221A70184B00225A801CE0164B174AC6
:10C6A800043307321188927819809A70124B5B888C
:10C6B800124A9279934210D90F4B00221A700E4BEE
:10C6C80000225A8009E00C4B00221A7006E000BFD5
:10C6D80004E000BF02E000BF00E000BFFFF726FE55
:10C6E8000748FFF7CFFE0648FFF70AFF00BFBD4621
:10C6F80080BD00BFA00900207C090020840900201B
:10C70800800900208B09002080B500AF0A4B0B4A36
:10C718001A60094B4FF0FF325A60074B4FF4807292
:10C728009A60054806F026F80346002B01D0FEF76C
:10C73800CDFA00BF80BD00BFA4090020002800403A
:10C7480080B584B000AF78607B681B680B4A934261
:10C7580010D104F0A3FF0A4BDB69094A43F00063D8
:10C76800D361074BDB6903F00063FB60FB68054B93
:10C7780001221A6000BF1037BD4680BD0028004066
:10C78800001002403C044242024659B370B50C46C0
:10C79800CB0758BF1549154D48BF144986B054BF3B
:10C7A8000B46134B14F0020F0491124908BF294697
:10C7B80014F0040F104808BF284614F0080F019021
:10C7C8000E480F4E08BF2E4614F0100F18BF05462E
:10C7D8000091CDE902650B4905940420FDF7C0FEE0
:10C7E80006B070BD04200849FDF7BABE688201088A
:10C7F800707E0108747E0108787E0108847E010835
:10C808007C7E0108AC7E01088C7E010830B54FF4AF
:10C818008072054683B01149114807F058FA08B9E3
:10C8280003B030BD04460E4807F063FE02462346B7
:10C8380014460C492A4604200094FDF791FE032073
:10C848002146FFF7A1FF084800F0C2FE002CE7D000
:10C85800034803B0BDE8304007F0FABADC0900200D
:10C8680060130020E07E01081C7F010838B51A4BD0
:10C878000C46834213D129B3B1F5807F16D802F054
:10C888005DFB0346154D164A214616482B6013607A
:10C8980000F0F6FDBDE838401348FFF7B7BF0A4679
:10C8A800BDE8384005201149FDF75ABE4FF48073A2
:10C8B8000A4604200E49FDF753FEBDE838400A48F1
:10C8C800FFF7A4BF05200B49FDF74AFEBDE8384035
:10C8D8000548FFF79BBF00BF60130020EC0C002049
:10C8E800F00C0020DC090020A87F0108387F01082F
:10C8F800B87F0108747F0108F8B5044607F0F9FD10
:10C90800294B05469C4232D0284EB44217D0284BBA
:10C918009C4245D00346002226490420FDF720FE0C
:10C9280029460020FFF730FF204607F091FA2046FD
:10C9380007F026FA2046BDE8F84001F005B903469D
:10C9480003221C490420FDF70BFE29460320FFF7AC
:10C958001BFF204607F07CFA204607F011FA002258
:10C96800154B16481A70BDE8F840FFF74FBF022272
:10C9780017460E4E2B460F490420FDF7F1FD2946B8
:10C988003846FFF701FF204607F062FA204607F015
:10C99800F7F9B442E3D02046BDE8F84001F0D4B836
:10C9A80005221746E6E700BF181300206013002091
:10C9B80088120020F87F0108DE0C0020448001085E
:10C9C80080B582B000AF78607B68164A934224D164
:10C9D800154B00221A70154B1B88002B1ED0134BC9
:10C9E8001B881A461249134809F033F80E4B0122E6
:10C9F8001A700E4B1B881A460E490A4807F09AF817
:10CA08000346002B05D0084B00221A700A4800F094
:10CA1800DFFD064B00221A8000E000BF0837BD4644
:10CA280080BD00BF60130020DE0C0020DC0C00205D
:10CA3800DC0B0020DC0A00205480010880B582B09D
:10CA480000AF02F07BFA0246A54B1B68D31A002BF5
:10CA580040F36B8202F072FA0346A14A136000F0B9
:10CA68007DFDA04B1B78002B03D09E4B1A789E4B64
:10CA78001A709C4B1B78032B1BD19C4B1B68002BFB
:10CA880005D102F05BFA0346984A136014E002F0FD
:10CA980055FA0246954B1B68D31A1A4642F20F7391
:10CAA8009A4209DD8F4B00221A70904B00221A60BF
:10CAB80002E08E4B00221A608A4B1B78012B19D199
:10CAC8008B4B1B68002B05D102F038FA0346884AC5
:10CAD800136012E002F032FA0246854B1B68D31A43
:10CAE800B3F57A7F09DB7F4B00221A70804B002256
:10CAF8001A6002E07E4B00221A6002F01FFA02461A
:10CB08007C4B1B68D31A0A2B5EDD02F017FA02462B
:10CB1800794B1B68D31AC72B06DD00F09BFB02F08C
:10CB28000DFA0346744A1360744B1B78002B08D027
:10CB380073490420FDF714FD00F02CFB6F4B002215
:10CB48001A70684B1B78012B07D0664B1B78032B98
:10CB580003D0644B5B7F002B1AD002F0EFF902463A
:10CB6800684B1B68D31AB3F57A7F11DD02F0E6F93A
:10CB78000346644A136064490520FDF7F1FC594BEC
:10CB88001B78032B02D16420FDF7A8FA00F002FB02
:10CB98005E4B1B780C2B03D05C4B1B780B2B13D1F3
:10CBA80002F0CCF90246574B1B68D31AB3F57A7FCB
:10CBB8000ADD02F0C3F90346524A136054490520BE
:10CBC800FDF7CEFC00F0E6FA524B1B68002B0CD0A8
:10CBD80002F0B4F902464F4B1B68D31A1A4641F2C9
:10CBE80088339A4201DD012300E00023FB71494BA1
:10CBF8001B68002B0CD002F0A1F90246454B1B68BC
:10CC0800D31A1A4642F210739A4201DD012300E05A
:10CC18000023BB71BB797B71FB79002B0AD03E4B9B
:10CC28001B78002B06D13D490420FDF799FC3A4BAF
:10CC380001221A70BB79002B0AD0394B1B78002BC4
:10CC480006D138490420FDF78BFC354B01221A70B8
:10CC5800FB79002B05D1304B00221A70304B002293
:10CC68001A70314ABB791370304B1B78052B00F2D0
:10CC7800138101A252F823F099CC0008C1CC000816
:10CC88003DCD000881CD0008BDCD000815CE0008B7
:10CC980000210520FCF78CFD0020FDF727F9244B27
:10CCA8001B78002B00F0ED807B79002B40F0E980A9
:10CCB8001E4B02221A70E4E000210520FCF778FDE3
:10CCC8000220FDF713F9074B5B7F002B40F0DB8058
:10CCD8007B79002B40F0D780144B02221A70D2E0E7
:10CCE800440D0020B0030020D8090020480D002082
:10CCF8004C0D0020D0090020500D0020DF0C002032
:10CD080070800108D409002084800108400D0020AB
:10CD18009C800108E40C0020E90C0020B880010880
:10CD2800EA0C0020CC800108E80C0020410D00200E
:10CD3800F011002001210520FCF73AFD0120FDF744
:10CD4800D5F87C4B1B78012B03D07A4B1B78022B30
:10CD580002D1794B03221A70784B5B7F002B00F0CD
:10CD68009480764B5B7F1A4675490420FDF7F8FBE3
:10CD7800714B01221A7088E001210520FCF718FD8B
:10CD88000420FDF7B3F86D4B1B78022B06D16D49D3
:10CD98000720FDF7E5FB684B04221A70654B1B78EA
:10CDA800002B74D168490720FDF7DAFB624B022299
:10CDB8001A706CE001210520FCF7FAFC634B1B7824
:10CDC800022B03D9614B1B78042B03D10320FDF7F9
:10CDD8008DF804E05D4B1B781846FDF787F8554B36
:10CDE8001B78002B06D158490720FDF7B9FB524B99
:10CDF80002221A70564B1B78002B4AD0554907203F
:10CE0800FDF7AEFB4C4B05221A7042E000210520CD
:10CE1800FCF7CEFC0D20FDF769F802F08FF802460A
:10CE28004D4B1B68D31AB3F57A7F1ADD02F086F8EA
:10CE38000346494A1360464B1B78002B0AD0444BE3
:10CE48001B78FF2B0DD0424B1B78013BDAB2404BCD
:10CE58001A7006E041490720FDF782FB364B022293
:10CE68001A703B4B1B78002B15D1324B1B78012BCA
:10CE780011D13B490720FDF773FB2F4B03221A7092
:10CE880009E000BF08E000BF06E000BF04E000BF03
:10CE980002E000BF00E000BFBB79002B14D0274B95
:10CEA8000022DA75294B00221A706420FDF716F962
:10CEB800214B1B78012B24D01F4B1B78002B20D033
:10CEC8001D4B01221A701CE0264B1B78012B03D145
:10CED8001A4B0022DA7514E0234B1B78002B14BF81
:10CEE80001230023DBB21A46144BDA75134BDB7DA2
:10CEF800002B06D1114B5B78032B02D10F4B00227C
:10CF0800DA750C4B1B78012B07D00A4B1B78022BC8
:10CF180003D0084B1B78032B03D1084B01229A77C7
:10CF280004E0064B00229A7700E000BF0837BD46B0
:10CF380080BD00BF05000020410D0020B003002087
:10CF4800F48001081C81010840810108400D00207F
:10CF5800E00C002050810108540D00206081010878
:10CF680088810108D8090020D909002080B500AFC0
:10CF7800FDF792F86420FDF7B1F8134B4FF47A727D
:10CF88001A80114B96225A800F4B40F232529A80E7
:10CF98000D4B0A22DA800C4B49F640429A6001F0A8
:10CFA800CDFF0346094A1360084B1B68084A136003
:10CFB8000848FFF72BFC00F0E3F807490720FDF7C6
:10CFC800CFFA00BF80BD00BFB8090020EC0C0020DC
:10CFD800F00C0020C4810108CC810108E9B3844623
:10CFE80000B58E464FF6FF701D49E6441CF8012B2C
:10CFF800424042F300030B4083EA520343F300022A
:10D008000A40C3F34E035A4042F300030B40C2F3F5
:10D018004E02534043F300020A40C3F34E035A4002
:10D0280042F300030B40C2F34E02534043F30002A5
:10D038000A40C3F34E035A4042F300030B40C2F3C5
:10D048004E02534043F300000840C3F34E035840D8
:10D05800E64580B2CAD15DF804FB4FF6FF70704711
:10D0680001A0FFFF80B586B000AFB9607B600346C2
:10D07800FB731346BB81BB890333FB82FA8A3B8C63
:10D088009A4201D9002329E07B68FA7B1A70BB8990
:10D09800002B09D0BB68002B06D07B680133BA8906
:10D0A800B968184608F0D5FCBB8901339BB219460C
:10D0B8007868FFF793FF0346BB82BB8901337A6820
:10D0C8001344BA8AD2B21A70BB8A1B0A99B2BB89B6
:10D0D80002337A681344CAB21A70FB8A18461837A2
:10D0E800BD4680BD80B586B002AF03463960FB718E
:10D0F8001346BB80BA88F8794FF480730093194BB4
:10D108003968FFF7AFFF0346FB81FB89002B1FD06F
:10D11800154B1B78002B09D0FB891A461149134877
:10D1280008F097FC124AFB89138011E00E4B01228C
:10D138001A70FB891A460B490E4806F0FBFC034699
:10D14800002B05D0084B00221A700B4800F040FA5B
:10D1580001F0F4FE0346094A136000BF1037BD46CC
:10D1680080BD00BFDC0A0020DE0C0020DC0B0020A4
:10D17800DC0C002060130020D8810108D0090020B1
:10D1880080B500AF002200215220FFF7ABFF00BF9F
:10D1980080BD00BF80B500AF002200215320FFF7FB
:10D1A800A1FF00BF80BD00BF80B582B000AF01F015
:10D1B800C5FE78601E4B1B687A68D31A3B601C4A10
:10D1C8007B6813601B4BB3F813309BB21A46194B9C
:10D1D800B3F815309BB202FB03F3174A82FB031224
:10D1E8009210DB17D31A1A46144B1A60134B1B689C
:10D1F8003A6802FB03F3124AA2FB03239A09114B74
:10D208001B6813440F4A13600F4B1B78012B02D184
:10D218000C4B00221A600B4B1B680C4AA2FB032321
:10D22800DB0A0B4A136000BF0837BD4680BD00BF4C
:10D23800580D0020B003002067666666C409002008
:10D24800D34D6210C8090020400D0020C5B3A2913B
:10D25800CC09002080B500AFFFF7A6FFFCF766FFFA
:10D2680003461A462A4B1A702A4BDA7A284B5A7008
:10D27800294BB3F813309AB2254B5A80264BB3F892
:10D2880015309AB2224B9A80244B1B68204AC2F868
:10D298000630234B1B681E4AC2F80A30214B1B7804
:10D2A800042B04D1204B1A78194BDA7402E0184B7E
:10D2B8000022DA741D4B1A88154B9A821B4B5A8828
:10D2C800134BDA82194B9A88114B1A83174BDA8859
:10D2D8000F4B5A83154B9B680D4AD361144B1A7830
:10D2E8000B4B9A740A4A002343F07F4343F47F03AD
:10D2F80043F43B4343F0A003D381002343F00D03E1
:10D308001382202202495020FFF7ECFE00BF80BDA7
:10D31800F40C00201C090020B0030020C4090020E0
:10D32800CC090020410D002005000020B80900208C
:10D33800E20C00204038C0B209289ABF024B33F8EB
:10D3480010004FF6FF70704708860108F8B50446CC
:10D358000D4601F0F3FD00233B4A3C4E13703C4A56
:10D36800306013703B4A1370A4F14003092B63D853
:10D37800DFE803F00914594C531B282C480501F029
:10D38800DDFD3060F8BD2878334B642828BF642061
:10D398001B78324A032B107041D1F8BD2B78304AE4
:10D3A800003B18BF01231370F8BD28882A4BA3F847
:10D3B8000F006A8880B2A3F81B2091B2BDE8F8403C
:10D3C800FDF746BD2A78274B1A70F8BD264F2C4624
:10D3D8003E4605F1200C354620686168A268E3687E
:10D3E800103464450FC506F11006F4D16168A268CF
:10D3F800206807C61D4A7B881749A2FB0323DB0860
:10D408008B70F8BD2A781A4B1A70F8BD2B78194A18
:10D41800003B18BF01231370F8BD104B1878BDE806
:10D42800F840FCF75BBE2B78002BABD0BDE8F8408A
:10D4380005201149FDF794B82246BDE8F8400520BB
:10D448000E49FDF78DB800BFE80C0020E40C002061
:10D45800E90C0020EA0C0020B00300206A0000203C
:10D46800D9090020E20C0020140D0020CDCCCCCC32
:10D47800400D0020E10C0020F48101080C82010815
:10D488002DE9F04102290C46054684B030D94318ED
:10D4980013F8012C13F8027CCE1E023989B247EA30
:10D4A800022790F80080FFF799FD8742B6B212D1A3
:10D4B8004046FFF73FFF4FF6FF7290423AD0864250
:10D4C8002AD13246FEB931464046FFF73FFF0120D8
:10D4D80004B0BDE8F0810290234642460420CDE91D
:10D4E80000671849FDF73CF8002004B0BDE8F0815A
:10D4F800D9B1012902784FF0050009D06B7812499B
:10D50800FDF72EF8F0E74046691CFFF71FFFDEE73E
:10D518000E49FDF725F8E7E703464246CDE90064E2
:10D528000B490420FDF71CF8DEE70A490520FDF742
:10D5380017F8D9E723464246074900960520FDF724
:10D548000FF8D1E7FC820108C88201089C82010813
:10D55800A48301086C8201086083010880B582B049
:10D5680000AF01F0EBFC0246144B1B68D31A7B603A
:10D5780001F0E4FC0246124B1B68D31A3B607B683F
:10D5880040F2DB52934215DD3B6840F2DB52934296
:10D5980010DD0C4B93F84230DBB2202B0AD10A483D
:10D5A800FFF734F9094800F013F801F0C7FC034607
:10D5B800034A136000BF0837BD4680BDEC0C00204D
:10D5C800F00C002060130020FC8301080884010887
:10D5D80080B586B004AF78600D4806F08AFF034630
:10D5E8000B4A92F84120D2B21146094A92F84220D9
:10D5F800D2B21046074A12780292019000917A68D6
:10D6080005490420FCF7ACFF00BF0837BD4680BDC4
:10D6180060130020DE0C00202084010880B400AFD5
:10D628000E4B1B681B689AB20D4B1A800B4B1B687C
:10D638005A790B4B9A70094B1B681A79084BDA70A8
:10D64800074B01229A80064B0022DA80044B1822ED
:10D658001A8100BFBD4680BC704700BF0000002093
:10D66800E011002080B500AF4FF4047200210D488E
:10D6780008F062F94FF4047200210B4808F05CF9D5
:10D688000A4B00221A7001F059FC0346084A13603D
:10D69800074B1B68074A136000F014FA00F036FACB
:10D6A80000BF80BD5C0D00206C0F00207D110020A4
:10D6B800801100208411002080B500AF01F03EFCED
:10D6C8000246214B1B68D31A002B3BDD01F036FCC8
:10D6D80003461D4A136000F0ADF900F0F3F900F0BD
:10D6E80015FA1A4B93F84130DBB2212B14D1184BA1
:10D6F800D3F80C32002B0FD001F020FC0246144B5B
:10D70800D3F80C32D31A642B06DD104806F038FB28
:10D718000F4B0022C3F80C220D4B93F80832DBB2F2
:10D72800002B10D0094B93F84130DBB2212B0AD0E3
:10D73800084800F087FA064B002283F8082200F018
:10D74800C1F900E000BF80BDEC11002018130020D3
:10D758005C0D00205C0F00202E4B70B51A68036822
:10D768000C46934219D02C4A1268934204D02B4A93
:10D77800126893424AD070BD99B329492246A1F54F
:10D78800807000F049F910BB224605202549FCF7B6
:10D79800E7FEBDE8704000F0B9B991B301F0CEFBE7
:10D7A8000022214B21491A700346214D214E224661
:10D7B800A1F580702B60336000F02EF90546A8B102
:10D7C80000221D4B1A70BDE8704000F07BB90122A1
:10D7D800194B1A481A7000F035FABDE8704000F08D
:10D7E80095B917490520FCF7BBFEC6E7224615493F
:10D7F8000520FCF7B5FE14222946284600F0B6F8A5
:10D80800DEE711490520FCF7ABFEC7E7BDE870402D
:10D81800FFF72CB81813002088120020601300208E
:10D828006C100020B48401087D1100205C0E0020DB
:10D8380084110020801100207C1100206C11002030
:10D8480090840108708401084C840108084B1A6808
:10D858000368934204D0074A1268934205D0704780
:10D868000022054BC3F80C227047FFF7A9B800BF88
:10D8780018130020601300205C0D0020C9B34FF07E
:10D88800FF3300B51C4A014410F801EB8EEA030E81
:10D898004EF300034EF3400C134083EA5E030CEA98
:10D8A800020C8CEA530C43F340034CF3400E134034
:10D8B80083EA5C030EEA020E8EEA530E43F340033A
:10D8C8004EF3400C134083EA5E030CEA020C8CEA28
:10D8D800530C43F3400313404CF3400E83EA5C03BC
:10D8E80081420EEA020C8CEA5303CDD1D8435DF88D
:10D8F80004FB0846704700BF2083B8ED70B5154695
:10D90800137060B359B39446022302784C1EA4B234
:10D918001C440CF8012F05E010F8011FFB2B0CF834
:10D92800011F20D0A34203F10103F5D1A1B24E1C7F
:10D93800B6B22846FFF7A2FF0346711CB21C2B554E
:10D94800C3F3072CC3F3074489B292B2C3F3076346
:10D9580005F806C0F01C6C54AB5480B270BD0124AD
:10D9680002262146E5E7002070BD00BF38B5134602
:10D97800114AFFF7C3FF80B10446104890F84130C0
:10D98800202B0BD10C4D224629460C4806F0D2F824
:10D9980058B901F0D3FAC5F80C0238BD06F0F0F911
:10D9A80007490520FCF7DCFDECE704490548BDE81C
:10D9B800384000F005B900BF5C0D002018130020A6
:10D9C800D4840108048501082DE978414B1FFB2BFD
:10D9D80013D804398CB203199D7890465A782D04CF
:10D9E80045EA0225025DDB781543214645EA0365D1
:10D9F8000646FFF743FF854202D00020BDE8788144
:10DA0800731CC8F804303378013C88F8003088F873
:10DA180001400120BDE8788110B50446084611464A
:10DA280004F50072FFF7D0FF18B10123184684F8F7
:10DA3800083210BD80B582B000AF01F07FFA78607F
:10DA48001A4B1B687A68D31A3B603B6841F28732ED
:10DA5800934212DD164B1B78DBB2002B09D1154B14
:10DA6800002283F8082241F2883213490520FCF786
:10DA780077FD0F4B01221A7002E00D4B00221A703D
:10DA88000E4B93F84230DBB2202B0AD10C4B1B68AB
:10DA98007A68D31AC72B04DD00F014F8084A7B68AB
:10DAA800136000BF0837BD4680BD00BF801100204D
:10DAB8007D1100205C0D002020850108181300202E
:10DAC8008411002080B500AF0C4B93F84230DBB2D4
:10DAD800202B11D10A4B93F80832DBB2002B0BD163
:10DAE800FF220849054806F0F2F80346002B03D048
:10DAF8000249054800F064F800BF80BD18130020F3
:10DB08005C0D00205C0E00204485010880B500AF44
:10DB18000A4B93F84230DBB2202B0DD1FF22084983
:10DB2800064806F077F80346002B04D00349054859
:10DB380000F046F800E000BF80BD00BF881200205A
:10DB48006C1000205C85010880B582B000AF786059
:10DB58007B68154A934215D11349144800F030F8F0
:10DB6800114806F075F9104806F00AF9104B002222
:10DB7800C3F80C22FFF7A6FF01F0E0F903460D4AAF
:10DB880013600CE07B680C4A934208D10A490B48A1
:10DB980000F016F8084806F05BF9FFF7B7FF00BF7A
:10DBA8000837BD4680BD00BF1813002074850108E2
:10DBB8005C0D00208411002088120020888501084F
:10DBC80090B587B004AF786039607B68002B1CD0B3
:10DBD8003B68002B19D03B681B681C46386806F068
:10DBE80088FC02463B6893F84130DBB219463B6833
:10DBF80093F84230DBB202930191009223467A688F
:10DC080004490420FCF7ACFC00E000BF0C37BD461B
:10DC180090BD00BF9C85010880B400AFBFF34F8F53
:10DC280000BF064BDB6803F4E0620449044B13436E
:10DC3800CB60BFF34F8F00BF00BFFDE700ED00E0F2
:10DC48000400FA0580B584B000AF78601323FB7335
:10DC58007B681B78C22B00F3D180B02B0FDA602BC6
:10DC680042D0602B00F3CA80502B43D0502B00F3D6
:10DC7800C580012B00F0AB80402B2DD0BEE0B03B1F
:10DC8800122B00F2BB8001A252F823F003DD00083A
:10DC980005DE000805DE000805DE000805DE0008D0
:10DCA800B5DD000805DE0008ABDD000805DE00086C
:10DCB80005DE000805DE000805DE000805DE0008B0
:10DCC80005DE000805DE000805DE000841DD000865
:10DCD800A5DD000879DD000800F0B6F840225821DB
:10DCE8004D48FFF743FE94E060220A214B48FFF7B6
:10DCF8003DFE8EE0FCF7D2FB8BE07B685B780B2B5C
:10DD080017D17B685A68464B1068516803C311895C
:10DD1800927A19809A70434B01221A70404BD3F8BB
:10DD280003303F4A40490720FCF71AFC1223FB73D3
:10DD380067E01323FB7364E07B685B78012B14D1E5
:10DD48007B685B681B781A464FF47A7302FB03F30F
:10DD58001A46364B5A61354B5B691A4634490720D7
:10DD6800FCF7FEFB1223FB734BE01323FB7348E025
:10DD78007B685B78012B0ED17B685B681A782D4B2A
:10DD88001A702C4B1B781A462B490720FCF7E8FB26
:10DD98001223FB7335E01323FB7332E01323FB7369
:10DDA8002FE0FCF75BFC1223FB732AE01222002110
:10DDB8000020FFF7DBFD00BF204B93F84130DBB2BA
:10DDC800212BF9D00A2001F0C3F8FFF725FF7B6863
:10DDD8005B78092B0FD17B685A68194B106851681A
:10DDE80003C3127A1A70174B1B78DBB2012B0FD0C2
:10DDF8001223FB7305E01323FB7302E01323FB7369
:10DE080000BFFB7B1A4600210020FFF7AFFD00E0B2
:10DE180000BF1037BD4680BD88110020E0110020EA
:10DE280078000020F0110020CC8501081C09002092
:10DE3800E0850108B0030020F485010818130020CC
:10DE48006C0000207C11002080B500AF8F4B9A78C1
:10DE58008F4B9A708D4BD3F807308D4AC2F8033038
:10DE68008A4BB3F80F309AB2894BA3F80720874B37
:10DE7800B3F81B309AB2864BA3F80920834BB3F84A
:10DE880013309AB2824BA3F80B20804BB3F81530AD
:10DE98009AB27F4BA3F80D207C4B1A7E7C4BDA7329
:10DEA8007A4B5A7F7A4B5A70784B5A78784B1A705B
:10DEB800774B00221A7400225A74754B00229A7408
:10DEC800734B0022DA7400221A750420FBF7E0FC79
:10DED800034603F00103D9B26D4A537D61F3000391
:10DEE80053750320FBF7D4FC034603F00103D9B2B2
:10DEF800674A537D61F3410353750020FBF7C8FC63
:10DF0800034603F00103D9B2614A537D61F38203EA
:10DF180053755F4A537D23F0080353750320FBF7BD
:10DF2800C7FC0346002B0CBF01230023D9B2584A73
:10DF3800537D61F304135375FCF79CFA0346002BD9
:10DF480014BF01230023D9B2514A537D61F345130D
:10DF580053754F4A537D23F0400353754D4B1B7A3D
:10DF680003F00103D9B24A4A537D61F3C7135375CD
:10DF78000020FBF7C3FD03465AB2454B5A760120F1
:10DF8800FBF7BCFD03465AB2414B9A76414B1B6ADC
:10DF98005AB23F4BDA763E4B00221A773C4B0022AE
:10DFA8005A773B4B00229A770022DA77384B0022C7
:10DFB80083F82020384B9B689AB2354BA3F8212070
:10DFC800354BDB689AB2324BA3F82320324B1B69DE
:10DFD8009AB22F4BA3F82520112200212F4807F0D1
:10DFE800ABFC2B4B002283F83820294B002283F806
:10DFF8003920002283F83A20254B002283F83B2061
:10E00800002283F83C2004220021254807F094FCD4
:10E018001F4B002283F84120002283F8422000226F
:10E0280083F84320002283F84420194B002283F808
:10E038004720174B002283F84620154B002283F80F
:10E048004520134B002283F84820002283F84920FA
:10E058000F4B002283F84A2008220021114807F0BC
:10E068006BFC0B4B002283F85320094B002283F8EA
:10E078005420002283F85520054B002283F85620AF
:10E08800002283F8572000BF80BD00BFB0030020E6
:10E09800881100201C090020F0080020AF11002082
:10E0A800C5110020D311002080B485B000AF78607E
:10E0B8007B68002B18D07B6800221A607B680022DE
:10E0C8009A807B680022DA800023FB8108E0FA89C5
:10E0D8007B680232002143F82210FB890133FB815F
:10E0E800FB89072BF3D900E000BF1437BD4680BC7D
:10E0F800704780B485B000AF786039607B68002BCA
:10E1080001D13B6856E07B68DB88072B27D87B6802
:10E118009B881A467B680232396843F822107B686C
:10E128001A683B681A447B681A607B689B880133CD
:10E138009AB27B689A807B689B88072B02D97B6898
:10E1480000229A807B68DB8801339AB27B68DA8088
:10E158007B681B687A68D28893FBF2F32AE07B68B5
:10E168009B881A467B68023253F82230FB607B6832
:10E178009B881A467B680232396843F822107B680C
:10E188001A683968FB68CB1A1A447B681A607B687E
:10E198009B8801339AB27B689A807B689B88072B9F
:10E1A80002D97B6800229A807B681B68002B00DA02
:10E1B8000733DB1018461437BD4680BC7047000093
:10E1C80080B485B000AF154B9B69144A43F0010336
:10E1D8009361124B9B6903F00103BB60BB680F4B53
:10E1E800DB690E4A43F08053D3610C4BDB6903F0C3
:10E1F80080537B607B680A4B5B68FB60FB6823F09D
:10E20800E063FB60FB6843F00073FB60044AFB6853
:10E21800536000BF1437BD4680BC704700100240F1
:10E2280000000140FEE700BFFEE700BFFEE700BFB9
:10E23800FEE700BFFEE700BF704700BF704700BFA2
:10E24800704700BF00F068BE10B5094C01224FF4BA
:10E258000061204603F009FA064802F0F7FD20465F
:10E26800BDE8104000224FF4006103F0FEB900BF82
:10E27800000C0140C0020020014802F0E7BD00BFC9
:10E2880074140020014802F0E1BD00BF30140020E2
:10E29800014802F0DBBD00BFA8130020014802F0CE
:10E2A800D5BD00BFEC13002010B5094C01224FF476
:10E2B8000061204603F0D9F9064801F023F820460A
:10E2C800BDE8104000224FF4006103F0CEB900BF52
:10E2D800000C01409002002010B5094C01224FF4B7
:10E2E8008061204603F0C1F9064802F047F820464D
:10E2F800BDE8104000224FF4806103F0B6B900BFBA
:10E30800000C01405C03002010B5094C01224FF4B9
:10E318000061204603F0A9F9064804F087FD20466D
:10E32800BDE8104000224FF4006103F09EB900BF21
:10E33800000C0140F8110020014805F02DBE00BF77
:10E34800D012002010B5084C01222021204603F0ED
:10E358008CF9064805F020FE2046BDE81040002252
:10E36800202103F082B900BF0008014018130020E3
:10E3780010B5084C01224021204603F076F90648E2
:10E3880005F00AFE2046BDE810400022402103F0B7
:10E398006CB900BF000801406013002010B5084C9C
:10E3A80001220421204603F060F9064805F0F4FD37
:10E3B8002046BDE810400022042103F056B900BFF2
:10E3C800001001408812002010B5094C01224FF4BA
:10E3D8008061204603F049F9064801F0CFFF204646
:10E3E800BDE8104000224FF4806103F03EB900BF41
:10E3F800000C01408403002010B5094C01224FF4A1
:10E408008061204603F031F9064801F0B7FF204645
:10E41800BDE8104000224FF4806103F026B900BF28
:10E42800000C01408403002080B400AF012318468B
:10E43800BD4680BC704780B582B000AF7860396057
:10E4480007F0CCFA034616221A604FF0FF3318463D
:10E458000837BD4680BD80B582B000AF78604FF008
:10E46800FF317868FFF7E7FF00BFFDE780B586B0AA
:10E4780000AFF860B9607A6000237B610AE0AFF30F
:10E4880000800146BB685A1CBA60CAB21A707B6920
:10E4980001337B617A697B689A42F0DB7B681846B6
:10E4A8001837BD4680BD80B483B000AF78604FF0A8
:10E4B800FF3318460C37BD4680BC704780B483B024
:10E4C80000AF786039603B684FF400525A6000230F
:10E4D80018460C37BD4680BC704780B483B000AF87
:10E4E8007860012318460C37BD4680BC704780B45D
:10E4F80085B000AFF860B9607A6000231846143719
:10E50800BD4680BC7047000080B586B000AF78601B
:10E51800144A154BD31A7B617B693B61134B1B680B
:10E52800002B02D1114B124A1A60104B1A687B68F3
:10E5380013443A699A4207D207F050FA03460C226C
:10E548001A604FF0FF3309E0084B1B68FB60074B6C
:10E558001A687B681344054A1360FB681846183725
:10E56800BD4680BD0000012000040000F411002019
:10E578000816002080B400AF00BFBD4680BC7047BD
:10E5880080B58EB000AF07F1280300221A605A60E8
:10E598009A60DA6007F1200300221A605A603B1D76
:10E5A80000221A605A609A60DA601A615A619A61A8
:10E5B800384B394A1A60374B00225A60354B0022D3
:10E5C8009A60344B4FF6FF72DA60324B00221A61C0
:10E5D800304B00229A612F4804F0D5F90346002BEE
:10E5E80001D0FCF773FB4FF48053BB6207F128039B
:10E5F8001946284804F028FE0346002B01D0FCF7F2
:10E6080065FB244804F00EFA0346002B01D0FCF702
:10E618005DFB204804F008FB0346002B01D0FCF703
:10E6280055FB30233B6200237B6207F12003194628
:10E63800184805F0B7F90346002B01D0FCF746FB54
:10E6480000237B600123BB600023FB6000237B6108
:10E658003B1D002219460F4804F0D8FC0346002B46
:10E6680001D0FCF733FB60237B600023BB603B1DBC
:10E6780004221946074804F025FD0346002B01D063
:10E68800FCF724FB034800F0CFF800BF3837BD463D
:10E6980080BD00BFF81100200004004080B58EB096
:10E6A80000AF07F1280300221A605A609A60DA6006
:10E6B80007F1200300221A605A603B1D00221A60ED
:10E6C8005A609A60DA601A615A619A61374B384A1F
:10E6D8001A60364B4FF434725A60344B00229A60F9
:10E6E800324B6422DA60314B00221A612F4B002230
:10E6F8009A612E4804F047F90346002B01D0FCF735
:10E70800E5FA4FF48053BB6207F1280319462748FE
:10E7180004F09AFD0346002B01D0FCF7D7FA2348F2
:10E7280004F082FA0346002B01D0FCF7CFFA00234D
:10E738003B6200237B6207F1200319461B4805F062
:10E7480031F90346002B01D0FCF7C0FA60237B6047
:10E758000023BB600023FB6000237B613B1D042278
:10E768001946124804F0AEFC0346002B01D0FCF712
:10E77800ADFA3B1D082219460C4804F0A3FC0346D9
:10E78800002B01D0FCF7A2FA3B1D0C2219460748C2
:10E7980004F098FC0346002B01D0FCF797FA0348D5
:10E7A80000F042F800BF3837BD4680BD4012002057
:10E7B8000008004080B584B000AF78607B681B68B3
:10E7C800164A934214D1164BDB69154A43F00203EB
:10E7D800D361134BDB6903F00203FB60FB68002283
:10E7E80006211D2002F0C5F81D2002F0DEF810E019
:10E7F8007B681B680B4A93420BD1094BDB69084ABB
:10E8080043F00403D361064BDB6903F00403BB60E8
:10E81800BB6800BF1037BD4680BD00BF0004004084
:10E82800001002400008004080B58AB000AF786050
:10E8380007F1140300221A605A609A60DA607B6854
:10E848001B68264A934218D1254B9B69244A43F0FA
:10E8580004039361224B9B6903F004033B613B690A
:10E8680080237B610223BB6102233B6207F114030F
:10E8780019461C4802F05EFD2BE07B681B681A4AAB
:10E88800934226D1164B9B69154A43F020039361A6
:10E89800134B9B6903F02003FB60FB684FF4604354
:10E8A8007B610223BB6102233B6207F11403194613
:10E8B8000E4802F03FFD0E4B5B687B627B6A43F0BB
:10E8C800E0637B627B6A43F480537B62084A7B6A1D
:10E8D800536000BF2837BD4680BD00BF000400401C
:10E8E80000100240000801400008004000140140E8
:10E8F8000000014080B500AF114B124A1A60104B5E
:10E908004FF416525A600E4B00229A600C4B0022AC
:10E91800DA600B4B00221A61094B0C225A61084B32
:10E9280000229A61064B0022DA61054805F0B2F828
:10E938000346002B01D0FCF7C9F900BF80BD00BF1A
:10E94800881200200050004080B500AF114B124AD9
:10E958001A60104B4FF4E1325A600E4B00229A6055
:10E968000C4B0022DA600B4B00221A61094B0C2277
:10E978005A61084B00229A61064B0022DA61054869
:10E9880005F088F80346002B01D0FCF79FF900BF7B
:10E9980080BD00BFD01200200038014080B500AF14
:10E9A800114B124A1A60104B4FF4E1325A600E4B69
:10E9B80000229A600C4B0022DA600B4B00221A618D
:10E9C800094B0C225A61084B00229A61064B00221F
:10E9D800DA61054805F05EF80346002B01D0FCF724
:10E9E80075F900BF80BD00BF181300200044004027
:10E9F80080B500AF114B124A1A60104B4FF4E13248
:10EA08005A600E4B00229A600C4B0022DA600B4BC6
:10EA180000221A61094B0C225A61084B00229A61A4
:10EA2800064B0022DA61054805F034F80346002B4E
:10EA380001D0FCF74BF900BF80BD00BF6013002078
:10EA48000048004080B592B000AF786007F130030D
:10EA580000221A605A609A60DA607B681B68924AE2
:10EA6800934245D1914BDB69904A43F48013D361BB
:10EA78008E4BDB6903F48013FB62FB6A8B4B9B694B
:10EA88008A4A43F010039361884B9B6903F0100393
:10EA9800BB62BB6A854B9B69844A43F02003936140
:10EAA800824B9B6903F020037B627B6A4FF480539F
:10EAB8003B6302237B630323FB6307F1300319469F
:10EAC8007B4802F037FC04233B6300237B6300236D
:10EAD800BB6307F130031946764802F02BFC00228D
:10EAE8000521352001F045FF352001F05EFF93E157
:10EAF8007B681B68704A93423AD16C4B9B696B4A9E
:10EB080043F480439361694B9B6903F480433B6200
:10EB18003B6A664B9B69654A43F004039361634B08
:10EB28009B6903F00403FB61FB694FF400733B63CB
:10EB380002237B630323FB6307F1300319465F4815
:10EB480002F0F8FB4FF480633B6300237B630023F0
:10EB5800BB6307F130031946584802F0EBFB00226B
:10EB68000521252001F005FF252001F01EFF53E1B6
:10EB78007B681B68524A934240F0AE804B4BDB697E
:10EB88004A4A43F40033D361484BDB6903F400334A
:10EB9800BB61BB69454B9B69444A43F020039361C1
:10EBA800424B9B6903F020037B617B6920233B6315
:10EBB80002237B630323FB6307F1300319463D48B7
:10EBC80002F0B8FB40233B6300237B630023BB6355
:10EBD80007F130031946374802F0ACFB394B5B6844
:10EBE8003B643B6C43F0E0633B643B6C43F00803DD
:10EBF8003B64344A3B6C5360334B344A1A60324BA3
:10EC080000225A60304B00229A602F4B8022DA6033
:10EC18002D4B00221A612C4B00225A612A4B0022EC
:10EC28009A61294B4FF44052DA61274801F0F4FE0B
:10EC38000346002B01D0FCF749F87B68224ADA63C7
:10EC4800214A7B685362224B224A1A60204B1022C9
:10EC58005A601F4B00229A601D4B8022DA601C4BC1
:10EC680000221A611A4B00225A61194B00229A613C
:10EC7800174B4FF40052DA61154801F0CDFE0346F8
:10EC8800002B01D0FCF722F87B68114A9A63104ADE
:10EC98007B68536200220221262001F06AFE2620AA
:10ECA80001F083FEB8E000BF0050004000100240B1
:10ECB80000100140001401400038014000080140E4
:10ECC8000044004000000140A81300206C000240EE
:10ECD800EC130020800002407B681B68504A934276
:10ECE80040F09A804F4BDB694E4A43F48023D3614E
:10ECF8004C4BDB6903F480233B613B69494B9B69BF
:10ED0800484A43F010039361464B9B6903F0100394
:10ED1800FB60FB684FF480633B6302237B63032340
:10ED2800FB6307F1300319463F4802F003FB4FF439
:10ED380000633B6300237B630023BB6307F130035D
:10ED48001946394802F0F6FA384B5B687B647B6CED
:10ED580023F030037B647B6C43F0E0637B647B6C63
:10ED680043F010037B64314A7B6C5360304B314A6B
:10ED78001A602F4B00225A602D4B00229A602C4BB0
:10ED88008022DA602A4B00221A61294B00225A613C
:10ED9800274B00229A61264B4FF44052DA612448EF
:10EDA80001F03AFE0346002B01D0FBF78FFF7B688A
:10EDB8001F4ADA631E4A7B6853621F4B1F4A1A6058
:10EDC8001D4B10225A601C4B00229A601A4B80225D
:10EDD800DA60194B00221A61174B00225A61164B50
:10EDE80000229A61144B4FF40052DA61124801F084
:10EDF80013FE0346002B01D0FBF768FF7B680E4A21
:10EE08009A630D4A7B68536200220221272001F091
:10EE1800B0FD272001F0C9FD00BF4837BD4680BDC1
:10EE2800004800400010024000100140000001406E
:10EE38003014002030000240741400201C000240EE
:10EE4800FFF798FB0B480C490C4A002302E0D45802
:10EE5800C4500433C4188C42F9D3094A094C00231E
:10EE680001E013600432A242FBD306F0BDFDFBF7BC
:10EE780043FE70470000002058020020FC8901086A
:10EE88005802002008160020FEE7000080B500AFF9
:10EE9800084B1B68074A43F010031360032001F076
:10EEA8005DFD0F2000F008F8FFF78AF900231846E7
:10EEB80080BD00BF0020024080B582B000AF7860FE
:10EEC800124B1A68124B1B7819464FF47A73B3FB2E
:10EED800F1F3B2FBF3F3184601F075FD0346002B7E
:10EEE80001D001230EE07B680F2B0AD80022796835
:10EEF8004FF0FF3001F03DFD064A7B6813600023A8
:10EF080000E0012318460837BD4680BD8400002074
:10EF18008C0000208800002080B400AF054B1B78CF
:10EF28001A46054B1B681344034A136000BFBD46CD
:10EF380080BC70478C000020B814002080B400AF5B
:10EF4800024B1B681846BD4680BC7047B8140020A9
:10EF580080B584B000AF7860FFF7F0FFB8607B68D9
:10EF6800FB60FB68B3F1FF3F05D00A4B1B781A46DC
:10EF7800FB681344FB6000BFFFF7E0FF0246BB6875
:10EF8800D31AFA689A42F7D800BF00BF1037BD46B7
:10EF980080BD00BF8C00002080B586B000AF7860CF
:10EFA8000023FB7500233B610023BB600023FB604B
:10EFB8007B68002B01D10123BEE07B689B68002B96
:10EFC8007B689B6A002B09D17B680022DA627B6828
:10EFD800002283F824207868FAF760FB786800F04C
:10EFE800BDFB0346FB757B689B6A03F01003002B8F
:10EFF80040F09980FB7D002B40F095807B689B6AF0
:10F0080023F4885323F0020343F002027B689A62D8
:10F018007B685A687B68DB691A437B681B7B5B00EB
:10F028001343BA681343BB607B689B68B3F5807F62
:10F0380003D07B689B68012B02D14FF4807300E0FA
:10F0480000233A6913433B617B681B7D012B19D16F
:10F058007B681B7B002B09D17B689B69013B5A03AA
:10F068003B69134343F400633B610BE07B689B6A95
:10F0780043F020027B689A627B68DB6A43F00102F6
:10F088007B68DA627B681B685B6823F469417B688C
:10F098001B683A690A435A607B681B689A68284B60
:10F0A80013407A681268B9680B4393607B689B6861
:10F0B800B3F5807F03D07B689B68012B04D17B6804
:10F0C8001B69013B1B05FB607B681B68DB6A23F43B
:10F0D80070017B681B68FA680A43DA627B681B6800
:10F0E8009A68184B1340BA689A420BD17B68002281
:10F0F800DA627B689B6A23F0030343F001027B68B2
:10F108009A6218E07B689B6A23F0120343F01002AE
:10F118007B689A627B68DB6A43F001027B68DA628B
:10F128000123FB7507E07B689B6A43F010027B684C
:10F138009A620123FB75FB7D18461837BD4680BDD2
:10F14800FDF7E1FFFE0E1FFF80B586B000AFF86047
:10F15800B9607A600023FB75FB681B68644A9342B8
:10F1680004D0FB681B68634A934206D1604B5B6816
:10F1780003F47023002B40F0B380FB6893F824302D
:10F18800012B01D10223AEE0FB68012283F8242081
:10F19800F86800F089FA0346FB75FB7D002B40F008
:10F1A8009A80FB689B6A23F4706323F0010343F49D
:10F1B8008072FB689A62FB681B684E4A934205D1CD
:10F1C8004B4B5B6803F47023002B15D1FB689B6ADB
:10F1D80023F48012FB689A62FB681B685B6803F47F
:10F1E8008063002B26D0FB689B6A23F4405343F4CA
:10F1F8008052FB689A621DE0FB689B6A43F48012A8
:10F20800FB689A62FB681B68394A934204D0FB6822
:10F218001B68384A93420DD1354B5B6803F4806311
:10F22800002B07D0FB689B6A23F4405343F48052B9
:10F23800FB689A62FB689B6A03F48053002B06D034
:10F24800FB68DB6A23F00602FB68DA6202E0FB680F
:10F258000022DA62FB68002283F82420FB681B6A1C
:10F26800254A9A62FB681B6A244ADA62FB681B6AB1
:10F27800234A1A63FB681B686FF002021A60FB6876
:10F288001B689A68FB681B6842F480729A60FB6886
:10F29800186AFB681B684C331946BA687B6801F02A
:10F2A80031FCFB681B689B6803F46023B3F5602F8F
:10F2B80008D1FB681B689A68FB681B6842F4A002C7
:10F2C8009A600FE0FB681B689A68FB681B6842F449
:10F2D80080129A6006E0FB68002283F8242001E08F
:10F2E8000123FB75FB7D18461837BD4680BD00BF5E
:10F2F8000024014000280140E7F7000863F80008EF
:10F308007FF8000880B584B000AF78607B681B6820
:10F318001B68FB607B681B685B68BB60BB6803F0AD
:10F328002003002B3ED0FB6803F00203002B39D0EA
:10F338007B689B6A03F01003002B05D17B689B6AEE
:10F3480043F400727B689A627B681B689B6803F4CD
:10F358006023B3F5602F1DD17B681B7B002B19D16F
:10F368007B681B685A687B681B6822F020025A6019
:10F378007B689B6A23F480727B689A627B689B6ACD
:10F3880003F48053002B05D17B689B6A43F001028C
:10F398007B689A627868FAF7D5F87B681B686FF023
:10F3A80012021A60BB6803F08003002B4DD0FB6883
:10F3B80003F00403002B48D07B689B6A03F010031A
:10F3C800002B05D17B689B6A43F400527B689A62E4
:10F3D8007B681B689B6803F4E043B3F5E04F12D0E9
:10F3E8007B681B685B6803F48063002B25D17B680E
:10F3F8001B689B6803F46023B3F5602F1DD17B68FD
:10F408001B7B002B19D17B681B685A687B681B68BB
:10F4180022F080025A607B689B6A23F480527B68E2
:10F428009A627B689B6A03F48073002B05D17B6822
:10F438009B6A43F001027B689A62786800F0E4FAFC
:10F448007B681B686FF00C021A60BB6803F040030E
:10F45800002B12D0FB6803F00103002B0DD07B6852
:10F468009B6A43F480327B689A62786800F012F8ED
:10F478007B681B686FF001021A6000BF1037BD4639
:10F4880080BD80B483B000AF786000BF0C37BD4644
:10F4980080BC704780B483B000AF786000BF0C3781
:10F4A800BD4680BC704780B483B000AF786000BFB1
:10F4B8000C37BD4680BC704780B485B000AF78601B
:10F4C80039600023FB730023BB607B6893F824300A
:10F4D800012B01D10223DCE07B68012283F8242080
:10F4E8003B685B68062B1CD87B681B68596B3B68BC
:10F4F8005A6813469B001344053B1F2202FA03F384
:10F50800DB4319403B6818683B685A6813469B0000
:10F518001344053B00FA03F27B681B680A435A63ED
:10F528003CE03B685B680C2B1CD87B681B68196B3C
:10F538003B685A6813469B001344233B1F2202FA78
:10F5480003F3DB4319403B6818683B685A68134665
:10F558009B001344233B00FA03F27B681B680A43B1
:10F568001A631BE07B681B68D96A3B685A681346B4
:10F578009B001344413B1F2202FA03F3DB4319406B
:10F588003B6818683B685A6813469B001344413B24
:10F5980000FA03F27B681B680A43DA623B681B685F
:10F5A800092B1CD97B681B68D9683B681A68134605
:10F5B8005B0013441E3B072202FA03F3DB431940A6
:10F5C8003B6898683B681A6813465B0013441E3B07
:10F5D80000FA03F27B681B680A43DA6019E07B686B
:10F5E8001B6819693B681A6813465B0013440722B5
:10F5F80002FA03F3DB4319403B6898683B681A68D2
:10F6080013465B00134400FA03F27B681B680A4345
:10F618001A613B681B68102B03D03B681B68112BD1
:10F6280032D17B681B681D4A934225D17B681B68D1
:10F638009B6803F40003002B26D17B681B689A683B
:10F648007B681B6842F400029A603B681B68102BB9
:10F658001AD1134B1B68134AA2FB03239A0C1346B7
:10F668009B0013445B00BB6002E0BB68013BBB60CE
:10F67800BB68002BF9D107E07B689B6A43F0200246
:10F688007B689A620123FB737B68002283F824203D
:10F69800FB7B18461437BD4680BC704700240140E8
:10F6A8008400002083DE1B4380B584B000AF7860FF
:10F6B8000023FB600023BB607B681B689B6803F02A
:10F6C8000103012B40D07B681B689A687B681B6824
:10F6D80042F001029A601F4B1B681F4AA2FB0323DA
:10F6E8009B0CBB6002E0BB68013BBB60BB68002BA6
:10F6F800F9D1FFF723FCF8601FE0FFF71FFC024673
:10F70800FB68D31A022B18D97B681B689B6803F027
:10F718000103012B11D07B689B6A43F010027B68C0
:10F728009A627B68DB6A43F001027B68DA627B6875
:10F73800002283F82420012307E07B681B689B686C
:10F7480003F00103012BD8D1002318461037BD461A
:10F7580080BD00BF8400002083DE1B4380B584B0D9
:10F7680000AF78600023FB607B681B689B6803F030
:10F778000103012B2ED17B681B689A687B681B6884
:10F7880022F001029A60FFF7D9FBF8601BE0FFF74F
:10F79800D5FB0246FB68D31A022B14D97B681B6879
:10F7A8009B6803F00103012B0DD17B689B6A43F032
:10F7B80010027B689A627B68DB6A43F001027B680F
:10F7C800DA62012307E07B681B689B6803F001038A
:10F7D800012BDCD0002318461037BD4680BD80B50C
:10F7E80084B000AF78607B685B6AFB60FB689B6AEB
:10F7F80003F05003002B27D1FB689B6A43F4007287
:10F80800FB689A62FB681B689B6803F46023B3F586
:10F81800602F15D1FB681B7B002B11D1FB689B6AFD
:10F8280023F48072FB689A62FB689B6A03F4805336
:10F83800002B05D1FB689B6A43F00102FB689A62C2
:10F84800F868F9F77FFE04E0FB681B6A1B6B7868B1
:10F85800984700BF1037BD4680BD80B584B000AF63
:10F8680078607B685B6AFB60F868FFF70AFE00BF98
:10F878001037BD4680BD80B584B000AF78607B6826
:10F888005B6AFB60FB689B6A43F04002FB689A6214
:10F89800FB68DB6A43F00402FB68DA62F868FFF78A
:10F8A80002FE00BF1037BD4680BD000090B587B08E
:10F8B80000AF78600023FB750023FB607B6893F83A
:10F8C8002430012B01D1022397E07B68012283F8C1
:10F8D80024207868FFF742FF0346FB757868FFF736
:10F8E800E3FE0346FB75FB7D002B40F081807B68BF
:10F8F8009B6A23F4885323F0020343F002027B68D7
:10F908009A62404B1C68022002F0E2FD0346B4FBF9
:10F91800F3F35B00FB6002E0FB68013BFB60FB6804
:10F92800002BF9D17B681B689A687B681B6842F0DA
:10F9380008029A60FFF702FB38611BE0FFF7FEFA46
:10F9480002463B69D31A0A2B14D97B681B689B684B
:10F9580003F00803002B0DD07B689B6A23F0120389
:10F9680043F010027B689A627B68002283F82420A7
:10F97800012342E07B681B689B6803F00803002BA7
:10F98800DCD17B681B689A687B681B6842F00402BC
:10F998009A60FFF7D3FA38611BE0FFF7CFFA024607
:10F9A8003B69D31A0A2B14D97B681B689B6803F040
:10F9B8000403002B0DD07B689B6A23F0120343F0ED
:10F9C80010027B689A627B68002283F82420012356
:10F9D80013E07B681B689B6803F00403002BDCD1F1
:10F9E8007B689B6A23F0030343F001027B689A62F9
:10F9F8007B68002283F82420FB7D18461C37BD460F
:10FA080090BD00BF8400002080B483B000AF786050
:10FA180000BF0C37BD4680BC704780B584B000AFCE
:10FA280078607B68002B01D10123EDE07B6893F8B7
:10FA38002030DBB2002B02D17868FAF719F97B681D
:10FA48001B681A687B681B6842F001021A60FFF79E
:10FA580075FAF86012E0FFF771FA0246FB68D31AEC
:10FA68000A2B0BD97B685B6A43F400327B685A62C5
:10FA78007B68052283F820200123C5E07B681B688A
:10FA88005B6803F00103002BE5D07B681B681A68EC
:10FA98007B681B6822F002021A60FFF74FFAF860D1
:10FAA80012E0FFF74BFA0246FB68D31A0A2B0BD970
:10FAB8007B685B6A43F400327B685A627B68052284
:10FAC80083F8202001239FE07B681B685B6803F0B4
:10FAD8000203002BE5D17B681B7E012B08D17B68D4
:10FAE8001B681A687B681B6842F080021A6007E08E
:10FAF8007B681B681A687B681B6822F080021A60A2
:10FB08007B685B7E012B08D17B681B681A687B6861
:10FB18001B6842F040021A6007E07B681B681A689D
:10FB28007B681B6822F040021A607B689B7E012B71
:10FB380008D17B681B681A687B681B6842F0200242
:10FB48001A6007E07B681B681A687B681B6822F0EC
:10FB580020021A607B68DB7E012B08D17B681B685A
:10FB68001A687B681B6822F010021A6007E07B683D
:10FB78001B681A687B681B6842F010021A607B6871
:10FB88001B7F012B08D17B681B681A687B681B6880
:10FB980042F008021A6007E07B681B681A687B68F5
:10FBA8001B6822F008021A607B685B7F012B08D172
:10FBB8007B681B681A687B681B6842F004021A603D
:10FBC80007E07B681B681A687B681B6822F00402E0
:10FBD8001A607B689A687B68DB681A437B681B69D4
:10FBE8001A437B685B6942EA03017B685B685A1EBB
:10FBF8007B681B680A43DA617B6800225A627B686B
:10FC0800012283F82020002318461037BD4680BD06
:10FC180080B487B000AF786039607B681B687B610F
:10FC28007B6893F82030FB74FB7C012B03D0FB7CB2
:10FC3800022B40F0BE80654B7B617B69D3F80032B4
:10FC480043F001027B69C3F800227B69D3F80032D4
:10FC580023F47C527B69C3F800227B69D3F8002225
:10FC68003B685B6A1B021A437B69C3F800223B6846
:10FC78005B6903F01F03012202FA03F3FB607B694F
:10FC8800D3F81C22FB68DB431A407B69C3F81C22AB
:10FC98003B68DB69002B23D17B69D3F80C22FB6816
:10FCA800DB431A407B69C3F80C223B68DB68190404
:10FCB8003B685B689BB23A68526919437B69483272
:10FCC80043F832103B689B6819043B681B689AB27A
:10FCD8003B685B690A4379694833DB000B445A6027
:10FCE8003B68DB69012B22D17B69D3F80C22FB68C6
:10FCF8001A437B69C3F80C223B681B6819043B68EC
:10FD08005B689BB23A68526919437B69483243F889
:10FD180032103B689B6819043B68DB689AB23B6801
:10FD28005B690A4379694833DB000B445A603B68D6
:10FD38009B69002B09D17B69D3F80422FB68DB435C
:10FD48001A407B69C3F8042207E07B69D3F80422D0
:10FD5800FB681A437B69C3F804223B681B69002BC4
:10FD680009D17B69D3F81422FB68DB431A407B690D
:10FD7800C3F8142207E07B69D3F81422FB681A43FE
:10FD88007B69C3F814223B681B6A012B07D17B6986
:10FD9800D3F81C22FB681A437B69C3F81C227B69D1
:10FDA800D3F8003223F001027B69C3F80022002354
:10FDB80006E07B685B6A43F480227B685A62012311
:10FDC80018461C37BD4680BC704700BF0064004021
:10FDD80080B584B000AF78607B6893F82030DBB2E0
:10FDE800012B2ED17B68022283F820207B681B68B8
:10FDF8001A687B681B6822F001021A60FFF79EF8F8
:10FE0800F86012E0FFF79AF80246FB68D31A0A2B4B
:10FE18000BD97B685B6A43F400327B685A627B6863
:10FE2800052283F82020012312E07B681B685B68A9
:10FE380003F00103002BE5D17B6800225A620023FE
:10FE480006E07B685B6A43F400227B685A62012300
:10FE580018461037BD4680BD80B584B000AF7860C5
:10FE68007B6893F82030DBB2022B33D17B681B68A8
:10FE78001A687B681B6842F001021A60FFF75EF897
:10FE8800F86012E0FFF75AF80246FB68D31A0A2B0B
:10FE98000BD97B685B6A43F400327B685A627B68E3
:10FEA800052283F8202001231BE07B681B685B6820
:10FEB80003F00103002BE5D07B681B681A687B6898
:10FEC8001B6822F002021A607B68012283F8202056
:10FED800002306E07B685B6A43F480127B685A6201
:10FEE800012318461037BD4680BD80B489B000AFE5
:10FEF800F860B9607A603B60FB6893F82030FB7764
:10FF0800FB681B689B68BB61FB7F012B03D0FB7FF1
:10FF1800022B40F0AD80BB6903F08063002B0AD14F
:10FF2800BB6903F00063002B05D1BB6903F0805364
:10FF3800002B00F09580BB691B0E03F003037B6167
:10FF480001227B699A403B681A60BB689B68002B5A
:10FF58000DD1BB681B685A05BB68DB68F96809687E
:10FF68001A437B6918331B010B441A600FE0BB6806
:10FF78005B68DA00BB689B681A43BB68DB68F96892
:10FF880009681A437B6918331B010B441A60FB6824
:10FF98001968BB681A697B6918331B010B44043361
:10FFA8001A60BB681B7D012B11D1FB681A687B693D
:10FFB80018331B01134404331B68FA68116843F4AF
:10FFC80080727B6918331B010B4404331A607B6809
:10FFD80007331B781A067B6806331B781B041A4301
:10FFE8007B6805331B781B0213437A680432127846
:08FFF8001046FA68116843EAA3
:020000040801F1
:1000000000027B691B010B4403F5C6731A607B6811
:1000100003331B781A067B6802331B781B041A43D0
:100020007B6801331B781B0213437A6812781046F1
:10003000FA68116843EA00027B691B010B4403F56F
:10004000C4731A60FB681A687B6918331B01134478
:100050001B68FA68116843F001027B6918331B01C1
:100060000B441A6000230EE0FB685B6A43F4001245
:10007000FB685A62012306E0FB685B6A43F4802256
:10008000FB685A62012318462437BD4680BC70477E
:1000900080B485B000AF78600023FB607B6893F884
:1000A0002030FB72FB7A012B02D0FB7A022B1DD190
:1000B0007B681B689B6803F08063002B02D0FB68A1
:1000C0000133FB607B681B689B6803F00063002BB7
:1000D00002D0FB680133FB607B681B689B6803F000
:1000E0008053002B02D0FB680133FB60FB6818468D
:1000F0001437BD4680BC704780B487B000AFF8604D
:10010000B9607A603B60FB6893F82030FB75FB7D3B
:10011000012B03D0FB7D022B40F00381BB68002B39
:100120000ED1FB681B68DB6803F00303002B16D1BC
:10013000FB685B6A43F40012FB685A620123F7E034
:10014000FB681B681B6903F00303002B07D1FB68E6
:100150005B6A43F40012FB685A620123E8E0FB6823
:100160001A68BB681B331B0113441B6803F00402AD
:100170007B689A607B689B68002B0CD1FB681A68CF
:10018000BB681B331B0113441B685B0DC3F30A02DE
:100190007B681A600BE0FB681A68BB681B331B01A5
:1001A00013441B68DB0823F060427B685A60FB68DD
:1001B0001A68BB681B331B0113441B6803F002025F
:1001C0007B68DA60FB681A68BB681B331B01134449
:1001D00004331B6803F00803002B03D07B6808225C
:1001E0001A610BE0FB681A68BB681B331B011344E0
:1001F00004331B6803F00F027B681A61FB681A68FE
:10020000BB681B331B01134404331B681B0ADAB29F
:100210007B689A61FB681A68BB681B331B01134437
:1002200004331B681B0C9AB27B685A61FB681A681E
:10023000BB681B01134403F5DC731B68DAB23B682F
:100240001A70FB681A68BB681B01134403F5DC7362
:100250001B681A0A3B680133D2B21A70FB681A682D
:10026000BB681B01134403F5DC731B681A0C3B6865
:100270000233D2B21A70FB681A68BB681B011344C0
:1002800003F5DC731B681A0E3B680333D2B21A7095
:10029000FB681A68BB681B01134403F5DE731A6818
:1002A0003B680433D2B21A70FB681A68BB681B0142
:1002B000134403F5DE731B681A0A3B680533D2B298
:1002C0001A70FB681A68BB681B01134403F5DE73E0
:1002D0001B681A0C3B680633D2B21A70FB681A68A6
:1002E000BB681B01134403F5DE731B681A0E3B68E1
:1002F0000733D2B21A70BB68002B08D1FB681B68A9
:10030000DA68FB681B6842F02002DA6007E0FB68ED
:100310001B681A69FB681B6842F020021A610023FF
:1003200006E0FB685B6A43F48022FB685A620123A3
:1003300018461C37BD4680BC704780B485B000AFFE
:10034000786039607B6893F82030FB73FB7B012B6E
:1003500002D0FB7B022B09D17B681B6859697B6843
:100360001B683A680A435A61002306E07B685B6AAF
:1003700043F480227B685A62012318461437BD4635
:1003800080BC704780B58AB000AF786000237B6284
:100390007B681B685B693B627B681B685B68FB6111
:1003A0007B681B689B68BB617B681B68DB687B6143
:1003B0007B681B681B693B617B681B689B69FB60F2
:1003C0003B6A03F00103002B7CD0BB6903F00103FF
:1003D000002B23D07B681B6801229A60BB6903F065
:1003E0000203002B03D0786800F083F916E0BB69A4
:1003F00003F00403002B04D07B6A43F400637B62A8
:100400000CE0BB6903F00803002B04D07B6A43F4C3
:1004100080537B6202E0786800F086F9BB6903F4E0
:100420008073002B24D07B681B684FF480729A6025
:10043000BB6903F40073002B03D0786800F062F905
:1004400016E0BB6903F48063002B04D07B6A43F49D
:1004500000537B620CE0BB6903F40063002B04D003
:100460007B6A43F480437B6202E0786800F065F9C0
:10047000BB6903F48033002B24D07B681B684FF4E6
:1004800080329A60BB6903F40033002B03D0786894
:1004900000F041F916E0BB6903F48023002B04D07F
:1004A0007B6A43F400437B620CE0BB6903F40023E6
:1004B000002B04D07B6A43F480337B6202E07868CF
:1004C00000F044F93B6A03F00803002B0CD07B6971
:1004D00003F01003002B07D07B6A43F400737B62A8
:1004E0007B681B681022DA603B6A03F00403002B70
:1004F0000BD07B6903F00803002B06D07B681B68D8
:100500000822DA60786800F033F93B6A03F00203EE
:10051000002B09D07B681B68DB6803F00303002B0A
:1005200002D0786800F01BF93B6A03F04003002B0F
:100530000CD03B6903F01003002B07D07B6A43F417
:1005400080637B627B681B6810221A613B6A03F040
:100550002003002B0BD03B6903F00803002B06D0CF
:100560007B681B6808221A61786800F00AF93B6A08
:1005700003F01003002B09D07B681B681B6903F094
:100580000303002B02D07868FAF7DCFE3B6A03F421
:100590000033002B0BD0FB6903F01003002B06D0B7
:1005A0007B681B6810225A60786800F0F3F83B6A99
:1005B00003F48033002B0BD0FB6903F00803002BFE
:1005C00006D07B681B6808225A60786800F0EBF858
:1005D0003B6A03F40043002B7BD0FB6903F0040368
:1005E000002B72D03B6A03F48073002B08D0FB68A9
:1005F00003F00103002B03D07B6A43F001037B620D
:100600003B6A03F40073002B08D0FB6803F002037D
:10061000002B03D07B6A43F002037B623B6A03F446
:100620008063002B08D0FB6803F00403002B03D089
:100630007B6A43F004037B623B6A03F40063002B94
:1006400043D0FB6803F07003002B3ED0FB6803F03F
:100650007003602B2BD0602B2ED8502B22D0502B28
:100660002AD8402B19D0402B26D8302B10D0302B35
:1006700022D8102B02D0202B05D01DE07B6A43F03E
:1006800008037B6219E07B6A43F010037B6214E08D
:100690007B6A43F020037B620FE07B6A43F04003F8
:1006A0007B620AE07B6A43F080037B6205E07B6A41
:1006B00043F480737B6200E000BF7B681B689A692B
:1006C0007B681B6822F070029A617B681B680422B9
:1006D0005A607B6A002B08D07B685A6A7B6A1A438F
:1006E0007B685A62786800F067F800BF2837BD461B
:1006F00080BD80B483B000AF786000BF0C37BD46CA
:1007000080BC704780B483B000AF786000BF0C3706
:10071000BD4680BC704780B483B000AF786000BF36
:100720000C37BD4680BC704780B483B000AF7860A2
:1007300000BF0C37BD4680BC704780B483B000AFAB
:10074000786000BF0C37BD4680BC704780B483B072
:1007500000AF786000BF0C37BD4680BC704780B4E6
:1007600083B000AF786000BF0C37BD4680BC7047D7
:1007700080B483B000AF786000BF0C37BD4680BC4A
:10078000704780B483B000AF786000BF0C37BD46BF
:1007900080BC704780B483B000AF786000BF0C3776
:1007A000BD4680BC704780B483B000AF786000BFA6
:1007B0000C37BD4680BC704780B483B000AF786012
:1007C00000BF0C37BD4680BC7047000080B485B0C8
:1007D00000AF78607B6803F00703FB600C4BDB68BD
:1007E000BB60BA684FF6FF031340BB60FB681A0298
:1007F000BB68134343F0BF6343F40033BB60044A58
:10080000BB68D36000BF1437BD4680BC704700BFD3
:1008100000ED00E080B400AF044BDB681B0A03F07E
:1008200007031846BD4680BC704700BF00ED00E0DE
:1008300080B483B000AF0346FB7197F90730002BFB
:100840000BDBFB7903F01F02064997F907305B09C0
:10085000012000FA02F241F8232000BF0C37BD4608
:1008600080BC704700E100E080B483B000AF034675
:100870003960FB7197F90730002B0ADB3B68DAB26D
:100880000C4997F907301201D2B20B4483F80023C8
:100890000AE03B68DAB20849FB7903F00F03043B36
:1008A0001201D2B20B441A7600BF0C37BD4680BC91
:1008B000704700BF00E100E000ED00E080B489B0C7
:1008C00000AFF860B9607A60FB6803F00703FB6172
:1008D000FB69C3F10703042B28BF0423BB61FB6939
:1008E0000433062B02D9FB69033B00E000237B6144
:1008F0004FF0FF32BB6902FA03F3DA43BB681A40D8
:100900007B699A404FF0FF317B6901FA03F3D943C9
:100910007B680B40134318462437BD4680BC7047A4
:1009200080B582B000AF78607B68013BB3F1807F17
:1009300001D301230FE00A4A7B68013B53600F217A
:100940004FF0FF30FFF790FF054B00229A60044BF9
:1009500007221A60002318460837BD4680BD00BF35
:1009600010E000E080B582B000AF78607868FFF7F3
:100970002DFF00BF0837BD4680BD80B586B000AFF3
:100980000346B9607A60FB7300237B61FFF742FF87
:1009900078617A68B9687869FFF790FF024697F93D
:1009A0000F3011461846FFF75FFF00BF1837BD46EE
:1009B00080BD80B582B000AF0346FB7197F9073068
:1009C0001846FFF735FF00BF0837BD4680BD80B52C
:1009D00082B000AF78607868FFF7A2FF0346184640
:1009E0000837BD4680BD80B582B000AF78607B68B7
:1009F000002B01D101230EE07B685B79DBB2002B79
:100A000005D17B6800221A717868F9F7A9FC7B6828
:100A100001225A71002318460837BD4680BD0000E8
:100A200080B485B000AF78600023FB607B68002B4A
:100A300001D1012359E07B681B681A462D4B9A426D
:100A40000FD87B681B681A462B4B13442B4AA2FB1A
:100A500003231B099A007B681A647B68284ADA63BF
:100A60000EE07B681B681A46264B1344234AA2FB00
:100A700003231B099A007B681A647B68224ADA63A5
:100A80007B68022283F821207B681B681B68FB605F
:100A9000FB6823F47F5323F03003FB607B685A68C4
:100AA0007B689B681A437B68DB681A437B681B6919
:100AB0001A437B685B691A437B689B691A437B68AE
:100AC000DB691343FA681343FB607B681B68FA68B1
:100AD0001A607B6800229A637B68012283F82120D8
:100AE0007B68002283F82020002318461437BD4677
:100AF00080BC704707040240F8FFFDBFCDCCCCCCD2
:100B000000000240F8FBFDBF0004024080B586B043
:100B100000AFF860B9607A603B600023FB75FB684A
:100B200093F82030012B01D102234BE0FB68012216
:100B300083F82020FB6893F82130DBB2012B3AD1F7
:100B4000FB68022283F82120FB6800229A63FB687D
:100B50001B681A68FB681B6822F001021A603B6878
:100B60007A68B968F86800F0BCFBFB68DB6A002BA8
:100B700008D0FB681B681A68FB681B6842F00E020D
:100B80001A600FE0FB681B681A68FB681B6822F09C
:100B900004021A60FB681B681A68FB681B6842F055
:100BA0000A021A60FB681B681A68FB681B6842F03F
:100BB00001021A6005E0FB68002283F8202002236E
:100BC000FB75FB7D18461837BD4680BD80B485B0E7
:100BD00000AF78600023FB737B6893F82130DBB2B1
:100BE000022B08D07B6804229A637B68002283F87A
:100BF0002020012320E07B681B681A687B681B6843
:100C000022F00E021A607B681B681A687B681B68FA
:100C100022F001021A607B681A6C7B68DB6B012191
:100C200001FA02F25A607B68012283F821207B6876
:100C3000002283F82020FB7B18461437BD4680BC79
:100C40007047000080B584B000AF78600023FB736C
:100C50007B6893F82130DBB2022B05D07B6804223D
:100C60009A630123FB73D6E07B681B681A687B6874
:100C70001B6822F00E021A607B681B681A687B688A
:100C80001B6822F001021A607B681B681A46644BDD
:100C90009A4258D97B681B68624A93424FD07B685E
:100CA0001B68614A934248D07B681B685F4A934245
:100CB00040D07B681B685E4A934238D07B681B68D3
:100CC0005C4A934230D07B681B685B4A934228D0D1
:100CD0007B681B68524A934220D07B681B68574A46
:100CE000934219D07B681B68554A934212D07B68A7
:100CF0001B68544A93420AD07B681B68524A93424D
:100D000002D14FF480531BE04FF4803318E04FF4CE
:100D1000807315E0102313E0012311E04FF080737E
:100D20000EE04FF480130BE04FF4803308E04FF4F3
:100D3000805305E04FF4807302E0102300E00123AC
:100D4000424A536057E07B681B68364A93424FD053
:100D50007B681B68344A934248D07B681B68334ADF
:100D6000934240D07B681B68314A934238D07B68FD
:100D70001B68304A934230D07B681B682E4A9342EE
:100D800028D07B681B68264A934220D07B681B686A
:100D90002A4A934219D07B681B68294A934212D091
:100DA0007B681B68274A93420AD07B681B68264AE7
:100DB000934202D14FF480531BE04FF4803318E08C
:100DC0004FF4807315E0102313E0012311E04FF07E
:100DD00080730EE04FF480130BE04FF4803308E093
:100DE0004FF4805305E04FF4807302E0102300E0DD
:100DF0000123174A53607B68012283F821207B6816
:100E0000002283F820207B685B6B002B03D07B687B
:100E10005B6B78689847FB7B18461037BD4680BDF2
:100E200080000240080002401C00024030000240E6
:100E300044000240580002406C0002400804024096
:100E40001C040240300402404404024000040240FA
:100E50000000024080B584B000AF78607B68DB6B37
:100E60001B68FB607B681B681B68BB607B681B6C36
:100E700004229A40FB681340002B00F0F180BB680D
:100E800003F00403002B00F0EB807B681B681B68F9
:100E900003F02003002B07D17B681B681A687B686E
:100EA0001B6822F004021A607B681B681A465F4BBD
:100EB0009A4258D97B681B685D4A93424FD07B6841
:100EC0001B685C4A934248D07B681B685A4A93422D
:100ED00040D07B681B68594A934238D07B681B68B6
:100EE000574A934230D07B681B68564A934228D0B9
:100EF0007B681B684D4A934220D07B681B68524A2E
:100F0000934219D07B681B68504A934212D07B6889
:100F10001B684F4A93420AD07B681B684D4A934234
:100F200002D14FF480431BE04FF4802318E04FF4CC
:100F3000806315E0402313E0042311E04FF0806349
:100F40000EE04FF480030BE04FF4802308E04FF4F1
:100F5000804305E04FF4806302E0402300E0042377
:100F60003D4A536057E07B681B68314A93424FD03B
:100F70007B681B682F4A934248D07B681B682E4AC7
:100F8000934240D07B681B682C4A934238D07B68E0
:100F90001B682B4A934230D07B681B68294A9342D6
:100FA00028D07B681B68214A934220D07B681B684D
:100FB000254A934219D07B681B68244A934212D079
:100FC0007B681B68224A93420AD07B681B68214ACF
:100FD000934202D14FF480431BE04FF4802318E08A
:100FE0004FF4806315E0402313E0042311E04FF039
:100FF00080630EE04FF480030BE04FF4802308E0A1
:101000004FF4804305E04FF4806302E0402300E0AA
:101010000423124A53607B68DB6A002B00F03681A0
:101020007B68DB6A7868984730E100BF8000024047
:10103000080002401C000240300002404400024010
:10104000580002406C000240080402401C040240A8
:101050003004024044040240000402400000024008
:101060007B681B6C02229A40FB681340002B00F047
:10107000DD80BB6803F00203002B00F0D7807B68A3
:101080001B681B6803F02003002B0BD17B681B68D7
:101090001A687B681B6822F00A021A607B680122CA
:1010A00083F821207B681B681A467B4B9A4258D9EB
:1010B0007B681B68794A93424FD07B681B68784AEB
:1010C000934248D07B681B68764A934240D07B6845
:1010D0001B68754A934238D07B681B68734A9342F9
:1010E00030D07B681B68724A934228D07B681B68AB
:1010F000694A934220D07B681B686E4A934219D09C
:101100007B681B686C4A934212D07B681B686B4AF1
:1011100093420AD07B681B68694A934202D14FF41C
:1011200000531BE04FF4003318E04FF4007315E058
:10113000202313E0022311E04FF000730EE04FF480
:1011400000130BE04FF4003308E04FF4005305E0C8
:101150004FF4007302E0202300E00223594A536059
:1011600057E07B681B684D4A93424FD07B681B68F1
:101170004B4A934248D07B681B684A4A934240D00E
:101180007B681B68484A934238D07B681B68474A93
:10119000934230D07B681B68454A934228D07B68D5
:1011A0001B683D4A934220D07B681B68414A9342AA
:1011B00019D07B681B68404A934212D07B681B6839
:1011C0003E4A93420AD07B681B683D4A934202D153
:1011D0004FF400531BE04FF4003318E04FF400735A
:1011E00015E0202313E0022311E04FF000730EE01E
:1011F0004FF400130BE04FF4003308E04FF40053BA
:1012000005E04FF4007302E0202300E002232E4AA1
:1012100053607B68002283F820207B689B6A002B48
:1012200034D07B689B6A786898472FE07B681B6C9A
:1012300008229A40FB681340002B28D0BB6803F0BB
:101240000803002B23D07B681B681A687B681B6827
:1012500022F00E021A607B681A6C7B68DB6B01213E
:1012600001FA02F25A607B6801229A637B680122CC
:1012700083F821207B68002283F820207B681B6B89
:10128000002B04D07B681B6B7868984700BF00BFB9
:101290001037BD4680BD00BF8000024008000240FC
:1012A0001C0002403000024044000240580002404E
:1012B0006C000240080402401C040240300402405A
:1012C00044040240000402400000024080B483B0A5
:1012D00000AF78607B689B6B18460C37BD4680BCBE
:1012E000704780B485B000AFF860B9607A603B6049
:1012F000FB681A6CFB68DB6B012101FA02F25A6091
:10130000FB681B683A685A60FB685B68102B08D161
:10131000FB681B687A689A60FB681B68BA68DA60C9
:1013200007E0FB681B68BA689A60FB681B687A680C
:10133000DA6000BF1437BD4680BC704780B48BB004
:1013400000AF7860396000237B6200233B6269E173
:1013500001227B6A02FA03F3FB613B681B68FA69AE
:101360001340BB61BA69FB699A4240F058813B68FF
:101370005B689A4A93425ED0984A934275D8984ADD
:10138000934258D0964A93426FD8964A934252D08D
:10139000944A934269D8944A93424CD0924A9342D9
:1013A00063D8924A934246D0904A93425DD8122B1A
:1013B0002AD8122B59D801A252F823F03714010869
:1013C0001114010823140108651401086B140108A5
:1013D0006B1401086B1401086B1401086B140108ED
:1013E0006B1401086B1401086B1401086B140108DD
:1013F0006B1401086B1401086B1401086B140108CD
:10140000191401082D140108794A934213D02CE0D5
:101410003B68DB683B6229E03B68DB6804333B6286
:1014200024E03B68DB6808333B621FE03B68DB6815
:101430000C333B621AE03B689B68002B02D104230B
:101440003B6213E03B689B68012B05D108233B629C
:101450007B68FA691A6109E008233B627B68FA69D4
:101460005A6103E000233B6200E000BFBB69FF2B31
:1014700001D87B6801E07B6804337B61BB69FF2B8B
:1014800002D87B6A9B0002E07B6A083B9B003B61C1
:101490007B691A680F213B6901FA03F3DB431A40A9
:1014A000396A3B6901FA03F31A437B691A603B68A6
:1014B0005B6803F08053002B00F0B1804D4B9B69BB
:1014C0004C4A43F0010393614A4B9B6903F00103CB
:1014D000BB60BB68484A7B6A9B08023352F82330E2
:1014E000FB607B6A03F003039B000F2202FA03F305
:1014F000DB43FA681340FB607B68404A934213D099
:101500007B683F4A93420DD07B683E4A934207D0A6
:101510007B683D4A934201D1032306E0042304E0A3
:10152000022302E0012300E000237A6A02F00302B2
:1015300092009340FA681343FB602F497B6A9B0833
:101540000233FA6841F823203B685B6803F4801398
:10155000002B06D02D4B9A682C49BB6913438B6036
:1015600006E02A4B9A68BB69DB43284913408B602D
:101570003B685B6803F40013002B06D0234BDA684A
:101580002249BB691343CB6006E0204BDA68BB6994
:10159000DB431E491340CB603B685B6803F40033B8
:1015A000002B06D0194B5A681849BB6913434B608E
:1015B00006E0164B5A68BB69DB43144913404B6085
:1015C0003B685B6803F48033002B21D00F4B1A6813
:1015D0000E49BB6913430B6021E000BF00003210CD
:1015E0000000311000002210000021100000121035
:1015F00000001110001002400000014000080140EE
:10160000000C0140001001400014014000040140A2
:101610000B4B1A68BB69DB43094913400B607B6ABB
:1016200001337B623B681A687B6A22FA03F3002B62
:101630007FF48EAE00BF00BF2C37BD4680BC704724
:101640000004014080B485B000AF78600B467B8019
:101650007B689A687B881340002B02D00123FB73C0
:1016600001E00023FB73FB7B18461437BD4680BCAA
:10167000704780B483B000AF78600B467B80134620
:101680007B707B78002B03D07A887B681A6103E03B
:101690007B881A047B681A6100BF0C37BD4680BC8A
:1016A0007047000080B400AF034B01221A6000BFF6
:1016B000BD4680BC704700BF20000E4280B582B09E
:1016C00000AFFDF73FFC7860604B1B685F4A43F05A
:1016D0000103136008E0FDF735FC02467B68D31A6E
:1016E000022B01D90323ACE0584B1B6803F0020323
:1016F000002BF0D0554B1B6823F0F803534A43F0FE
:1017000080031360FDF71EFC7860504B00225A6086
:101710000AE0FDF717FC02467B68D31A41F28832D3
:10172000934201D903238CE0484B5B6803F00C0320
:10173000002BEED1464B474A1A60474B1B681846B0
:10174000FDF7BEFB0346002B01D0012379E0FDF736
:10175000F9FB78603D4B1B683C4A23F080731360B3
:1017600008E0FDF7EFFB02467B68D31A022B01D994
:10177000032366E0354B1B6803F00073002BF0D1A8
:10178000324B00225A60FDF7DDFB78602F4B1B685F
:101790002E4A23F41023136008E0FDF7D3FB024622
:1017A0007B68D31A642B01D903234AE0274B1B68BB
:1017B00003F40033002BF0D1244B1B68234A23F49D
:1017C00080231360FDF7BEFB7860204B1B681F4A27
:1017D00023F08063136008E0FDF7B4FB02467B68EA
:1017E000D31A642B01D903232BE0184B1B6803F099
:1017F0000063002BF0D1FDF7A5FB7860134B1B684D
:10180000124A23F08053136008E0FDF79BFB024669
:101810007B68D31A642B01D9032312E00B4B1B689E
:1018200003F00053002BF0D1084B0022DA62074B83
:101830005B6A064A43F080735362044B00229A604D
:10184000002318460837BD4680BD00BF0010024087
:101850008400002000127A008800002080B586B045
:1018600000AF78607B68002B01D1012304E37B6823
:101870001B6803F00103002B00F08780924B5B682C
:1018800003F00C03042B0CD08F4B5B6803F00C03AC
:10189000082B12D18C4B5B6803F48033B3F5803F87
:1018A0000BD1894B1B6803F40033002B6CD07B6891
:1018B0009B68002B68D10123DEE27B689B68B3F54F
:1018C000803F06D1804B1B687F4A43F4803313600E
:1018D0002EE07B689B68002B0CD17B4B1B687A4AFF
:1018E00023F480331360784B1B68774A23F48023FA
:1018F00013601DE07B689B68B3F5A02F0CD1724B81
:101900001B68714A43F4802313606F4B1B686E4A57
:1019100043F4803313600BE06B4B1B686A4A23F47B
:1019200080331360684B1B68674A23F4802313607D
:101930007B689B68002B13D0FDF704FB386108E03F
:10194000FDF700FB02463B69D31A642B01D9032340
:1019500092E25D4B1B6803F40033002BF0D014E0DF
:10196000FDF7F0FA386108E0FDF7ECFA02463B6952
:10197000D31A642B01D903237EE2534B1B6803F473
:101980000033002BF0D100E000BF7B681B6803F040
:101990000203002B63D04C4B5B6803F00C03002B5D
:1019A0000BD0494B5B6803F00C03082B1CD1464B52
:1019B0005B6803F48033002B16D1434B1B6803F0A4
:1019C0000203002B05D07B685B69012B01D001234A
:1019D00052E23D4B1B6823F0F8027B689B69DB00F9
:1019E000394913430B603AE07B685B69002B20D0D8
:1019F000364B01221A60FDF7A5FA386108E0FDF7C1
:101A0000A1FA02463B69D31A022B01D9032333E220
:101A10002D4B1B6803F00203002BF0D02A4B1B68F0
:101A200023F0F8027B689B69DB00274913430B60B6
:101A300015E0264B00221A60FDF784FA386108E0B1
:101A4000FDF780FA02463B69D31A022B01D9032322
:101A500012E21D4B1B6803F00203002BF0D17B68E0
:101A60001B6803F00803002B3AD07B68DB69002B6E
:101A700019D0174B01221A60FDF764FA386108E0AB
:101A8000FDF760FA02463B69D31A022B01D9032302
:101A9000F2E10D4B5B6A03F00203002BF0D0012052
:101AA00000F0CAFB1CE00A4B00221A60FDF74AFA5C
:101AB00038610FE0FDF746FA02463B69D31A022B64
:101AC00008D90323D8E100BF0010024000004242C1
:101AD000800442429B4B5B6A03F00203002BE9D176
:101AE0007B681B6803F00403002B00F0A680002332
:101AF000FB75944BDB6903F08053002B0DD1914BA8
:101B0000DB69904A43F08053D3618E4BDB6903F06D
:101B10008053BB60BB680123FB758B4B1B6803F4D0
:101B20008073002B18D1884B1B68874A43F480735D
:101B30001360FDF707FA386108E0FDF703FA024683
:101B40003B69D31A642B01D9032395E17E4B1B68B3
:101B500003F48073002BF0D07B681B69012B06D146
:101B6000784B1B6A774A43F0010313622DE07B68D0
:101B70001B69002B0CD1734B1B6A724A23F00103C3
:101B80001362704B1B6A6F4A23F0040313621CE05C
:101B90007B681B69052B0CD16A4B1B6A694A43F0B1
:101BA00004031362674B1B6A664A43F00103136226
:101BB0000BE0644B1B6A634A23F001031362614B21
:101BC0001B6A604A23F0040313627B681B69002BC5
:101BD00015D0FDF7B7F938610AE0FDF7B3F9024611
:101BE0003B69D31A41F28832934201D9032343E17E
:101BF000544B1B6A03F00203002BEED014E0FDF7F8
:101C0000A1F938610AE0FDF79DF902463B69D31A54
:101C100041F28832934201D903232DE1494B1B6ADB
:101C200003F00203002BEED1FB7D012B05D1454BC8
:101C3000DB69444A23F08053D3617B68DB6A002B65
:101C400000F08C803F4B5B6803F48033B3F5803F3A
:101C50000ED13C4B5B6803F00C03082B08D1394BC9
:101C6000DB6A03F48033B3F5803F01D1012303E144
:101C70007B68DB6A022B4ED1324B1B6803F080532A
:101C8000002B09D02F4BDB6A03F0F0027B685B6B03
:101C90009A4201D00123EFE02C4B00221A60FDF79D
:101CA00051F9386108E0FDF74DF902463B69D31A56
:101CB000642B01D90323DFE0224B1B6803F0006390
:101CC000002BF0D11F4BDB6A23F0F0027B685B6BCB
:101CD0001C491343CB621B4BDB6A23F470627B68A5
:101CE0001B6B18491343CB62184B01221A60FDF796
:101CF00029F9386108E0FDF725F902463B69D31A56
:101D0000642B01D90323B7E00E4B1B6803F000637B
:101D1000002BF0D022E00B4BDB6A0A4A23F480331D
:101D2000D3620A4B00221A60FDF70CF938610FE00C
:101D3000FDF708F902463B69D31A642B08D903233F
:101D40009AE000BF0010024000700040680042426C
:101D50004B4B1B6803F00063002BE9D17B681B6AC7
:101D6000002B00F08880464B5B6803F00C03082BC7
:101D700068D07B681B6A022B4DD1424B00221A604F
:101D8000FDF7E0F8386108E0FDF7DCF802463B6952
:101D9000D31A022B01D903236EE0394B1B6803F0E1
:101DA0000073002BF0D17B685B6AB3F5803F0FD1E5
:101DB000334BDA6A7B685B6831491343CB62304B43
:101DC000DB6A23F00F027B68DB682D491343CB628B
:101DD0002B4B5B6823F474127B68596A7B689B6A9F
:101DE0000B43274913434B60264B01221A60FDF732
:101DF000A9F8386108E0FDF7A5F802463B69D31A57
:101E0000022B01D9032337E01D4B1B6803F000733D
:101E1000002BF0D02FE01B4B00221A60FDF792F848
:101E2000386108E0FDF78EF802463B69D31A022BB1
:101E300001D9032320E0124B1B6803F00073002B31
:101E4000F0D118E07B681B6A012B01D1012313E05C
:101E50000B4B5B68FB60FB6803F480327B685B6A5A
:101E60009A4206D1FB6803F470127B689B6A9A421F
:101E700001D0012300E0002318461837BD4680BD7D
:101E8000001002406000424280B584B000AF78602C
:101E900039607B68002B01D10123D0E06A4B1B68BD
:101EA00003F007033A689A4210D9674B1B6823F086
:101EB000070265493B6813430B60634B1B6803F0E3
:101EC00007033A689A4201D00123B8E07B681B6897
:101ED00003F00203002B20D07B681B6803F004038F
:101EE000002B05D0594B5B68584A43F4E0635360BC
:101EF0007B681B6803F00803002B05D0534B5B681D
:101F0000524A43F460535360504B5B6823F0F00235
:101F10007B689B684D4913434B607B681B6803F0EB
:101F20000103002B40D07B685B68012B07D1474B36
:101F30001B6803F40033002B15D101237FE07B687D
:101F40005B68022B07D1414B1B6803F00073002B29
:101F500009D1012373E03D4B1B6803F00203002B02
:101F600001D101236BE0394B5B6823F003027B68EE
:101F70005B68364913434B60FCF7E4FFF8600AE006
:101F8000FCF7E0FF0246FB68D31A41F28832934225
:101F900001D9032353E02D4B5B6803F00C027B68EF
:101FA0005B689B009A42EBD1274B1B6803F0070349
:101FB0003A689A4210D2244B1B6823F00702224948
:101FC0003B6813430B60204B1B6803F007033A6820
:101FD0009A4201D0012332E07B681B6803F00403BE
:101FE000002B08D0194B5B6823F4E0627B68DB6848
:101FF000164913434B607B681B6803F00803002BF2
:1020000009D0124B5B6823F460527B681B69DB00CC
:102010000E4913434B6000F021F802460B4B5B68FE
:102020001B0903F00F030A49CB5C22FA03F3094AA8
:102030001360094B1B681846FCF742FF0023184643
:102040001037BD4680BD00BF002002400010024096
:102050001C86010884000020880000202DE9B04F74
:102060008EB000AF0023FB620023BB6200237B63C2
:1020700000237B6200233B6300233B620023FB6160
:102080004E4B5B68FB62FB6A03F00C03042B02D02F
:10209000082B03D089E04A4B3B6389E0FB6A9B0C29
:1020A00003F00F02474B9B5C7B62FB6A03F48033B7
:1020B000002B72D0414BDB6A03F00F02424B9B5C5A
:1020C000BB623E4BDB6A03F48033002B53D03B4BA7
:1020D000DB6A1B0903F00F0301333B62374BDB6AFA
:1020E0001B0A03F00F030233FB61FB6900229A46CF
:1020F00093467B6A00223B617A613B6903FB0BF2EA
:102100007B690AFB03F313443A69AAFB02010B44FF
:1021100019462B4B03FB01F2002300FB03F313448E
:10212000274AA0FB02452B441D463B6A0022BB60A8
:10213000FA60BB6A00223B607A60D7E902010B4675
:10214000D7E900AB524602FB03F25B4684460CFB28
:1021500003F3134402465146A2FB01894B449946BE
:1021600042464B4620462946F7F744F802460B46BE
:1021700013467B6307E07B6A114A03FB02F2BB6AEA
:10218000B2FBF3F37B630F4B5B7B1A467B6A934294
:1021900008D17B6B5B087B6304E07B6A0B4A02FB24
:1021A00003F37B637B6B3B6302E0094B3B6300BF44
:1021B0003B6B18463837BD46BDE8B08F0010024073
:1021C00040787D01348601084486010800093D00FD
:1021D00000127A0080B400AF024B1B681846BD465F
:1021E00080BC70478400002080B500AFFFF7F2FF8D
:1021F0000246054B5B681B0A03F007030349CB5CEF
:1022000022FA03F3184680BD001002402C86010814
:1022100080B500AFFFF7DEFF0246054B5B68DB0AC7
:1022200003F007030349CB5C22FA03F3184680BD91
:10223000001002402C86010880B485B000AF7860A1
:102240000A4B1B680A4AA2FB03235B0A7A6802FB5B
:1022500003F3FB6000BFFB685A1EFA60002BF9D144
:1022600000BF00BF1437BD4680BC7047840000200B
:10227000D34D621080B588B000AF786000237B61D9
:1022800000233B610023FB617B681B6803F00103B3
:10229000002B7DD00023FB768B4BDB6903F0805352
:1022A000002B0DD1884BDB69874A43F08053D36103
:1022B000854BDB6903F08053FB60FB680123FB76F1
:1022C000824B1B6803F48073002B18D17F4B1B6873
:1022D0007E4A43F480731360FCF734FE786108E0B3
:1022E000FCF730FE02467B69D31A642B01D9032325
:1022F000E5E0764B1B6803F48073002BF0D0724B43
:102300001B6A03F440733B613B69002B2ED07B6852
:102310005B6803F440733A699A4227D06A4B1B6AA0
:1023200023F440733B616A4B01221A60684B002220
:102330001A60654A3B6913623B6903F00103002B95
:1023400014D0FCF7FFFD78610AE0FCF7FBFD0246C4
:102350007B69D31A41F28832934201D90323AEE05C
:10236000594B1B6A03F00203002BEED0564B1B6A3D
:1023700023F440727B685B68534913430B62FB7E16
:10238000012B05D1504BDB694F4A23F08053D361B9
:102390007B681B6803F00203002B08D04A4B5B6884
:1023A00023F440427B689B68474913434B607B683A
:1023B0001B6803F00403002B08D0434BDB6A23F4B3
:1023C00000327B68DB6840491343CB627B681B6843
:1023D00003F00803002B08D03B4BDB6A23F4802278
:1023E0007B681B6938491343CB62374BDB6A03F4C4
:1023F0000033002B05D1344BDB6A03F48023002B20
:1024000001D00123FB61FB69012B48D12E4B1B68D6
:1024100003F08053002B38D12B4B1B6803F08063F3
:10242000002B09D0284BDB6A03F0F0027B689B6924
:102430009A4201D0012342E0234BDB6A23F0F002F1
:102440007B689B6920491343CB621F4BDB6A23F4F3
:1024500070427B685B691C491343CB621D4B0122B0
:102460001A60FCF76FFD786108E0FCF76BFD02462F
:102470007B69D31A642B01D9032320E0124B1B681C
:1024800003F00053002BF0D009E00F4BDB6A03F49C
:1024900070427B685B699A4201D001230FE07B6840
:1024A0001B6803F01003002B08D0074B5B6823F474
:1024B00080027B68DB69044913434B6000231846A4
:1024C0002037BD4680BD00BF0010024000700040B4
:1024D000400442427000424280B58AB000AF78604A
:1024E0000023FB6100237B620023BB6100237B612F
:1024F00000233B610023FB600023BB6000233B62A1
:102500007B68013B0F2B00F21D8101A252F823F0E2
:10251000C5260108292701084527010823260108A7
:1025200045270108452701084527010875260108A8
:1025300045270108452701084527010845270108C7
:1025400045270108452701084527010851250108AD
:10255000834B5B68BB60824B1B6803F08073002B6E
:1025600000F0F280BB689B0C03F00F037D4AD35C44
:10257000BB61BB6803F48033002B3BD0784BDB6A34
:1025800003F00F03784AD35CFB61754BDB6A03F4FD
:102590008033002B1CD0724BDB6A1B0903F00F0346
:1025A0000133FB606E4BDB6A1B0A03F00F0302333F
:1025B0007B616E4AFB68B2FBF3F37A6903FB02F2BC
:1025C000FB69B2FBF3F2BB6902FB03F37B6207E03A
:1025D000664AFB69B2FBF3F2BB6902FB03F37B6261
:1025E000604B5B7B1A46BB69934208D17B6A5B08F0
:1025F0007B6204E0BB695E4A02FB03F37B62584BDB
:102600005B6803F48003B3F5800F02D17B6A3B6201
:102610009AE07B6A5B00574AA2FB03235B083B629C
:1026200092E04F4BDB6A03F40033002B03D1FFF73A
:1026300015FD38628AE04A4B1B6803F08053002B7B
:1026400000F08480464BDB6A1B0903F00F03013363
:10265000FB60434BDB6A1B0B03F00F0302333B6150
:10266000424AFB68B2FBF3F33A6902FB03F35B00F7
:102670003B626BE03A4BDB6A03F48023002B03D10F
:10268000FFF7ECFC386263E0354B1B6803F08053C6
:10269000002B5DD0324BDB6A1B0903F00F030133C3
:1026A000FB602F4BDB6A1B0B03F00F0302333B6114
:1026B0002E4AFB68B2FBF3F33A6902FB03F35B00BB
:1026C0003B6245E0264B1B6ABB60BB6803F440736A
:1026D000B3F5807F08D1BB6803F00203002B03D061
:1026E0004FF400433B621EE0BB6803F44073B3F554
:1026F000007F09D11A4B5B6A03F00203002B03D061
:1027000049F640433B620EE0BB6803F44073B3F507
:10271000407F1FD1124B1B6803F40033002B19D0EC
:10272000154B3B6216E015E0FFF772FD02460C4BBD
:102730005B689B0B03F0030301335B00B2FBF3F315
:102740003B6208E000BF06E000BF04E000BF02E01B
:1027500000BF00E000BF3B6A18462837BD4680BD79
:1027600000100240548601086486010840787D010B
:1027700000093D00ABAAAAAAF0FA020080B584B015
:1027800000AF78600023FB607B68002B01D1012340
:102790007AE07B685B7CDBB2002B05D17B68002292
:1027A0001A747868F9F7D0FF7B6802225A74786847
:1027B00000F070F80346002B04D07B6804225A74A2
:1027C000012361E0786800F092F80346002B04D002
:1027D0007B6804225A74012356E07B681B685A68A0
:1027E0007B681B6822F007025A607B689B68002B9D
:1027F00005D0274B1B6B264A23F001031363244BA0
:10280000DB6A23F460727B689B6821491343CB62C7
:102810007B685B68B3F1FF3F03D07B685B68FB605C
:102820000EE00120FFF758FEF860FB68002B04D192
:102830007B6804225A74012326E0FB68013BFB609D
:10284000FB681A0C7B681B6802F00F029A607B68B9
:102850001B68FA6892B2DA60786800F070F8034694
:10286000002B04D07B6804225A7401230CE07B689F
:102870000022DA737B6801225A737B6801229A7303
:102880007B6801225A74002318461037BD4680BD6C
:10289000006C004080B584B000AF78600023FB601E
:1028A0007B68002B01D101231DE07B681B685A68FF
:1028B0007B681B6822F008025A60FCF743FBF86053
:1028C00009E0FCF73FFB0246FB68D31AB3F57A7FB9
:1028D00001D9032307E07B681B685B6803F00803EA
:1028E000002BEED0002318461037BD4680BD80B5C2
:1028F00084B000AF78600023FB60FCF723FBF86036
:1029000009E0FCF71FFB0246FB68D31AB3F57A7F98
:1029100001D903230FE07B681B685B6803F0200389
:10292000002BEED07B681B685A687B681B6842F0FE
:1029300010025A60002318461037BD4680BD80B58E
:1029400084B000AF78600023FB607B681B685A6826
:102950007B681B6822F010025A60FCF7F3FAF860FB
:1029600009E0FCF7EFFA0246FB68D31AB3F57A7F69
:1029700001D9032307E07B681B685B6803F0200331
:10298000002BEED0002318461037BD4680BD80B521
:1029900082B000AF78607B68002B01D1012341E059
:1029A0007B6893F83D30DBB2002B06D17B680022B8
:1029B00083F83C207868FBF701FF7B68022283F8EC
:1029C0003D207B681A687B6804331946104600F086
:1029D00033FD7B68012283F846207B68012283F85F
:1029E0003E207B68012283F83F207B68012283F828
:1029F00040207B68012283F841207B68012283F814
:102A000042207B68012283F843207B68012283F8FF
:102A100044207B68012283F845207B68012283F8EB
:102A20003D20002318460837BD4680BD80B582B0E2
:102A300000AF78607B68002B01D1012341E07B6807
:102A400093F83D30DBB2002B06D17B68002283F87F
:102A50003C20786800F039F87B68022283F83D203A
:102A60007B681A687B6804331946104600F0E4FC62
:102A70007B68012283F846207B68012283F83E2090
:102A80007B68012283F83F207B68012283F8402085
:102A90007B68012283F841207B68012283F8422071
:102AA0007B68012283F843207B68012283F844205D
:102AB0007B68012283F845207B68012283F83D2052
:102AC000002318460837BD4680BD80B483B000AFF0
:102AD000786000BF0C37BD4680BC704780B584B0BD
:102AE00000AF786039603B68002B09D17B6893F8B0
:102AF0003E30DBB2012B14BF01230023DBB222E006
:102B00003B68042B09D17B6893F83F30DBB2012B83
:102B100014BF01230023DBB215E03B68082B09D169
:102B20007B6893F84030DBB2012B14BF01230023F4
:102B3000DBB208E07B6893F84130DBB2012B14BFB5
:102B400001230023DBB2002B01D0012363E03B68AB
:102B5000002B04D17B68022283F83E2013E03B68FF
:102B6000042B04D17B68022283F83F200BE03B68F2
:102B7000082B04D17B68022283F8402003E07B68A5
:102B8000022283F841207B681B68012239681846BD
:102B900000F0E8FE7B681B68214A934207D17B68FE
:102BA0001B685A6C7B681B6842F400425A647B685D
:102BB0001B681B4A934213D07B681B68B3F1804F9C
:102BC0000ED07B681B68174A934209D07B681B684C
:102BD000154A934204D07B681B68144A934211D172
:102BE0007B681B689B6803F00703FB60FB68062B90
:102BF00010D07B681B681A687B681B6842F0010272
:102C00001A6007E07B681B681A687B681B6842F0E3
:102C100001021A60002318461037BD4680BD00BF70
:102C2000002C01400004004000080040000C00405F
:102C300080B582B000AF78607B68002B01D10123A2
:102C400041E07B6893F83D30DBB2002B06D17B6816
:102C5000002283F83C20786800F039F87B68022273
:102C600083F83D207B681A687B6804331946104658
:102C700000F0E2FB7B68012283F846207B6801229A
:102C800083F83E207B68012283F83F207B68012285
:102C900083F840207B68012283F841207B68012271
:102CA00083F842207B68012283F843207B6801225D
:102CB00083F844207B68012283F845207B68012249
:102CC00083F83D20002318460837BD4680BD80B4F8
:102CD00083B000AF786000BF0C37BD4680BC704742
:102CE00080B584B000AF786039603B68002B09D1B3
:102CF0007B6893F83E30DBB2012B14BF0123002325
:102D0000DBB222E03B68042B09D17B6893F83F30AB
:102D1000DBB2012B14BF01230023DBB215E03B68BB
:102D2000082B09D17B6893F84030DBB2012B14BF2C
:102D300001230023DBB208E07B6893F84130DBB26B
:102D4000012B14BF01230023DBB2002B01D0012390
:102D500063E03B68002B04D17B68022283F83E20AD
:102D600013E03B68042B04D17B68022283F83F20E8
:102D70000BE03B68082B04D17B68022283F84020DB
:102D800003E07B68022283F841207B681B680122F4
:102D90003968184600F0E6FD7B681B68214A9342BB
:102DA00007D17B681B685A6C7B681B6842F4004241
:102DB0005A647B681B681B4A934213D07B681B686C
:102DC000B3F1804F0ED07B681B68174A934209D03D
:102DD0007B681B68154A934204D07B681B68144AC1
:102DE000934211D17B681B689B6803F00703FB606B
:102DF000FB68062B10D07B681B681A687B681B6811
:102E000042F001021A6007E07B681B681A687B6861
:102E10001B6842F001021A60002318461037BD46B5
:102E200080BD00BF002C01400004004000080040AD
:102E3000000C004080B584B000AF78607B681B68F0
:102E4000DB68FB607B681B681B69BB60BB6803F0C9
:102E50000203002B20D0FB6803F00203002B1BD0E1
:102E60007B681B686FF002021A617B6801221A7787
:102E70007B681B689B6903F00303002B03D0786811
:102E800000F0BFFA05E0786800F0B2FA786800F068
:102E9000C1FA7B6800221A77BB6803F00403002B99
:102EA00020D0FB6803F00403002B1BD07B681B6859
:102EB0006FF004021A617B6802221A777B681B6834
:102EC0009B6903F44073002B03D0786800F099FAF3
:102ED00005E0786800F08CFA786800F09BFA7B686F
:102EE00000221A77BB6803F00803002B20D0FB6890
:102EF00003F00803002B1BD07B681B686FF00802EF
:102F00001A617B6804221A777B681B68DB6903F00F
:102F10000303002B03D0786800F073FA05E07868AB
:102F200000F066FA786800F075FA7B6800221A777C
:102F3000BB6803F01003002B20D0FB6803F01003E4
:102F4000002B1BD07B681B686FF010021A617B6836
:102F500008221A777B681B68DB6903F44073002B37
:102F600003D0786800F04DFA05E0786800F040FA88
:102F7000786800F04FFA7B6800221A77BB6803F08C
:102F80000103002B0CD0FB6803F00103002B07D0DA
:102F90007B681B686FF001021A61786800F01FFA05
:102FA000BB6803F08003002B0CD0FB6803F08003A8
:102FB000002B07D07B681B686FF080021A6178686D
:102FC00000F063FDBB6803F04003002B0CD0FB68EE
:102FD00003F04003002B07D07B681B686FF04002B2
:102FE0001A61786800F01FFABB6803F02003002B19
:102FF0000CD0FB6803F02003002B07D07B681B6814
:103000006FF020021A61786800F036FD00BF1037BB
:10301000BD4680BD80B586B000AFF860B9607A600B
:103020000023FB75FB6893F83C30012B01D1022390
:1030300048E0FB68012283F83C207B680C2B39D8E0
:1030400001A252F823F000BF7D300108B53001081D
:10305000B5300108B53001088B300108B5300108E2
:10306000B5300108B530010899300108B5300108C4
:10307000B5300108B5300108A7300108FB681B68AE
:10308000B968184600F050FA17E0FB681B68B96889
:10309000184600F0AFFA10E0FB681B68B9681846E4
:1030A00000F012FB09E0FB681B68B968184600F0E5
:1030B00075FB02E00123FB7500BFFB68002283F86B
:1030C0003C20FB7D18461837BD4680BD80B586B0D4
:1030D00000AFF860B9607A600023FB75FB6893F875
:1030E0003C30012B01D10223AEE0FB68012283F8C2
:1030F0003C207B680C2B00F29F8001A252F823F049
:1031000035310108393201083932010839320108F4
:1031100075310108393201083932010839320108A4
:10312000B731010839320108393201083932010852
:10313000F7310108FB681B68B968184600F0F4F91C
:10314000FB681B689A69FB681B6842F008029A6179
:10315000FB681B689A69FB681B6822F004029A618D
:10316000FB681B689969BB681A69FB681B680A439E
:103170009A6164E0FB681B68B968184600F03AFA87
:10318000FB681B689A69FB681B6842F400629A61DD
:10319000FB681B689A69FB681B6822F480629A616D
:1031A000FB681B689969BB681B691A02FB681B688E
:1031B0000A439A6143E0FB681B68B968184600F04F
:1031C00083FAFB681B68DA69FB681B6842F0080237
:1031D000DA61FB681B68DA69FB681B6822F004028D
:1031E000DA61FB681B68D969BB681A69FB681B68F0
:1031F0000A43DA6123E0FB681B68B968184600F0EF
:10320000CDFAFB681B68DA69FB681B6842F4006250
:10321000DA61FB681B68DA69FB681B6822F480626C
:10322000DA61FB681B68D969BB681B691A02FB6815
:103230001B680A43DA6102E00123FB7500BFFB68EB
:10324000002283F83C20FB7D18461837BD4680BD20
:1032500080B584B000AF786039600023FB737B6871
:1032600093F83C30012B01D10223B4E07B680122AA
:1032700083F83C207B68022283F83D207B681B6832
:103280009B68BB60BB6823F07703BB60BB6823F41B
:103290007F43BB607B681B68BA689A603B681B68A9
:1032A000B3F5005F3ED0B3F5005F00F28780B3F561
:1032B000805F00F08680B3F5805F7FD8702B1AD0D6
:1032C000702B7BD8602B50D0602B77D8502B3CD004
:1032D000502B73D8402B58D0402B6FD8302B64D054
:1032E000302B6BD8202B60D0202B67D8002B5CD0E4
:1032F000102B5AD062E07B6818683B6899683B687D
:103300005A683B68DB6800F00EFB7B681B689B68B3
:10331000BB60BB6843F07703BB607B681B68BA681F
:103320009A604FE07B6818683B6899683B685A6808
:103330003B68DB6800F0F7FA7B681B689A687B687B
:103340001B6842F480429A603CE07B6818683B68E6
:1033500059683B68DB681A4600F06EFA7B681B68A8
:103360005021184600F0C5FA2CE07B6818683B68CD
:1033700059683B68DB681A4600F08CFA7B681B686A
:103380006021184600F0B5FA1CE07B6818683B68BD
:1033900059683B68DB681A4600F04EFA7B681B6888
:1033A0004021184600F0A5FA0CE07B681A683B68DB
:1033B0001B681946104600F09CFA03E00123FB73DA
:1033C00000E000BF7B68012283F83D207B6800227B
:1033D00083F83C20FB7B18461037BD4680BD80B487
:1033E00083B000AF786000BF0C37BD4680BC70472B
:1033F00080B483B000AF786000BF0C37BD4680BC9E
:10340000704780B483B000AF786000BF0C37BD4612
:1034100080BC704780B483B000AF786000BF0C37C9
:10342000BD4680BC704780B483B000AF786000BFF9
:103430000C37BD4680BC704780B485B000AF786063
:1034400039607B681B68FB607B68334A93420FD00E
:103450007B68B3F1804F0BD07B68304A934207D032
:103460007B682F4A934203D07B682E4A934208D14F
:10347000FB6823F07003FB603B685B68FA681343EA
:10348000FB607B68244A93420FD07B68B3F1804F86
:103490000BD07B68214A934207D07B68204A934235
:1034A00003D07B681F4A934208D1FB6823F4407322
:1034B000FB603B68DB68FA681343FB60FB6823F042
:1034C00080023B685B691343FB607B68FA681A60A3
:1034D0003B689A687B68DA623B681A687B689A6224
:1034E0007B680D4A934203D13B681A697B681A6373
:1034F0007B6801225A617B681B6903F00103002B82
:1035000005D07B681B6923F001027B681A6100BF4C
:103510001437BD4680BC7047002C014000040040B9
:1035200000080040000C004080B487B000AF786015
:1035300039607B681B6A7B617B681B6A23F0010230
:103540007B681A627B685B683B617B689B69FB6098
:10355000FB6823F07003FB60FB6823F00303FB6050
:103560003B681B68FA681343FB607B6923F0020326
:103570007B613B689B687A6913437B617B681C4A6B
:1035800093420CD17B6923F008037B613B68DB68C5
:103590007A6913437B617B6923F004037B617B6859
:1035A000134A934211D13B6923F480733B613B6919
:1035B00023F400733B613B685B693A6913433B61E9
:1035C0003B689B693A6913433B617B683A695A607F
:1035D0007B68FA689A613B685A687B685A637B68C3
:1035E0007A691A6200BF1C37BD4680BC704700BFB5
:1035F000002C014080B487B000AF786039607B68F0
:103600001B6A7B617B681B6A23F010027B681A626D
:103610007B685B683B617B689B69FB60FB6823F4AC
:10362000E043FB60FB6823F44073FB603B681B686E
:103630001B02FA681343FB607B6923F020037B6164
:103640003B689B681B017A6913437B617B681D4A59
:1036500093420DD17B6923F080037B613B68DB687B
:103660001B017A6913437B617B6923F040037B6113
:103670007B68144A934213D13B6923F480633B6116
:103680003B6923F400633B613B685B699B003A69DB
:1036900013433B613B689B699B003A6913433B6161
:1036A0007B683A695A607B68FA689A613B685A6835
:1036B0007B689A637B687A691A6200BF1C37BD46D3
:1036C00080BC7047002C014080B487B000AF7860A8
:1036D00039607B681B6A7B617B681B6A23F480729C
:1036E0007B681A627B685B683B617B68DB69FB60B7
:1036F000FB6823F07003FB60FB6823F00303FB60AF
:103700003B681B68FA681343FB607B6923F4007312
:103710007B613B689B681B027A6913437B617B6812
:103720001D4A93420DD17B6923F400637B613B68A2
:10373000DB681B027A6913437B617B6923F4806336
:103740007B617B68144A934213D13B6923F4805315
:103750003B613B6923F400533B613B685B691B01A0
:103760003A6913433B613B689B691B013A69134308
:103770003B617B683A695A607B68FA68DA613B684A
:103780005A687B68DA637B687A691A6200BF1C3703
:10379000BD4680BC704700BF002C014080B487B09C
:1037A00000AF786039607B681B6A3B617B681B6A8D
:1037B00023F480527B681A627B685B687B617B685C
:1037C000DB69FB60FB6823F4E043FB60FB6823F4E8
:1037D0004073FB603B681B681B02FA681343FB6085
:1037E0003B6923F400533B613B689B681B033A69C8
:1037F00013433B617B680F4A934209D17B6923F4F1
:1038000080437B613B685B699B017A6913437B6101
:103810007B687A695A607B68FA68DA613B685A6843
:103820007B681A647B683A691A6200BF1C37BD4620
:1038300080BC7047002C014080B487B000AFF860B6
:10384000B9607A60FB681B6A7B61FB681B6A23F0C6
:103850000102FB681A62FB689B693B613B6923F0CC
:10386000F0033B617B681B013A6913433B617B6951
:1038700023F00A037B617A69BB6813437B61FB68B1
:103880003A699A61FB687A691A6200BF1C37BD46C3
:1038900080BC704780B487B000AFF860B9607A60D0
:1038A000FB681B6A7B61FB681B6A23F01002FB68E4
:1038B0001A62FB689B693B613B6923F470433B617F
:1038C0007B681B033A6913433B617B6923F0A003C8
:1038D0007B61BB681B017A6913437B61FB683A69B2
:1038E0009A61FB687A691A6200BF1C37BD4680BCCA
:1038F000704780B485B000AF786039607B689B68A2
:10390000FB60FB6823F07003FB603A68FB681343BD
:1039100043F00703FB607B68FA689A6000BF1437C6
:10392000BD4680BC704780B487B000AFF860B96016
:103930007A603B60FB689B687B617B6923F47F4313
:103940007B613B681A027B681A43BB6813437A6940
:1039500013437B61FB687A699A6000BF1C37BD46E0
:1039600080BC704780B487B000AFF860B9607A60FF
:10397000BB6803F01F03012202FA03F37B61FB68BB
:103980001A6A7B69DB431A40FB681A62FB681A6A91
:10399000BB6803F01F03796801FA03F31A43FB685D
:1039A0001A6200BF1C37BD4680BC704780B485B02A
:1039B00000AF786039607B6893F83C30012B01D10F
:1039C00002234BE07B68012283F83C207B680222C3
:1039D00083F83D207B681B685B68FB607B681B6825
:1039E0009B68BB60FB6823F07003FB603B681B684F
:1039F000FA681343FB607B681B68FA685A607B684F
:103A00001B68194A934213D07B681B68B3F1804F3F
:103A10000ED07B681B68154A934209D07B681B68EF
:103A2000134A934204D07B681B68124A93420CD11C
:103A3000BB6823F08003BB603B685B68BA681343D4
:103A4000BB607B681B68BA689A607B68012283F858
:103A50003D207B68002283F83C2000231846143761
:103A6000BD4680BC704700BF002C014000040040F0
:103A700000080040000C004080B483B000AF7860C4
:103A800000BF0C37BD4680BC704780B483B000AF28
:103A9000786000BF0C37BD4680BC704780B582B0EF
:103AA00000AF78607B68002B01D1012342E07B6886
:103AB00093F84130DBB2002B06D17B68002283F8FB
:103AC00040207868FAF7C2FF7B68242283F84120FF
:103AD0007B681B68DA687B681B6822F40052DA6036
:103AE000786801F003F97B681B681A697B681B68BA
:103AF00022F490421A617B681B685A697B681B68D4
:103B000022F02A025A617B681B68DA687B681B68AE
:103B100042F40052DA607B6800225A647B682022FB
:103B200083F841207B68202283F842207B680022B2
:103B30005A63002318460837BD4680BD80B58CB057
:103B400000AFF860B9601346FB80FB6893F8413022
:103B5000DBB2202B56D1BB68002B02D0FB88002B98
:103B600001D101234FE0BA68FB681A62FB68FA884A
:103B70009A84FB68FA88DA84FB6800225A64FB683E
:103B8000212283F84120FB689B6B214A9A62FB68E3
:103B90009B6B204ADA62FB689B6B1F4A1A63FB68C7
:103BA0009B6B00225A6307F10803FB62FB68986B6A
:103BB000FB6A1968FB681B6804331A46FB88FCF72C
:103BC000A5FFFB681B686FF040021A60FB681B686A
:103BD0001433BB61BB6953E8003F7B617B6943F0F1
:103BE0008003BB62FB681B681433BA6A7A623B626B
:103BF000396A7A6A41E80023FB61FB69002BE5D151
:103C0000002300E0022318463037BD4680BD00BFC8
:103C100011450108AB4501082F47010880B58CB05C
:103C200000AFF860B9601346FB80FB6893F8423040
:103C3000DBB2202B4AD1BB68002B02D0FB88002BC3
:103C400001D1012343E0FB6801221A63FB680022D3
:103C50005A63FB881A46B968F86800F0B2FD03465B
:103C600087F82F3097F82F30002B2CD1FB681B6B77
:103C7000012B25D100233B61FB681B681B683B615E
:103C8000FB681B685B683B613B69FB681B680C3326
:103C9000BB61BB6953E8003F7B617B6943F0100364
:103CA000BB62FB681B680C33BA6A7A623B62396A92
:103CB0007A6A41E80023FB61FB69002BE5D102E051
:103CC000012387F82F3097F82F3000E002231846A1
:103CD0003037BD4680BD80B58CB000AFF860B960AC
:103CE0001346FB80FB6893F84230DBB2202B46D1B1
:103CF000BB68002B02D0FB88002B01D101233FE0E1
:103D0000FB6801221A63FB6800225A63FB881A468B
:103D1000B968F86800F08EFD034687F82F30FB681D
:103D20001B6B012B25D100233B61FB681B681B68C3
:103D30003B61FB681B685B683B613B69FB681B6818
:103D40000C33BB61BB6953E8003F7B617B6943F087
:103D50001003BB62FB681B680C33BA6A7A623B6271
:103D6000396A7A6A41E80023FB61FB69002BE5D1DF
:103D700002E0012387F82F3097F82F3000E002236C
:103D800018463037BD4680BD80B58EB000AF786034
:103D90007B681B680C333B623B6A53E8003FFB6166
:103DA000FB6923F0C0037B637B681B680C337A6B71
:103DB000FA62BB62B96AFA6A41E800237B627B6AF5
:103DC000002BE5D17B681B685B6903F08003002B47
:103DD00036D07B681B681433FB60FB6853E8003FF8
:103DE000BB60BB6823F080033B637B681B681433B4
:103DF0003A6BBA617B617969BA6941E800233B613A
:103E00003B69002BE5D17B689B6B002B18D07B684E
:103E10009B6B00225A637B689B6B1846FCF7D6FEAF
:103E20000346002B0CD07B689B6B1846FDF74EFABF
:103E30000346202B04D17B6810225A64032307E039
:103E40007B680022DA847B68202283F841200023EB
:103E500018463837BD4680BD80B59AB000AF78604F
:103E60007B681B680C33BB64BB6C53E8003F7B640E
:103E70007B6C23F490737B667B681B680C337A6ED3
:103E80007A653B65396D7A6D41E80023FB64FB6C14
:103E9000002BE5D17B681B6814337B637B6B53E895
:103EA000003F3B633B6B23F001033B667B681B6871
:103EB00014333A6E3A64FB63F96B3A6C41E80023C1
:103EC000BB63BB6B002BE5D17B681B6B012B19D14E
:103ED0007B681B680C333B623B6A53E8003FFB6125
:103EE000FB6923F01003FB657B681B680C33FA6DDC
:103EF000FA62BB62B96AFA6A41E800237B627B6AB4
:103F0000002BE5D17B681B685B6903F04003002B45
:103F100036D07B681B681433FB60FB6853E8003FB6
:103F2000BB60BB6823F04003BB657B681B68143330
:103F3000BA6DBA617B617969BA6941E800233B6176
:103F40003B69002BE5D17B68DB6B002B18D07B68CD
:103F5000DB6B00225A637B68DB6B1846FCF736FE8E
:103F60000346002B0CD07B68DB6B1846FDF7AEF9DF
:103F70000346202B04D17B6810225A6403230AE0F5
:103F80007B680022DA857B68202283F842207B68E8
:103F900000221A63002318466837BD4680BD000022
:103FA00080B5BAB000AF78607B681B681B68C7F843
:103FB000E4307B681B68DB68C7F8E0307B681B680F
:103FC0005B69C7F8DC300023C7F8D8300023C7F896
:103FD000D430D7F8E43003F00F03C7F8D830D7F85F
:103FE000D830002B0FD1D7F8E43003F02003002B9A
:103FF00009D0D7F8E03003F02003002B03D0786815
:1040000000F0B6FD5BE2D7F8D830002B00F0DE8080
:10401000D7F8DC3003F00103002B06D1D7F8E030ED
:1040200003F49073002B00F0D180D7F8E43003F054
:104030000103002B0BD0D7F8E03003F48073002B82
:1040400005D07B685B6C43F001027B685A64D7F84B
:10405000E43003F00403002B0BD0D7F8DC3003F07E
:104060000103002B05D07B685B6C43F002027B6888
:104070005A64D7F8E43003F00203002B0BD0D7F8D2
:10408000DC3003F00103002B05D07B685B6C43F050
:1040900004027B685A64D7F8E43003F00803002B6D
:1040A00011D0D7F8E03003F02003002B05D1D7F86A
:1040B000DC3003F00103002B05D07B685B6C43F020
:1040C00008027B685A647B685B6C002B00F0F2810D
:1040D000D7F8E43003F02003002B08D0D7F8E03005
:1040E00003F02003002B02D0786800F041FD7B68CC
:1040F0001B685B6903F04003002B14BF01230023FE
:10410000DBB2C7F8D4307B685B6C03F00803002B8C
:1041100003D1D7F8D430002B4FD0786800F04BFC97
:104120007B681B685B6903F04003002B41D07B6810
:104130001B681433C7F89C30D7F89C3053E8003F15
:10414000C7F89830D7F8983023F04003C7F8D0303C
:104150007B681B681433D7F8D020C7F8A820C7F8AD
:10416000A430D7F8A410D7F8A82041E80023C7F856
:10417000A030D7F8A030002BD9D17B68DB6B002BA7
:1041800013D07B68DB6B7E4A5A637B68DB6B184617
:10419000FCF758FD0346002B16D07B68DB6B5B6B8E
:1041A0007A68D26B104698470EE07868F8F7A8FB5B
:1041B0000AE07868F8F7A4FB06E07868F8F7A0FB57
:1041C0007B6800225A6475E100BF73E17B681B6B5A
:1041D000012B40F04F81D7F8E43003F01003002B9F
:1041E00000F04881D7F8E03003F01003002B00F016
:1041F00041810023BB607B681B681B68BB607B68D8
:104200001B685B68BB60BB687B681B685B6903F00D
:104210004003002B00F0B6807B68DB6B1B685B689B
:10422000A7F8BE30B7F8BE30002B00F045817B68A0
:104230009B8DB7F8BE209A4280F03E817B68B7F82C
:10424000BE20DA857B68DB6B9B69202B00F08880C1
:104250007B681B680C33C7F88830D7F8883053E880
:10426000003FC7F88430D7F8843023F48073C7F850
:10427000B8307B681B680C33D7F8B820C7F8942097
:10428000C7F89030D7F89010D7F8942041E8002371
:10429000C7F88C30D7F88C30002BD9D17B681B68DD
:1042A00014337B677B6F53E8003F3B673B6F23F022
:1042B0000103C7F8B4307B681B681433D7F8B42007
:1042C000C7F88020FB67F96FD7F8802041E800230A
:1042D000BB67BB6F002BE1D17B681B6814333B6667
:1042E0003B6E53E8003FFB65FB6D23F04003C7F8CE
:1042F000B0307B681B681433D7F8B020FA66BB6611
:10430000B96EFA6E41E800237B667B6E002BE3D129
:104310007B68202283F842207B6800221A637B6836
:104320001B680C33FB64FB6C53E8003FBB64BB6C45
:1043300023F01003C7F8AC307B681B680C33D7F848
:10434000AC20BA657B65796DBA6D41E800233B65A9
:104350003B6D002BE3D17B68DB6B1846FCF736FC2A
:104360007B6802225A637B689A8D7B68DB8D9BB2E7
:10437000D31A9BB219467868F9F7F2F99CE000BFAE
:104380007B4A01087B689A8D7B68DB8D9BB2D31AD0
:10439000A7F8CE307B68DB8D9BB2002B00F08E80BF
:1043A000B7F8CE30002B00F089807B681B680C3397
:1043B000BB63BB6B53E8003F7B637B6B23F4907361
:1043C000C7F8C8307B681B680C33D7F8C8207A64FC
:1043D0003B64396C7A6C41E80023FB63FB6B002B78
:1043E000E3D17B681B6814337B627B6A53E8003F30
:1043F0003B623B6A23F00103C7F8C4307B681B684B
:104400001433D7F8C4203A63FB62F96A3A6B41E887
:104410000023BB62BB6A002BE3D17B68202283F8B8
:1044200042207B6800221A637B681B680C333B6167
:104430003B6953E8003FFB60FB6823F01003C7F8BB
:10444000C0307B681B680C33D7F8C020FA61BB61B1
:10445000B969FA6941E800237B617B69002BE3D1EC
:104460007B6802225A63B7F8CE3019467868F9F7AC
:1044700077F923E0D7F8E43003F08003002B09D06C
:10448000D7F8E03003F08003002B03D0786800F009
:1044900008FB14E0D7F8E43003F04003002B0ED003
:1044A000D7F8E03003F04003002B08D0786800F024
:1044B00047FB04E000BF02E000BF00E000BFE837B8
:1044C000BD4680BD80B483B000AF786000BF0C37BC
:1044D000BD4680BC704780B483B000AF786000BF39
:1044E0000C37BD4680BC704780B483B000AF7860A5
:1044F00000BF0C37BD4680BC704780B483B000AFAE
:1045000078607B685B6C18460C37BD4680BC704792
:1045100080B590B000AF78607B685B6AFB637B68B6
:104520001B681B6803F02003002B37D1FB6B0022B4
:10453000DA84FB6B1B6814337B627B6A53E8003FB1
:104540003B623B6A23F08003BB63FB6B1B68143345
:10455000BA6B3A63FB62F96A3A6B41E80023BB62CB
:10456000BB6A002BE5D1FB6B1B680C333B613B69DD
:1045700053E8003FFB60FB6843F040037B63FB6B49
:104580001B680C337A6BFA61BB61B969FA6941E85F
:1045900000237B617B69002BE5D102E0F86BF9F722
:1045A00059F900BF4037BD4680BD80B584B000AF2B
:1045B00078607B685B6AFB60F868FFF783FF00BF89
:1045C0001037BD4680BD80B59CB000AF78607B6879
:1045D0005B6AFB667B681B681B6803F02003002B8B
:1045E00072D1FB6E0022DA85FB6E1B680C33FB6414
:1045F000FB6C53E8003FBB64BB6C23F48073BB6669
:10460000FB6E1B680C33BA6EBA657B65796DBA6D4B
:1046100041E800233B653B6D002BE5D1FB6E1B6839
:104620001433BB63BB6B53E8003F7B637B6B23F0AE
:1046300001037B66FB6E1B6814337A6E7A643B64FD
:10464000396C7A6C41E80023FB63FB6B002BE5D1EE
:10465000FB6E1B6814337B627B6A53E8003F3B624E
:104660003B6A23F040033B66FB6E1B6814333A6ED3
:104670003A63FB62F96A3A6B41E80023BB62BB6AAA
:10468000002BE5D1FB6E202283F84220FB6E1B6BD2
:10469000012B19D1FB6E1B680C333B613B6953E85E
:1046A000003FFB60FB6823F01003FB65FB6E1B689B
:1046B0000C33FA6DFA61BB61B969FA6941E800230C
:1046C0007B617B69002BE5D1FB6E00225A63FB6E98
:1046D0001B6B012B06D1FB6E9B8D1946F86EF9F70B
:1046E0003FF802E0F86EFFF7F6FE00BF7037BD46F8
:1046F00080BD80B584B000AF78607B685B6AFB608A
:10470000FB6801225A63FB681B6B012B08D1FB6815
:104710009B8D5B089BB21946F868F9F721F802E017
:10472000F868FFF7E1FE00BF1037BD4680BD80B5D9
:1047300084B000AF78600023FB607B685B6ABB607D
:10474000BB681B685B6903F08003002B14BF012367
:104750000023DBB2FB60BB6893F84130DBB2212B56
:1047600008D1FB68002B05D0BB680022DA84B8684A
:1047700000F0FAF8BB681B685B6903F04003002B8C
:1047800014BF01230023DBB2FB60BB6893F8423007
:10479000DBB2222B08D1FB68002B05D0BB680022BE
:1047A000DA85B86800F007F9BB685B6C43F010026B
:1047B000BB685A64B868F8F7A3F800BF1037BD4665
:1047C00080BD80B485B000AFF860B9601346FB804F
:1047D000FB68BA689A62FB68FA889A85FB68FA886F
:1047E000DA85FB6800225A64FB68222283F84220A3
:1047F000FB681B69002B07D0FB681B68DA68FB6845
:104800001B6842F48072DA60FB681B685A69FB68B7
:104810001B6842F001025A61FB681B68DA68FB689A
:104820001B6842F02002DA60002318461437BD46A8
:1048300080BC704780B598B000AFF860B96013468F
:10484000FB80BA68FB689A62FB68FA889A85FB6805
:1048500000225A64FB68222283F84220FB68DB6B4B
:104860003E4A9A62FB68DB6B3D4ADA62FB68DB6BAF
:104870003C4A1A63FB68DB6B00225A6307F10803AA
:10488000FB65FB68D86BFB681B6804331946FB6D3E
:104890001A68FB88FCF73AF900233B61FB681B6848
:1048A0001B683B61FB681B685B683B613B69FB689D
:1048B0001B69002B19D0FB681B680C333B643B6CF5
:1048C00053E8003FFB63FB6B43F48073BB65FB68FD
:1048D0001B680C33BA6DFA64BB64B96CFA6C41E8BE
:1048E00000237B647B6C002BE5D1FB681B681433D1
:1048F000FB62FB6A53E8003FBB62BB6A43F0010303
:104900007B65FB681B6814337A6DBA637B63796BD4
:10491000BA6B41E800233B633B6B002BE5D1FB689E
:104920001B681433BB61BB6953E8003F7B617B6943
:1049300043F040033B65FB681B6814333A6D7A62B1
:104940003B62396A7A6A41E80023FB61FB69002B0C
:10495000E5D1002318466037BD4680BDC745010834
:10496000F34601082F47010880B489B000AF786092
:104970007B681B680C33FB60FB6853E8003FBB603F
:10498000BB6823F0C003FB617B681B680C33FA69CA
:10499000BA617B617969BA6941E800233B613B698F
:1049A000002BE5D17B68202283F8412000BF24370B
:1049B000BD4680BC704780B495B000AF78607B681E
:1049C0001B680C337B637B6B53E8003F3B633B6BA3
:1049D00023F49073FB647B681B680C33FA6C3A64B5
:1049E000FB63F96B3A6C41E80023BB63BB6B002BA4
:1049F000E5D17B681B6814333B623B6A53E8003F98
:104A0000FB61FB6923F00103BB647B681B68143303
:104A1000BA6CFA62BB62B96AFA6A41E800237B6247
:104A20007B6A002BE5D17B681B6B012B19D17B685E
:104A30001B680C33FB60FB6853E8003FBB60BB683E
:104A400023F010037B647B681B680C337A6CBA61BB
:104A50007B617969BA6941E800233B613B69002BBE
:104A6000E5D17B68202283F842207B6800221A630C
:104A700000BF5437BD4680BC704780B584B000AFDE
:104A800078607B685B6AFB60FB680022DA85FB6804
:104A90000022DA84F868F7F733FF00BF1037BD460D
:104AA00080BD80B485B000AF78607B6893F84130FA
:104AB000DBB2212B3ED17B689B68B3F5805F14D1BC
:104AC0007B681B69002B10D17B681B6AFB60FB684D
:104AD0001B881A467B681B68C2F308025A607B6811
:104AE0001B6A9A1C7B681A6208E07B681B6A591C67
:104AF0007A6811621A787B681B685A607B68DB8C65
:104B00009BB2013B9BB27A681946D184002B0FD12E
:104B10007B681B68DA687B681B6822F08002DA60B9
:104B20007B681B68DA687B681B6842F04002DA60C9
:104B3000002300E0022318461437BD4680BC7047AE
:104B400080B582B000AF78607B681B68DA687B68EC
:104B50001B6822F04002DA607B68202283F8412043
:104B60007868F8F777FE002318460837BD4680BD01
:104B700080B58CB000AF78607B6893F84230DBB2D0
:104B8000222B40F0AE807B689B68B3F5805F17D125
:104B90007B681B69002B13D10023FB627B689B6A37
:104BA000BB627B681B685B689BB2C3F308039AB265
:104BB000BB6A1A807B689B6A9A1C7B689A6226E0B3
:104BC0007B689B6AFB620023BB627B689B68B3F5D2
:104BD000805F07D07B689B68002B0AD17B681B69CC
:104BE000002B06D17B681B685B68DAB2FB6A1A701F
:104BF00008E07B681B685B68DBB203F07F03DAB216
:104C0000FB6A1A707B689B6A5A1C7B689A627B6895
:104C1000DB8D9BB2013B9BB27A681946D185002B94
:104C20005DD17B681B68DA687B681B6822F0200214
:104C3000DA607B681B68DA687B681B6822F4807224
:104C4000DA607B681B685A697B681B6822F0010286
:104C50005A617B68202283F842207B6800225A63D5
:104C60007B681B6B012B35D17B6800221A637B6844
:104C70001B680C337B617B6953E8003F3B613B69F8
:104C800023F010037B627B681B680C337A6A3A62FC
:104C9000FB61F9693A6A41E80023BB61BB69002BFB
:104CA000E5D17B681B681B6803F01003102B0AD149
:104CB0000023FB607B681B681B68FB607B681B68CC
:104CC0005B68FB60FB687B689B8D19467868F8F72A
:104CD00047FD02E07868FFF7FEFB002302E00023B7
:104CE00000E0022318463037BD4680BD80B584B051
:104CF00000AF78607B681B681B6923F440517B68B8
:104D0000DA687B681B680A431A617B689A687B686B
:104D10001B691A437B685B691343BB607B681B6834
:104D2000DB6823F4B05323F00C037A681268B96887
:104D30000B43D3607B681B685B6923F440717B681D
:104D40009A697B681B680A435A617B681B682C4A16
:104D5000934203D1FDF75CFAF86002E0FDF744FAF4
:104D6000F860FA6813469B0013449A001A447B6863
:104D70005B689B00B2FBF3F3224AA2FB03235B09AF
:104D80001901FA6813469B0013449A001A447B6881
:104D90005B689B00B2FBF3F21A4BA3FB02035B09B7
:104DA000642000FB03F3D31A1B013233154AA2FB24
:104DB00003235B0903F0F0031944FA6813469B00D0
:104DC00013449A001A447B685B689B00B2FBF3F2C1
:104DD0000C4BA3FB02035B09642000FB03F3D31A13
:104DE0001B013233074AA2FB03235B0903F00F02C6
:104DF0007B681B680A449A6000BF1037BD4680BDBF
:104E0000003801401F85EB51002B2DE9F0471D466E
:104E1000BBBF03F100431D4600232D2388B0144679
:104E2000B8BF1446129A109E1370149BDDF84CA064
:104E300023F02008B8F1460F05D0B8F1450F00D196
:104E40000136022300E0032307AA049206AACDE953
:104E500002A2CDE9003622462B4600F0B5FEB8F19D
:104E6000470F074619D1119BDB070ED500EB06094A
:104E70000022002320462946F3F702FE08B1CDF8B0
:104E80001C903022079B4B451ED33846079B159A32
:104E9000DB1B136008B0BDE8F087B8F1460F00EBEC
:104EA0000609E5D10378302B0AD1002200232046E1
:104EB0002946F3F7E5FD18B9C6F10106CAF8006006
:104EC000DAF800309944D3E7591C07911A70D9E7F2
:104ED000F7B50029B6BF2D232B23494209290270BB
:104EE000437029DD0DF107031D460A27B1FBF7F6D4
:104EF0001A4607FB1614303402F8014C0C46632C9A
:104F0000314603F1FF33F1DC3031941E03F8011C0C
:104F10002346411CAB420AD30DF109039B1AAC4254
:104F200088BF002302330344181A03B0F0BD13F8FE
:104F3000016B01F8016FEDE7302330318370C170F0
:104F4000031DF1E72DE9F04F91B00C46DDF86880C4
:104F500016461F46054600F0FBFC036818460893FA
:104F6000F3F762F900230E93D8F800300990073365
:104F700023F0070303F1080294F818A0D4F800B056
:104F8000C8F80020D3E9008929F000430B93CDF83D
:104F900028804FF0FF32DDE90A01C4E912899C4BF9
:104FA000F3F7A0FD70BBDDE90A014FF0FF32984B2B
:104FB000F3F77AFD30BB0022002340464946F3F761
:104FC00069FD10B12D2384F84330924A924BBAF117
:104FD000470F8CBF9046984603234FF0000923618A
:104FE0002BF00403236033462146284600970FAA7E
:104FF00000F0D4F9013040F090804FF0FF3011B054
:10500000BDE8F08F42464B4640464946F3F76AFDFD
:1050100048B14B46002BB8BF2D23804AB8BF84F857
:1050200043307F4BD3E763680AF0DF015A1C3FD15E
:105030000623636000224BF48063236006920EAA6D
:10504000CDE904A20DAA03920DF13302CDE901329C
:1050500063684246009328464B460A91FFF7D4FE08
:105060000A99804647290D9928D1C81C02DB63683C
:10507000994240DDAAF1020A5FFA8AFA52460139E2
:1050800004F150000D91FFF723FF0E9A814613188B
:10509000012A236102DC2268D20701D50133236192
:1050A0009DF83330002B9ED02D2384F843309AE7AF
:1050B0004729BFD1002BBDD10123BAE7BAF1650F53
:1050C000DCD9BAF1660F18D1002963680BDD2161C4
:1050D00013B92268D00702D501330B4423614FF086
:1050E0000009A165DCE713B92268D20701D50233B4
:1050F000F4E70123F2E74FF0670A0E9B994205DBC4
:1051000023682161D807EAD54B1CE7E70029CCBF0B
:105110000122C1F102021344E0E723685A0507D4D3
:105120002369424631462846B84701302BD164E70F
:10513000BAF1650F40F2DC80D4E9120100220023AD
:10514000F3F79EFC002833D0012331462846354A28
:10515000B84701303FF451AFDDE90D38434502DB7C
:105160002368D8070FD5DDE9082331462846B8471C
:1051700001303FF442AF4FF0000908F1FF3804F16D
:105180001A0AC84509DC23689B0700F10281E06820
:105190000F9B9842B8BF184631E70123524631466B
:1051A0002846B84701303FF428AF09F10109E8E784
:1051B0000D9B002B38DC012331462846194AB8479D
:1051C00001303FF41AAFDDE90D3959EA030302D18A
:1051D0002368D907D7D5DDE9082331462846B847E3
:1051E00001303FF40AAF4FF0000A04F11A0B0D9B97
:1051F0005B42534501DC4B4693E701235A46314657
:105200002846B84701303FF4F8AE0AF1010AEEE74C
:10521000FFFFEF7F78860108748601088086010809
:105220007C86010884860108A36DDDF838A053450B
:10523000A8BF5346002B994636DC4FF0000B29EAF5
:10524000E97904F11A02A36D0A93A3EB09035B4504
:1052500031DC0D9B9A453ADC2368DA0737D40D9B85
:10526000AAEB03090A9BAAEB03039945A8BF994639
:10527000B9F1000F33DC4FF0000829EAE97904F1B5
:105280001A0B0D9BAAEB0303A3EB090343457FF71E
:105290007AAF01235A4631462846B84701303FF4D9
:1052A000ACAE08F10108ECE7424631462846B84763
:1052B0000130C2D1A1E60123314628460A92B847FF
:1052C00001303FF49AAE0A9A0BF1010BBBE731466D
:1052D000DDE908232846B8470130C0D18DE60A9A97
:1052E0004B46314628464244B8470130C3D184E694
:1052F000DDF838A0BAF1010F01DCDB0736D5012358
:10530000424631462846B84701303FF476AEDDE9E3
:10531000082331462846B84701303FF46EAED4E941
:105320001201002200230AF1FF3AF3F7A9FBC0B9EA
:10533000534608F1010231462846B84701300CD1E6
:105340005BE601235A4631462846B84701303FF410
:1053500054AE08F10108D045F3DB4B4604F150028E
:10536000E0E64FF0000804F11A0BF4E7012342468F
:10537000E1E701234A4631462846B84701303FF469
:105380003CAE08F10108E3680F995B1A4345F0DC75
:10539000FDE64FF0000804F11909F4E72DE9F047A4
:1053A000164698468A680B6907469342B8BF13466B
:1053B000336091F843200C46DDF820900AB10133A8
:1053C00033602368990642BF33680233336025682F
:1053D00015F0060506D104F1190AE36832689B1A34
:1053E000AB422BDC94F843302268003B18BF01230A
:1053F000920630D44146384604F14302C847013092
:1054000023D02368226903F00603042B14BF002570
:1054100033684FF0000608BFE56804F11A0408BFBE
:10542000ED1A54F8123C08BF25EAE5759342C4BF53
:105430009B1AED18B5421AD1002008E0012352460C
:1054400041463846C847013003D14FF0FF30BDE830
:10545000F0870135C1E73020E11881F843005A1C7C
:1054600094F845102244023382F84310C2E7012326
:10547000224641463846C8470130E6D00136D9E7D2
:105480002DE9FF470F7E9146782F80460C469A46BD
:105490000C9E01F1430207D8622F0AD8002F00F0BA
:1054A000D180582F00F0B88004F1420684F8427091
:1054B0003AE0A7F16303152BF6D801A151F823F0C8
:1054C000195501082D550108A9540108A9540108CE
:1054D000A9540108A95401082D550108A95401082F
:1054E000A9540108A9540108A95401082B56010820
:1054F00057550108E5550108A9540108A9540108A8
:105500004D560108A954010857550108A95401082E
:10551000A9540108ED55010833681A1D1B68326053
:1055200004F1420684F8423001239CE0336820688D
:10553000191D3160060601D51D6803E04506FBD53F
:10554000B3F90050002D03DA2D236D4284F8433067
:105550000A23584811E021683368080653F8045BB1
:1055600002D4490648BFADB26F2F336014BF0A237F
:1055700008235048002184F843106668002EA66076
:1055800005DB21682E4321F0040121604BD0164633
:10559000B5FBF3F103FB1157C75D06F8017D2F46FC
:1055A000BB420D46F4D9082B0BD12368DF0708D581
:1055B000236961689942DEBF302306F8013C06F199
:1055C000FF36921B22614B4621464046CDF800A093
:1055D00003AAFFF7E3FE01304AD14FF0FF3004B0D9
:1055E000BDE8F087236843F0200323607827324822
:1055F00084F84570236831681F0651F8045B02D4B3
:105600005F0648BFADB23160D90744BF43F0200305
:1056100023601DB11023ADE72648E9E7236823F096
:1056200020032360F6E71646BDE733682568181D9A
:10563000616930602E061B6801D5196002E06806BA
:10564000FBD51980002316462361BCE7336800218F
:105650001A1D32601E686268304600F0F0F908B129
:10566000801B606063682361002384F84330AAE7ED
:105670003246494640462369D0470130ADD02368C1
:105680009B0713D4E068039B9842B8BF1846A6E76F
:105690000123324649464046D04701309DD001356E
:1056A000E36803995B1AAB42F2DCEBE7002504F1F7
:1056B0001906F5E78686010897860108002310B5CC
:1056C0000446C0E90033C0E9043383608181436646
:1056D000C2818361194608225C3000F031F90D4B1C
:1056E000246263620C4BA3620C4BE3620C4B23639A
:1056F0000C4B9C4206D003F16802944202D0D03396
:105700009C4205D104F15800BDE8104000F094B966
:1057100010BD00BF41580108635801089B5801089B
:10572000BF580108BC140020024A0349034800F096
:1057300069B800BF9000002011740108A00000208B
:1057400041680C4B10B59942044601D001F060FE4F
:10575000A168094B994202D0204601F059FEE16848
:10576000064B994204D02046BDE8104001F050BEDF
:1057700010BD00BFBC140020241500208C15002093
:1057800010B50B4B0B4C0C4A20461A60042100222A
:10579000FFF794FF04F1680001220921FFF78EFF53
:1057A00004F1D0000222BDE810401221FFF786BFAD
:1057B000F4150020BC14002029570108014800F00E
:1057C0003CB900BFFD150020014800F037B900BF0B
:1057D000FD15002010B50446FFF7F0FF236A1BB14A
:1057E000BDE81040FFF7F0BF044B2362044B1B6879
:1057F000002BF5D1FFF7C4FFF2E700BF41570108C6
:10580000F41500202DE9F843074688461446002683
:10581000D4E90195B9F1010905D52468002CF7D127
:105820003046BDE8F883AB89012B07D9B5F90E30B6
:10583000013303D029463846C04706436835E9E7B7
:1058400010B50C46B1F90E1000F0A8F80028ABBF57
:10585000636DA3891B1823F48053ACBF6365A381D8
:1058600010BD2DE9F0411F468B890546DB050C462E
:10587000164605D502230022B1F90E1000F07CF87F
:10588000A389324623F48053A38128463B46B4F9CA
:105890000E10BDE8F04100F093B810B50C46B1F918
:1058A0000E1000F069F8431CA38915BF606523F44E
:1058B000805343F48053A38118BFA38110BDB1F975
:1058C0000E1000F049B830B51446002C05461A46B3
:1058D0009BB005DA8B2303604FF0FF301BB030BD67
:1058E0004FF40273ADF80C304FF0000319930CBF66
:1058F000234604F1FF33029305934FF6FF730091A3
:105900000491ADF80E3069461E9B01F005FC431C66
:10591000BCBF8B232B60002CE0D00022009B1A70B0
:10592000DCE7000007B5009313460A46014603482A
:105930000068FFF7C8FF03B05DF804FB9C0000207F
:1059400003460244934200D1704703F8011BF9E774
:1059500000487047DC01002038B50023054D04469F
:1059600008462B60F8F7A3FD431C02D12B6803B156
:10597000236038BDF815002038B5044608461146A6
:105980000022054D2A601A46F8F7B5FD431C02D1E6
:105990002B6803B1236038BDF815002038B50446E4
:1059A000084611460022054D2A601A46F8F762FDA6
:1059B000431C02D12B6803B1236038BDF8150020C9
:1059C00038B50446084611460022054D2A601A469D
:1059D000F4F7E4FC431C02D12B6803B1236038BD0B
:1059E000F8150020014B1868704700BF9C0000208C
:1059F00070B500260C4D0D4C641BA410A64209D1B5
:105A000002F076F800260A4D0A4C641BA410A64248
:105A100005D170BD55F8043B98470136EEE755F8BF
:105A2000043B98470136F2E7F4890108F48901083C
:105A3000F4890108F88901087047704770470346E8
:105A400010B5C9B202449342184601D1002003E0C8
:105A5000047801338C42F6D110BD0A44914200F122
:105A6000FF3300D1704710B511F8014B914203F894
:105A7000014FF9D110BD00001FB514461A46094B5D
:105A800005461B68D8684CB1074BCDE9013400913D
:105A90002B46064901F0E4FC01F01EFD044B1C46B8
:105AA000F3E700BF9C000020A8860108B586010826
:105AB000E38601082DE9F74F03690C690746A34205
:105AC0007EDB013CA30000F1140501F114080093F2
:105AD00005EB8403019358F8243055F82420013352
:105AE0009A42B2FBF3F608EB84092ED34FF0000A7A
:105AF000C446AE46D3465CF8043B98B206FB00A011
:105B00001B0C020C06FB0323DEF8002080B292B2CD
:105B1000121A5A44DEF800004FEA134A9BB2C3EB54
:105B2000224303EB104392B242EA0342E1454FEABB
:105B3000234B4EF8042BDED2009BEB582BB9019B74
:105B4000043B9D421A462FD33C61384601F080F950
:105B5000002825DB2946002058F8042BD1F800C086
:105B60001FFA82FE1FFA8CF3A3EB0E030344120C00
:105B7000C2EB234202EB1C429BB243EA0243C14503
:105B80004FEA224041F8043BE6D255F8242005EBC9
:105B9000840322B9043B9D421A460BD33C61013673
:105BA000304603B0BDE8F08F1268043B002ACBD129
:105BB000013CC6E71268043B002AEFD1013CEAE74A
:105BC0000020EEE7000000002DE9F04F14461D46CE
:105BD000C76997B08146CDE90645239E7FB910205D
:105BE00000F00EFE0246C9F81C0020B9EF21AC4BB4
:105BF000AC48FFF741FFC0E901770760C760D9F8FB
:105C00001C30196859B15A68012393404A608B606F
:105C1000484600F0EBFE0022D9F81C301A602B1E1B
:105C2000AFBF0023012223F000430793A8BF3360D6
:105C3000DDF81C809C4BB8BF326033EA080312D1F8
:105C400042F20F73229A1360C8F31303234300F048
:105C50005E85249BDFF854A2002B00F060850AF1DA
:105C6000030300F05ABDDDE90623CDE90C23DDE98D
:105C70000C0100220023F2F703FF074658B101236D
:105C8000229A1360249B13B1894B249A1360DFF886
:105C900024A200F044BD14AB019315AB0093484619
:105CA000DDE90C2301F084F9C8F30A560390002EB5
:105CB00078D0DDE90C010D9BA6F2FF36C3F3130388
:105CC00043F07F5343F440131297194600227A4B56
:105CD000F2F7B6FA6CA3D3E90023F2F769FC6CA3E0
:105CE000D3E90023F2F7AEFA044630460D46F2F748
:105CF000F5FB69A3D3E90023F2F75AFC02460B46F1
:105D000020462946F2F79EFA04460D46F2F700FFB8
:105D100000220746002320462946F2F7BBFE40B189
:105D20003846F2F7DBFB22462B46F2F7A9FE00B914
:105D3000013F162F54D8DDE90C01604B03EBC7037C
:105D4000D3E90023F2F7A6FE00284BD00023013F41
:105D50000F93149B9B1B5A1E49BFC3F101030023E1
:105D600004930023099254BF04930993002F3BDB53
:105D7000099B0E973B44099300230A93209B092B10
:105D800065D8052BC4BF043B2093209BC8BF0024CB
:105D9000A3F10203D8BF0124032B64D8DFE803F08A
:105DA0005355382CDDE914631E4406F23243202B90
:105DB000C1BFC3F1400308FA03F806F2124324FA04
:105DC00003F3D6BFC3F1200348EA030004FA03F04B
:105DD000F2F774FB0122A1F1F873013E129274E70D
:105DE0000123B5E70F90B4E7049BDB1B04937B42D0
:105DF0000A9300230E93C1E701230B93219B07EB2A
:105E0000030B0BF10103012B0893B8BF012306E03C
:105E100001230B93219B002B28DD9B460893002137
:105E20000422D9F81C0002F114059D4226D94160D4
:105E3000484600F09BFD8246002843D1024640F2CE
:105E4000AF111F4BD4E60023E3E70023D5E701247D
:105E500000230B9420934FF0FF3B00221223CDF838
:105E600020B02192DBE701230B93F4E74FF0010B05
:105E70005B46CDF820B0CDF884B0D0E701315200B8
:105E8000D1E700BFAFF3008061436F63A787D23FC4
:105E9000B3C8608B288AC63FFB799F501344D33F19
:105EA000F1860108088701080000F07FED860108EF
:105EB00085860108848601080000F83F20880108D3
:105EC00060870108D9F81C301860089B0E2B00F27F
:105ED000A180002C00F09E80002F33DD9C4B07F04A
:105EE0000F0203EBC203F805D3E90034CDE9103407
:105EF0004FEA271416D5DDE90C01964B0326D3E9AA
:105F00000823F2F77FFCCDE9060104F00F04914D60
:105F100054B9DDE91023DDE90601F2F773FCCDE9A0
:105F2000060128E00226F2E7E10708D5DDE91001C5
:105F3000D5E90023F2F73CFBCDE9100101366410EE
:105F40000835E5E700F0AF80DDE90C017C42804BCD
:105F500004F00F0203EBC203D3E90023F2F728FB9E
:105F600002260023CDE906017A4D2411002C40F0D1
:105F70008F80002BD3D1DDE906450F9B002B00F06D
:105F80009480002220462946734BF2F783FD0028B7
:105F900000F08B80089B002B00F08780BBF1000F86
:105FA00034DD2046002229466C4BF2F701FB5C46AB
:105FB000CDE9060107F1FF3801363046F2F78EFAD7
:105FC000DDE90623F2F7F4FA0022654BF2F73AF91D
:105FD0000546A1F15076002C6AD1DDE906010022C8
:105FE000604BF2F72DF902460B46CDE906232A460F
:105FF0003346F2F76DFD002840F09882DDE9060196
:106000002A4606F10043F2F745FD38BBDDE90C34C2
:10601000CDE90634159B002BC0F257810E2F00F3FB
:1060200054814B4B03EBC703D3E90034CDE904346F
:10603000219B002B80F2E580089B002B00F3E18080
:106040000CD1DDE904010022464BF2F7B1FADDE99B
:106050000623F2F733FD002800F06682002425466F
:10606000219B56466FEA030800272146484600F068
:10607000BDFC002D00F0BD802FB1AF4203D03946EA
:10608000484600F0B3FC2946484600F0AFFCB0E0BB
:10609000E20705D5D5E90023F2F78AFA0123013694
:1060A0006410083562E7022665E7B846089C84E775
:1060B000274B0B9903EBC40353E9022354440029F3
:1060C00054D000202849F2F79DFB33462A46F2F7C8
:1060D000B7F85646CDE91001DDE90601F2F718FDE3
:1060E0000546F2F7FBF902460B46DDE90601F2F739
:1060F000A7F802460B463035CDE90623DDE910232B
:1061000006F8015BF2F7C6FC002872D1DDE9062330
:1061100000201149F2F794F8DDE91023F2F7BAFCF8
:10612000002840F0B480A6423FF470AFDDE91001D2
:1061300000220A4BF2F73CFA0022CDE91001DDE91A
:106140000601064BF2F734FACDE90601C4E700BFB9
:1061500020880108F88701080000F03F0000244073
:1061600000001C40000014400000E03F314628467B
:10617000F2F71EFA5646CDE910011394DDE9060147
:10618000F2F7C6FC0546F2F7A9F902460B46DDE92F
:106190000601F2F755F802460B46303506F8015B6A
:1061A000A642CDE906234FF0000224D1DDE910011B
:1061B000AE4BF2F747F802460B46DDE90601F2F76F
:1061C00087FC002863D1DDE910230020A749F2F7FE
:1061D00037F802460B46DDE90601F2F75BFC0028C2
:1061E0003FF414AF139E731E139316F8013C302B2B
:1061F000F8D047463BE09E4BF2F7DAF9CDE90601CD
:10620000BCE75646DDE90645DDE90423204629467C
:10621000F2F7F8FAF2F77CFC8046F2F75FF9DDE975
:106220000423F2F7C5F902460B4620462946F2F749
:1062300007F808F13004089D06F8014BA6EB0A04A4
:10624000A54202460B4633D1F1F7FCFFDDE90423FA
:1062500004460D46F2F73CFCC0B9DDE904232046B4
:106260002946F2F70DFC10B118F0010F0ED1484687
:10627000039900F0BBFB00233370229B01371F60A2
:10628000249B002B00F04B821E6048E2B846334648
:106290001E4613F8012D392A06D19A45F8D130222D
:1062A00008F101088AF800201A7801321A70A0E774
:1062B00000226F4BF2F77CF90022002304460D46C2
:1062C000F2F7DEFB00289FD0D1E70B9A002A00F0FE
:1062D000EA80209A012A00F3CD80129A002A00F069
:1062E000C18003F233430A9C049E049A01211A449C
:1062F0000492099A48461A44099200F02BFC05467C
:1063000066B1099B002B09DDB342A8BF3346049A4E
:10631000F61AD21A0492099AD31A09930A9B0BB35C
:106320000B9B002B00F0C680002C00F0C08029469B
:106330002246484600F0C6FC039A014605464846F8
:1063400000F01EFC03998046484600F04FFB0A9B74
:106350001B1B0A9300F0B18041460A9A484600F0A0
:10636000B1FC03900121484600F0F4FB0E9B04466B
:10637000002B00F0D8811A460146484600F0A2FCE6
:10638000209B0446012B00F39F80069B002B40F0CE
:106390009780079BC3F31303002B40F09380079B68
:1063A00023F000431B0D1B0533B1049B0133049301
:1063B000099B0133099301230A930E9B002B00F0E4
:1063C000B881236904EB8303186900F077FBC0F1FF
:1063D0002000099B184410F01F0000F08280C0F1DB
:1063E0002003042B73DD049BC0F11C0003440493C1
:1063F000099B064403440993049B002B05DD1A46C0
:106400004846039900F0B8FC0390099B002B05DD7A
:1064100021461A46484600F0AFFC04460F9B002B6D
:1064200061D02146039800F013FD00285BDA0023B9
:106430000A224846039900F0FBFA0B9B07F1FF384C
:106440000390002B00F07781294600230A2248465A
:1064500000F0EEFABBF1000F05466FDC209B022B2B
:1064600049DC6BE0149BC3F136033CE70000E03FDE
:1064700000002440089B5C1E0A9BA34209DB1C1BF6
:10648000089B002BBFF630AF049B089A9E1A00238E
:106490002BE70A9B0E9AE31A1A440A94049E0024DE
:1064A000089B0E9221E70A9C049E0B9D28E7DDF8CD
:1064B0000C8051E70A9A039950E7CDF80C8051E718
:1064C000002379E7069B77E700230A9379E793D0C7
:1064D000049A1C331A440492099A1E441A440992DD
:1064E0008AE70346F4E7089BB846002B20DC9B466E
:1064F000209B022B1EDDBBF1000F7FF4B1AD2146C6
:106500005B460522484600F093FA0146044603988C
:1065100000F09EFC00287FF7A3AD5646312308F11A
:10652000010806F8013B9FE5B846089C2546F4E7BC
:10653000DDF820B00B9B002B00F00181002E05DD63
:1065400029463246484600F017FC05460A9B002BB8
:106550005CD04846696800F009FA064628B9024648
:1065600040F2EF21804BFFF743BB2A6905F10C0194
:10657000023292000C30FFF770FA01223146484691
:1065800000F0FAFB2F4605460AF1010304930AEBDB
:106590000B030A93069B03F001030993049B214616
:1065A000039803F1FF3BFFF785FA03463946303382
:1065B000069003980B9300F04BFC2A460890214666
:1065C000484600F061FCC26806460B9B02BB0146D0
:1065D000039800F03DFC02460B9B31464846CDE94E
:1065E0000B3200F003FA209B0C9A049E42EA03014E
:1065F000099B19430B9B0DD1392B27D0089A002AF0
:1066000001DD069B31338BF800302EE52846B9E7D3
:106610000122E2E70899002904DB20980143099848
:10662000014320D1002AEEDD01220399484604935C
:1066300000F0A2FB2146039000F00AFC0028049B16
:1066400002DCE0D1DA07DED5392BDAD139238BF839
:10665000003033461E4616F8012C013B392A4ED035
:1066600001321A7001E5002A03DD392BEED0013327
:10667000C9E7049A0A9902F8013C8A4228D000230B
:106680000A220399484600F0D3F9AF4203904FF035
:1066900000034FF00A023946484607D100F0C8F916
:1066A00007460546049B0133049377E700F0C0F9E1
:1066B0002946074600230A22484600F0B9F9054654
:1066C000F0E7BBF1000FCCBF5E4601260027564421
:1066D000012203994846049300F04EFB21460390A3
:1066E00000F0B6FB0028B4DC02D1049BDB07B0D479
:1066F00033461E4613F8012D302AFAD0B5E49A45E8
:10670000A8D1312308F101088AF80030ADE4249BB8
:10671000DFF858A01BB10AF10803249A1360504611
:1067200017B0BDE8F08F209B012B7FF72EAE0E9B9C
:106730000A9301204DE6BBF1000F7FF7D9AE564614
:1067400021460398FFF7B6F900F1300306F8013B44
:10675000A6EB0A029345B4DD00230A2248460399BA
:1067600000F066F90390EBE760870108E486010812
:1067700038B50546002940D051F8043C0C1F002BC9
:10678000B8BFE41800F0E6F81C4A136833B9636038
:1067900014602846BDE8384000F0E2B8A34208D9AA
:1067A000206821188B4201BF19685B6809182160B5
:1067B000EDE71A465B680BB1A342FAD9116850188D
:1067C000A0420BD120680144501883421160E0D1EF
:1067D00018685B68084410605360DAE702D90C233C
:1067E0002B60D6E7206821188B4201BF19685B68CF
:1067F0000918216063605460CBE738BD041600209F
:10680000024B0146186800F025B800BF9C0000202C
:1068100070B50F4E0C463168054611B900F04CFEBC
:1068200030602146284600F047FE431C03D14FF05C
:10683000FF34204670BDC41C24F00304A042F8D0ED
:10684000211A284600F038FE0130F2D1EFE700BFF0
:10685000001600202DE9F843CD1C25F0030508356E
:106860000C2D38BF0C25002D064601DBA94204D9AA
:106870000C2333600020BDE8F883DFF8D48000F0FB
:1068800069F8D8F800301C4644BB29463046FFF76B
:10689000BFFF431C044658D1D8F800402746002FBC
:1068A00043D1002C4BD023683946304604EB030912
:1068B00000F002FE814542D1216830466D1A29461A
:1068C000FFF7A6FF01303AD023682B442360D8F8A5
:1068D00000305A6862BBC8F800700FE02268521B93
:1068E00020D40B2A17D96119A342256018BF59601B
:1068F000636808BFC8F8001062514B60304600F072
:106900002FF804F10B00231D20F00700C21A1CBF52
:106910001B1AA350AFE76268A3420CBFC8F800205F
:106920005A60EBE723466468AEE73C467F68B6E70B
:106930001A465B68A342FBD100235360DEE70C23B9
:106940003046336000F00CF894E70560D6E700BFEE
:10695000041600200148FFF770B800BFFC150020A6
:106960000148FFF76BB800BFFC15002070B5C66981
:1069700004460D4676B91020FFF742FF0246E0615B
:1069800020B96B21174B1848FFF776F8C0E901666C
:106990000660C660E669F36883B1E369DB6853F8B3
:1069A0002500B8B9012101FA05F6721D20469200B2
:1069B00000F099FD60B1C0E901560EE021220421EA
:1069C000204600F090FDE369F060DB68002BE4D125
:1069D000002070BD026843F825200023C0E903337E
:1069E000F7E700BFF18601087187010870B5C66935
:1069F00005460C4676B91020FFF702FF0246E86113
:106A000020B98F21084B0948FFF736F8C0E9016625
:106A10000660C6603CB1EB696268DB6853F822101F
:106A2000216043F8224070BDF1860108718701089A
:106A30002DE9F04107460C461E4600200D6901F184
:106A4000140CDCF80030013099B202FB01611E0C1D
:106A50000B0C02FB063389B201EB034185424FEA7E
:106A600013464CF8041BECDC0EB3A368AB4219DCF4
:106A7000616838460131FFF779FF804628B9024640
:106A8000BA210C4B0C48FEF7F7FF226904F10C0108
:106A9000023292000C30FEF7E0FF21463846FFF745
:106AA000A5FF444604EB850301355E612561204660
:106AB000BDE8F08160870108718701080346B0F5E1
:106AC000803F3ABF030410200020B3F1807F3CBF19
:106AD0001B020830B3F1805F3CBF1B010430B3F1EF
:106AE000804F3CBF9B000230002B05DB13F0804F32
:106AF00000F1010008BF202070470368024613F030
:106B000007000BD0D90721D4980749BF5B089B0821
:106B1000012013605CBF02201360704799B209B96D
:106B200010201B0CD9B209B908301B0A190704BF81
:106B30001B090430990704BF9B080230D90703D40E
:106B40005B0800F1010003D013607047002070471C
:106B50002020704710B50C460121FFF707FF0246C1
:106B600028B940F24511044B0448FEF785FF012384
:106B70004461036110BD00BF60870108718701088F
:106B80002DE9F04F17460A693B6989469A42A2BF30
:106B90003B460F4699463D69D9F810A0BB68796815
:106BA00005EB0A06B34285B0B8BF0131FFF7DEFE40
:106BB00030B902464FF4B171404B4148FEF75CFFDB
:106BC00000F114042346002204EB860E734520D303
:106BD00007F1140809F1140108EB850501EB8A039C
:106BE0000293EB1B153B23F0030304331537BD421F
:106BF00038BF04230193029B03918B420CD8002ED3
:106C000003DD5EF8043D002B55D0066105B0BDE8FC
:106C1000F08F43F8042BD9E7B1F800A0BAF1000FC8
:106C20001FD0C446A14600275CF8042BD9F80030D9
:106C30001FFA82FB9BB20AFB0B333B44D9F800706E
:106C4000120C3F0C0AFB027202EB13429BB243EAA6
:106C5000024365454FEA124749F8043BE4D8019BDB
:106C6000E750039B0431B3F80290B9F1000F20D034
:106C70004746A4464FF0000A2368B7F800B0BCF8B6
:106C800002209BB209FB0B22524443EA02434CF818
:106C9000043B57F8043B4FEA134ABCF80030BD42AE
:106CA00009FB0A3303EB12434FEA134AE5D8019A72
:106CB000A35004349FE7013EA1E700BF60870108AD
:106CC000718701082DE9F843154612F003020746C3
:106CD0000E4607D0254C013A002354F82220FFF736
:106CE000A7FE0646AD103DD0FC697CB91020FFF729
:106CF00087FD0246F86128B940F2B3111C4B1D48CC
:106D0000FEF7BAFEC0E901440460C460D7F81C80F5
:106D1000D8F808404CB940F271213846FFF71AFF05
:106D200000230446C8F8080003604FF00009EB0791
:106D30000AD5314622463846FFF722FF80463146C3
:106D40003846FFF753FE46466D100BD0206838B921
:106D5000224621463846FFF713FF2060C0F8009016
:106D60000446E4E73046BDE8F88300BFE887010841
:106D7000F1860108718701082DE9F0470C460746A6
:106D800091462369496803EB6218A3684FEA621AC7
:106D900008F10106B3420BDB3846FFF7E7FD054675
:106DA00048B902464FF4EF71274B2848FEF764FEBE
:106DB00001315B00EEE7002300F1140100F1100245
:106DC0001846534533DB20692AEAEA7A04F11403B2
:106DD00019F01F0901EB8A0103EB800C2BD08A46C6
:106DE0000022C9F1200E186800FA09F010434AF891
:106DF000040B53F8042B9C4522FA0EF2F3D8ACEBAB
:106E00000403153B23F00303043304F1150060452C
:106E100088BF0423CA500AB108F10206013E384671
:106E200021462E61FFF7E2FD2846BDE8F08742F8D3
:106E3000040F0133C5E7043953F8042B9C4541F88E
:106E4000042FF9D8EAE700BF6087010871870108BD
:106E500003460A69006930B5801A0ED11433143123
:106E600003EB820401EB820154F8045D51F8042D18
:106E7000954203D005D24FF0FF3030BDA342F3D38B
:106E8000FBE70120F9E700002DE9F74F89460646A8
:106E9000114648461446FFF7DBFF051E12D129466E
:106EA0003046FFF763FD024628B940F237213E4BDA
:106EB0003E48FEF7E1FD0123C0E90435104603B06A
:106EC000BDE8F08FBCBF4B46A1463046D9F8041050
:106ED000BABF1C4601250025FFF748FD024618B938
:106EE00040F24521304BE3E700F1140BD9F8107064
:106EF00009F11003C5604FF0000C09F11405D946E3
:106F0000266904F1140E05EB87080EEB8606019343
:106F1000019B5EF8040B53F804AF81B201931FFA92
:106F20008AF35B1A000C6344C0EB1A4000EB234069
:106F30009BB243EA004376454FEA204C49F8043BB4
:106F4000E6D8331B153B23F0030315340433A64264
:106F500038BF04231D445B441E462C4644450ED3D3
:106F600008F10301491B21F00301033DA84538BF87
:106F700000210B4453F8041D99B117619EE7E646C2
:106F800054F8041B1FFA81FCF444080C714400EB14
:106F90002C4089B241EA00414FEA204C46F8041BDC
:106FA000DCE7013FE6E700BF608701087187010861
:106FB0002DE97343012190469946089EFFF7D6FCC0
:106FC000044630B9024640F20F31234B2348FEF706
:106FD00053FDC9F30A55C9F313030DB143F48013EC
:106FE0000193B8F1000324D068460093FFF785FDB4
:106FF000DDE90012D8B1C0F1200302FA03F30B431C
:10700000C24063610192019B002B0CBF012202224E
:10701000A3612261ADB1A5F2334505443560C0F1ED
:107020003500099B1860204602B0BDE8708361619D
:10703000E9E701A8FFF761FD019B012263612030B0
:10704000E7E7A0F2324004EB820330601869FFF7F3
:1070500035FDC0EB4210E4E7608701087187010845
:107060002DE9F0471F468E688246BE420C46904688
:107070000B682DD8B1F90C2012F4906F26D06569F9
:10708000096905EB4505A3EB010905EBD5757B1CEB
:107090004B446D109D4238BF1D46530527D52946E8
:1070A000FFF7D8FB064660B34A462169FEF7D5FCD8
:1070B000A38923F4906343F08003A38126614E44A7
:1070C00026603E466561A5EB0905A560BE4200D974
:1070D0003E4632464146206800F0D4F90020A368BD
:1070E0009B1BA360236833442360BDE8F0872A46D6
:1070F00000F01FFA06460028E0D150462169FFF74C
:1071000037FB0C23CAF80030A3894FF0FF3043F05F
:107110004003A381E9E700002DE9F04F98468B89F1
:1071200007461B060D4614469DB010D50B6973B972
:107130004021FFF78FFB2860286130B90C233B60AA
:107140004FF0FF301DB0BDE8F08F40236B6100238E
:10715000099320238DF8293030234FF00109CDF811
:107160000C80DFF898818DF82A3023469A4613F870
:10717000012B0AB1252AF9D1BAEB040B0BD05B46DF
:10718000224629463846FFF76BFF013000F0A78002
:10719000099A5A4409929AF80030002B00F09F8017
:1071A00000234FF0FF32CDE905230AF1010A0493D1
:1071B00007938DF853301A935446052214F8011B97
:1071C0004E48FEF73CFC049AD8B9D00644BF2023B1
:1071D0008DF85330110744BF2B238DF853309AF8A4
:1071E00000302A2B15D0544600204FF00A0C079A85
:1071F000214611F8013B303B092B4BD9B0B1079226
:1072000014E0A0EB080309FA03F31343A246049326
:10721000D2E7039B191D1B680391002BBBBF5B4288
:1072200042F0020207930793B8BF049223782E2BF3
:107230000AD163782A2B32D1039B02341A1D1B68B2
:10724000039243EAE3730593DFF8B4A003225046A8
:107250002178FEF7F4FB38B14022049BA0EB0A0032
:10726000824013430134049314F8011B062225487D
:107270008DF82810FEF7E3FB002836D0224B1BBB0D
:10728000039B073323F0070308330393099B33441D
:1072900009936AE70C4601200CFB0232A8E70023A1
:1072A0004FF00A0C194601340593204610F8012BC3
:1072B000303A092A03D9002BC6D00591C4E7044609
:1072C00001230CFB0121F0E703AB00932A4638466B
:1072D0000E4B04A9FDF736FE421C0646D6D1AB89FB
:1072E0005B063FF52DAF09982CE703AB00932A46C8
:1072F0003846064B04A9FEF7C3F8EDE7CA87010834
:10730000D0870108D4870108454F01086170010842
:10731000B1F90C20F8B5160705460C4654D44B6855
:10732000002B02DC0B6C002B48DDE66A002E45D0FA
:10733000002312F480522F68216A2B6030D0626DD6
:10734000A389590705D56368D21A636B0BB1236C07
:10735000D21A00232846E66A216AB047431CA38953
:1073600006D129681D292BD8284ACA40D60727D517
:10737000002262602269D904226004D5421C01D136
:107380002B6803B96065616B2F60B9B104F14403E8
:10739000994202D02846FFF7EBF9002363630DE022
:1073A00001232846B0470246501CC9D12B68002B48
:1073B000C6D01D2B01D0162B1DD12F60002021E03F
:1073C00043F040031BB21AE00F69002FF6D0930779
:1073D00018BF00230E6808BF4B69F61B0F608B6057
:1073E000002EEBDD33463A462846216AD4F828C001
:1073F000E047002807DCB4F90C3043F040034FF0BD
:10740000FF30A381F8BD0744361AE9E701004020A8
:1074100038B50B6905460C4613B90025284638BD1A
:1074200018B1036A0BB9FEF7D5F9B4F90C30002B8B
:10743000F3D0626ED00704D4990502D4A06DFEF794
:10744000FCFA28462146FFF763FF636E0546DA071C
:10745000E4D4A3899B05E1D4A06DFEF7EFFADDE744
:107460000EB403B5014603AB054853F8042B00687E
:10747000019300F0C1F802B05DF804EB03B070476F
:107480009C000020884210B501EB020402D984421E
:10749000234607D8431EA14208D011F8012B03F858
:1074A000012FF8E7014602448A4200D110BD13F8CB
:1074B000014D02F8014DF7E738B50023054D0446AC
:1074C00008462B60F7F724F8431C02D12B6803B160
:1074D000236038BDF8150020062008B500F060FADA
:1074E0000120F6F7BCFF70B5A1FB025434B9294660
:1074F000FFF7B0F9064628B9304670BD0C220026C9
:107500000260F9E72A462146FEF71AFAF4E782B04C
:1075100001B901A942B14BB113780B601278101E6A
:1075200018BF012002B070471046FBE76FF0010062
:10753000F8E72DE9F041074614460D4621B91146FA
:10754000BDE8F041FFF786B92AB9FFF711F92546E2
:107550002846BDE8F08100F03FFA8442064602D892
:10756000B4EB500FF4D821463846FFF773F9804644
:1075700008B94546ECE7B4422246294628BF3246C0
:10758000FEF76BFA29463846FFF7F2F8F1E70346B3
:10759000084641B1FF2A04D98A224FF0FF301A6011
:1075A000704701200A707047936810B4013B002BAC
:1075B000936007DA9469A34201DB0A2902D110BC67
:1075C00000F032B91368581C10601970084610BCDE
:1075D0007047F8B506460F461446D518AC4201D19F
:1075E000002007E03A46304614F8011BFFF7DCFFA5
:1075F000431CF3D1F8BD00002DE9F04F0D461446B1
:10760000984606469DB018B1036A0BB9FEF7E2F83A
:107610006B6ED90705D4AB899A0502D4A86DFEF725
:107620000CFAAB891B0701D52B699BB9294630465B
:1076300000F038F970B16B6EDC0704D54FF0FF3005
:107640001DB0BDE8F08FAB899805F7D4A86DFEF7A3
:10765000F5F9F3E70023099320238DF8293030232F
:107660004FF00109CDF80C80DFF8A8818DF82A30A1
:1076700023469A4613F8012B0AB1252AF9D1BAEB11
:10768000040B0BD05B46224629463046FFF7A1FF8C
:10769000013000F0A780099A5A4409929AF8003004
:1076A000002B00F09F8000234FF0FF32CDE905232F
:1076B0000AF1010A049307938DF853301A93544644
:1076C000052214F8011B5348FEF7B9F9049AD8B9FA
:1076D000D10644BF20238DF85330130744BF2B231A
:1076E0008DF853309AF800302A2B15D054460020DC
:1076F0004FF00A0C079A214611F8013B303B092B49
:107700004BD9B0B1079214E0A0EB080309FA03F3D8
:107710001343A2460493D2E7039B191D1B680391F0
:10772000002BBBBF5B4242F0020207930793B8BF36
:10773000049223782E2B0AD163782A2B32D1039B13
:1077400002341A1D1B68039243EAE3730593DFF8C2
:10775000C8A0032250462178FEF771F938B14022C3
:10776000049BA0EB0A00824013430134049314F8F5
:10777000011B062229488DF82810FEF760F9002821
:107780003FD0274B1BBB039B073323F00703083372
:107790000393099B3B4409936AE70C4601200CFBC9
:1077A0000232A8E700234FF00A0C19460134059372
:1077B000204610F8012B303A092A03D9002BC6D0F5
:1077C0000591C4E7044601230CFB0121F0E703AB5C
:1077D00000932A463046134B04A9FDF7B3FB074636
:1077E000781CD6D16B6ED90705D4AB899A0502D423
:1077F000A86DFEF723F9AB895B063FF51FAF09982B
:107800001EE703AB00932A463046064B04A9FDF75A
:1078100037FEE4E7CA870108D0870108D48701084A
:10782000454F0108D3750108F8B50E4614460546C4
:1078300018B1036A0BB9FDF7CDFFA369A360A38953
:107840001A0701D5236943B92146284600F02AF8D2
:1078500018B14FF0FF373846F8BD23682269F6B2F9
:10786000981A63693746834205DC21462846FFF7AC
:10787000CFFD0028EDD1A368013BA36023685A1C0B
:1078800022601E706269431C9A4204D0A389DB0700
:10789000E1D50A2EDFD121462846FFF7B9FD0028A1
:1078A000D9D0D6E738B5294B054618680C4618B12B
:1078B000036A0BB9FDF78EFFB4F90C30190722D417
:1078C000DA0607D409222A6043F040034FF0FF3064
:1078D000A38133E0580712D5616B41B104F1440331
:1078E000994202D02846FEF743FF00236363A38931
:1078F00023F02403A3810023636023692360A38909
:1079000043F00803A38123694BB9A38903F42073CF
:10791000B3F5007F03D02146284600F08AF8B4F979
:107920000C3013F001020AD00022A26062695242B8
:10793000A261226942B913F08000C5D138BD990710
:1079400058BF6269A260F4E70020F7E79C000020BE
:107950001F2938B505460C4604D9162303604FF09D
:10796000FF3038BDC26B12B152F821304BB92846F6
:1079700000F030F8224601462846BDE8384000F0C5
:1079800017B8012B0AD0591C03D11623036001201C
:10799000E7E70021204642F8241098470020E0E75E
:1079A000024B01461868FFF7D3BF00BF9C000020C0
:1079B00038B50023064D0446084611462B60F6F7FD
:1079C0003EFD431C02D12B6803B1236038BD00BFCC
:1079D000F8150020F6F72CBD51F8043C181F002BB9
:1079E000BCBF0B58C018704770B50C46B1F90E10EB
:1079F000154600291E4696B00CDAA389002113F023
:107A0000800F14BF40234FF48063002031602B604F
:107A100016B070BD6A4600F049F80028EDDB019908
:107A200001F47041A1F50053594259414FF480636C
:107A3000EBE78B89F7B59D0706460C4607D504F1A1
:107A40004703236023610123636103B0F0BD6A46ED
:107A500001ABFFF7C9FF009F054639463046FEF7E8
:107A6000F9FE48B9B4F90C309A05EED423F00303BB
:107A700043F00203A381E2E7A389C4E9040743F0CA
:107A80008003A381019B20605BB13046B4F90E10E6
:107A900000F01EF828B1A38923F0030343F001038B
:107AA000A381A3891D43A581CFE7000038B500233A
:107AB000064D0446084611462B60F6F703FD431CAD
:107AC00002D12B6803B1236038BD00BFF815002038
:107AD00038B50023054D044608462B60F6F701FD36
:107AE000431C02D12B6803B1236038BDF815002078
:107AF000F8B500BFF8BC08BC9E467047F8B500BF9B
:087B0000F8BC08BC9E4670476A
:107B0800434F4E4E30204572726F723A2025640AF8
:107B180000000000436F6E6E6563746F723A205503
:107B28006E6B6E6F776E0A00436F6E6E6563746F6F
:107B3800723A20556E706C75676765640A000000BC
:107B4800436F6E6E6563746F723A20446973616245
:107B58006C65640A00000000436F6E6E6563746FA5
:107B6800723A20507265706172696E670A0000008F
:107B7800436F6E6E6563746F723A20417574685214
:107B8800657175697265640A00000000436F6E6E66
:107B98006563746F723A2057616974696E67466FDE
:107BA80072456E657267790A00000000436F6E6E59
:107BB8006563746F723A204368617267696E6750D3
:107BC800617573656445560A00000000436F6E6E68
:107BD8006563746F723A204368617267696E6750B3
:107BE8006175736564455653450A0000436F6E6EB0
:107BF8006563746F723A204368617267696E670AD9
:107C080000000000436F6E6E6563746F723A204126
:107C180075746854696D656F75740A00436F6E6E8C
:107C28006563746F723A2046696E69736865640AA1
:107C380000000000436F6E6E6563746F723A2046F1
:107C4800696E6973686564455653450A000000000B
:107C5800436F6E6E6563746F723A2046696E69731E
:107C680068656445560A0000436F6E6E6563746FFD
:107C7800723A205265706C756767696E670A000012
:107C88004350207374617465206368616E6765642E
:107C98003A202564202D3E2025640A0043502064A4
:107CA800757479206368616E6765643A202575206C
:107CB8002D3E2025750A00004649524520414C4179
:107CC800524D206163746976617465640A0000002E
:107CD80046617374206469736368617267652074B0
:107CE8007269676765722025752D3E257520493DA7
:107CF80025750A004661737420646973636861724C
:107D0800676520636F6D706C6574652C20563D2522
:107D1800750A000046617374206469736368617250
:107D280067652061626F727465642C20563D257505
:107D38000A000000434353206D6F64756C6520731F
:107D4800746172740A00000053657269616C206E78
:107D5800756D6265723A2025640A0000426F61728F
:107D680064207265766973696F6E3A2025640A002B
:107D780046572076657273696F6E3A2025642E2502
:107D8800642E25640A000000505355206F6E20743D
:107D9800696D656F75740A00436F6E746163746F03
:107DA80072206572726F722C2073746F7070696EB6
:107DB800672E2E2E0A0000004661737420646973D2
:107DC8006368617267652061626F7274202D3E205E
:107DD80073746F700A0000004661737420646973DD
:107DE800636861726765206F66662061636B2C202B
:107DF800563D2575202D3E207365742025750A0093
:107E08004661737420646973636861726765206F83
:107E180066662074696D656F75742C20563D2575EE
:107E28000A000000466173742064697363686172B4
:107E38006765206F6E2074696D656F75742C2056A8
:107E48003D25752028746172676574202575290A97
:107E580000000000505355206F66662074696D65F8
:107E68006F75740A00000000504520004E45200040
:107E7800464520004F52452000000000444D412057
:107E8800000000005541525425752048414C20659A
:107E980072726F72206465636F64653A204E4F4E4C
:107EA800450A00005541525425752048414C20652B
:107EB80072726F72206465636F64653A202573255A
:107EC800732573257325732573207261773D307888
:107ED8002530386C780A00005541525433205258E6
:107EE8002061726D206661696C656420282573299C
:107EF8003A2048414C5F5374617475733D25642082
:107F08006572725F61667465723D30782530386CD1
:107F1800780A000055415254332052582061726D3E
:107F2800206661696C65642064657461696C7300BE
:107F380055415254332052582064726F703A20775A
:107F4800726F6E6720687561727420696E2052784E
:107F58004576656E7443616C6C6261636B2028734F
:107F6800697A653D2575290A00000000554152547B
:107F7800332052582064726F703A205278457665E3
:107F88006E742073697A653D30202869646C652CAD
:107F9800206E6F207061796C6F6164290A0000009F
:107FA80052784576656E7443616C6C6261636B00F0
:107FB80055415254332052582064726F703A2073DE
:107FC800697A653D2575203E2072785F6275666620
:107FD800657220257520286F766572666C6F772C20
:107FE800206E6F7420706172736564290A00000046
:107FF8005541525425752048414C206572726F7264
:108008002028495352293A207261773D307825302B
:10801800386C7820E28094205258206D6179206273
:108028006520636F7272757074656420756E74690B
:108038006C2072652D61726D0A0000004572726FC6
:108048007243616C6C6261636B000000554152546D
:108058003320545820444D4120726573656E642066
:108068006661696C656400004553544F5020747212
:10807800696767657265640A0000000053746F7071
:1080880070696E67206368617267696E672E2E2E4D
:108098000A00000046696E697368656445562C20BD
:1080A80073746F7070696E672E2E2E0A00000000C0
:1080B800457665726573742074696D656F75740AA9
:1080C80000000000457665726573742074696D65FB
:1080D8006F75742C2073746F7070696E6720636895
:1080E800617267696E672E2E2E0A000043686172FE
:1080F80067696E67206572726F722025642C207321
:1081080074617465202D3E2064697361626C6564D6
:108118000A0000004368617267696E6720706572C3
:108128006D69747465642C2073746172742063685B
:10813800617267696E670A0043617220756E706CC0
:1081480075676765640A00005265706C75676769D2
:108158006E672E2E2E0A00005265706C756767696F
:108168006E672066696E69736865642C2062757431
:108178002063617220756E706C75676765640A00AC
:108188005265706C756767696E672066696E69739A
:108198006865642C2063617220706C75676765641C
:1081A8002C207374617465202D3E206175746820DD
:1081B80072657175697265640A000000496E6974B8
:1081C8000000000043435320696E69740A000000F0
:1081D800554152543320545820444D412073746102
:1081E8007274206661696C6564000000457665728A
:1081F80065737420726573657420636F6D6D616E4D
:10820800640A000055415254332052582077617255
:108218006E3A20636D6420307825303278204352DE
:10822800432F6C656E204F4B20627574206E6F2053
:108238007377697463682063617365202865787053
:1082480065637465645F7061796C6F6164207673CF
:10825800206170706C795F636F6D6D616E64290A5F
:108268000000000055415254332052582064726F68
:10827800703A20746F6F5F73686F7274206C656EEC
:108288003D302028656D707479206368756E6B29A0
:108298000A00000055415254332052582064726F2E
:1082A800703A20746F6F5F73686F7274206C656EBC
:1082B8003D312062303D3078253032780A000000A8
:1082C80055415254332052582064726F703A2074CA
:1082D8006F6F5F73686F7274206C656E3D322062D9
:1082E800303D3078253032782062313D3078253085
:1082F80032780A0055415254332052582064726F24
:10830800703A206372635F6D69736D61746368208E
:10831800636D643D30782530327820746F74616CF9
:108328005F6C656E3D2575207061796C6F61645F67
:108338006C656E3D2575206372635F72783D307899
:1083480025303478206372635F63616C633D3078F5
:10835800253034780A0000005541525433205258D1
:108368002064726F703A20756E6B6E6F776E5F6304
:108378006D6420636D643D30782530327820746FE9
:1083880074616C5F6C656E3D2575207061796C6FEA
:1083980061645F6C656E3D25750A00005541525455
:1083A800332052582064726F703A206C656E5F6D8E
:1083B80069736D6174636820636D643D307825303E
:1083C80032782065787065637465645F7061796C74
:1083D8006F61643D257520676F745F7061796C6F9C
:1083E80061643D257520746F74616C5F6C656E3DCA
:1083F80025750A005761746368646F6700000000A0
:108408005541525433207761746368646F672072F2
:108418006561726D0000000025733A206572723D37
:1084280030782530386C7820673D256C7520727857
:108438003D256C752074785F627573793D25750AE2
:108448000000000055415254322052582069646C93
:1084580065206576656E742077697468207A657220
:108468006F2073697A650A00554152543220525878
:1084780020696E76616C6964207061636B65742035
:108488006C656E3D25750A00554152543520525889
:108498002069646C65206576656E742077697468F8
:1084A800207A65726F2073697A650A0055415254C3
:1084B8003520525820696E76616C6964207061635A
:1084C8006B6574206C656E3D25750A0055415254E4
:1084D8003220545820627573792C2061626F72744F
:1084E800207472616E736D6974206265666F72655F
:1084F80020726573656E640A00000000554152548D
:108508003220545820444D4120737461727420669F
:1085180061696C656400000055415254322052581C
:10852800207061636B65742074696D656F75742064
:10853800282575206D73290A000000005541525402
:108548003220525820444D412061726D2066616985
:108558006C656400554152543520525820495420C6
:1085680061726D206661696C656400005541525402
:1085780032207265636F766572207374617274005D
:108588005541525435207265636F76657220737455
:108598006172740025733A20696E7374616E636545
:1085A8003D30782530386C78206572723D307825FA
:1085B80030386C7820673D256C752072783D256CC5
:1085C800750A000053657420436F6E6669673A2028
:1085D80025732025640A0000506F776572206C6946
:1085E8006D69743A2025640A0000000043686172CE
:1085F8006765207065726D69743A2025640A000009
:1086080001000100010001000100040001002C002C
:108618000100000000000000000000000102030447
:108628000607080900000000010203040000040511
:108638000607080900000000000D000001020304FD
:1086480005060708090A0B0C0D0E0F10000004059B
:108658000607080900000000000D000001020304DD
:1086680005060708090A0B0C0D0E0F10494E4600A7
:10867800696E66004E414E006E616E00300030310A
:108688003233343536373839414243444546003071
:1086980031323334353637383961626364656600A0
:1086A8002C2066756E6374696F6E3A20006173736F
:1086B800657274696F6E2022257322206661696C69
:1086C80065643A2066696C6520222573222C206C2B
:1086D800696E65202564257325730A00496E6669ED
:1086E8006E697479004E614E005245454E54206DB6
:1086F800616C6C6F632073756363656564656400A2
:108708002F6275696C642F676E752D746F6F6C734B
:108718002D666F722D73746D33325F31332E332EA5
:1087280072656C312E32303234303932362D313771
:1087380031352F7372632F6E65776C69622F6E65A2
:10874800776C69622F6C6962632F7374646C6962F9
:108758002F64746F612E630042616C6C6F632073C9
:108768007563636565646564002F6275696C642F61
:10877800676E752D746F6F6C732D666F722D7374C1
:108788006D33325F31332E332E72656C312E3230B9
:108798003234303932362D313731352F7372632FF9
:1087A8006E65776C69622F6E65776C69622F6C698C
:1087B80062632F7374646C69622F6D707265632EC7
:1087C8006300232D302B2000686C4C0065666745DC
:1087D8004647004300504F534958002E0000000000
:1087E80005000000190000007D00000000000000E6
:1087F8000080E03779C34143176E05B5B5B8934695
:10880800F5F93FE9034F384D321D30F94877825A60
:108818003CBF737FDD4F1575000000000000F03F7E
:108828000000000000002440000000000000594043
:108838000000000000408F40000000000088C34096
:1088480000000000006AF8400000000080842E410B
:1088580000000000D01263410000000084D7974157
:108868000000000065CDCD41000000205FA002425D
:10887800000000E876483742000000A2941A6D42D2
:10888800000040E59C30A2420000901EC4BCD642C5
:1088980000003426F56B0C430080E03779C3414370
:1088A80000A0D8855734764300C84E676DC1AB43E6
:1088B800003D9160E458E143408CB5781DAF154404
:1088C80050EFE2D6E41A4B4492D54D06CFF08044DF
:1088D800F64AE1C7022DB544B49DD9794378EA44F4
:1088E8000020202020202020202028282828282078
:1088F8002020202020202020202020202020202070
:1089080020881010101010101010101010101010D7
:1089180010040404040404040404041010101010C7
:108928001010414141414141010101010101010191
:1089380001010101010101010101010110101010E3
:108948001010424242424242020202020202020263
:1089580002020202020202020202020210101010B7
:1089680020000000000000000000000000000000DF
:1089780000000000000000000000000000000000EF
:1089880000000000000000000000000000000000DF
:1089980000000000000000000000000000000000CF
:1089A80000000000000000000000000000000000BF
:1089B80000000000000000000000000000000000AF
:1089C800000000000000000000000000000000009F
:1089D800000000000000000000000000000000008F
:0489E800000000008B
:0889EC003CF8FE7F01000000D1
:0489F4000D820008E8
:0489F800E981000809
:1089FC00E40100000606060601000000FA00000A69
:108A0C00050A050000000000FF00000A0A0A0A001F
:108A1C0000000000400000320A320040000000005C
:108A2C00008000320A320000800000000000FF0AC3
:108A3C000A0A0A000000000000FF00320A3200009F
:108A4C0020000000FFFFFF320A3200FFFFFF000092
:108A5C00FF0000320A3200200000640000FFFF001B
:108A6C00000000000000000052555301000000FE01
:108A7C00529E66000024F40010000000010000006B
:108A8C000000000003000000BC140020A000002027
:108A9C0000000000BC140020241500208C150020C0
:108AAC0000000000000000000000000000000000BA
:108ABC0000000000000000000000000000000000AA
:108ACC00000000000000000000000000000000009A
:108ADC000000000000000000000000004300000047
:108AEC00000000000000000000000000000000007A
:108AFC000000000000000000000000004300000027
:108B0C000000000000000000000000000000000059
:108B1C000000000000000000000000004300000006
:108B2C000000000000000000000000000000000039
:108B3C0000000000000000000000000043000000E6
:108B4C000000000000000000000000000000000019
:108B5C0000000000000000000000000043000000C6
:108B6C0000000000000000000000000000000000F9
:108B7C0000000000000000000000000043000000A6
:108B8C0000000000000000000000000000000000D9
:108B9C000000000000000000000000004300000086
:108BAC0000000000000000000000000000000000B9
:108BBC000000000000000000000000008F7501089C
:108BCC000F75010800000000E8880108E387010820
:108BDC00E3860108E3860108E3860108E3860108C1
:108BEC00E3860108E3860108E3860108E3860108B1
:108BFC00E3860108FFFFFFFFFFFFFFFFFFFFFFFF03
:108C0C00FFFF0000010041534349490000000000F0
:108C1C000000000000000000000000000000000048
:108C2C0000000000000041534349490000000000CF
:108C3C000000000000000000000000000000000028
:088C4C00000000000000000020
:040000050800EE49B8
:00000001FF
